:020000040000FA
:0400000035EF01F0E7
:100008005482D9CF05F0DACF06F00F0112A90FEF0D
:1000180000F011EF00F04EEF00F08EBC16EF00F08C
:1000280018EF00F01AEF00F0839483928EA81FEF68
:1000380000F021EF00F028EF00F083A226EF00F097
:1000480028EF00F03EEF00F0899425EE04F0010E51
:10005800DBBE38EF00F0000EDE5C020EDE58D8A0E2
:1000680038EF00F03AEF00F03DEF00F089923EEFF4
:1000780000F089828EA843EF00F045EF00F04DEFC5
:1000880000F083B24AEF00F04CEF00F04DEF00F0C3
:100098008984129912A153EF00F055EF00F02DEF6B
:1000A80001F08EA85AEF00F05CEF00F063EF00F06B
:1000B80083A261EF00F063EF00F064EF00F0899233
:1000C8009050FF0A096E8E50FF0A086E04C50AF0A8
:1000D80005C50BF00BBE7AEF00F0020E0B5CD8B032
:1000E80078EF00F07AEF00F0A6EF00F00A4A0B2A4A
:1000F8000AC004F50BC005F502C50AF003C50BF0EC
:10010800060E0A24D96E050E0B20DA6E09C0DFFF31
:10011800060E0A24D96E070E0B20DA6E08C0DFFF20
:100128000A4A0B2AFF0E016E010E026E0AC003F086
:100138000BC004F0015003160250041603C002F568
:1001480004C003F58EA8ABEF00F0ADEF00F0B4EFFC
:1001580000F083A2B2EF00F0B4EF00F0B5EF00F0CA
:10016800898489848EA0BBEF00F0BDEF00F0B6EF64
:1001780000F08EA8C2EF00F0C4EF00F0CBEF00F063
:1001880083A2C9EF00F0CBEF00F0CEEF00F0899426
:10019800CFEF00F0898425EE04F0010EDBBEDEEF20
:1001A80000F0000EDE5C020EDE58D8A0DEEF00F094
:1001B800E0EF00F0E3EF00F08992E4EF00F08982CD
:1001C80008A8E9EF00F0EBEF00F02BEF01F006EFE5
:1001D80001F0838283942BEF01F0838483922BEFC9
:1001E80001F083922BEF01F083942BEF01F083A2AF
:1001F80000EF01F002EF01F02BEF01F083948392FE
:100208002BEF01F00950016E026A0250000AD8B4BF
:1002180010EF01F02BEF01F00150040AD8B4FBEF06
:1002280000F0100AD8B4FBEF00F0340AD8B4EDEFB0
:1002380000F01F0AD8B4F5EF00F07F0AD8B4F1EF48
:1002480000F01F0AD8B4F8EF00F02BEF01F00F010F
:1002580012910E01CA9906C0DAFF05C0D9FF54925F
:10026800110003EF60F084C0D9FF85C0DAFF000EEB
:10027800DE6E000EDD6E86C00CF087C00DF051EC0E
:1002880059F00CC0C1F00DC0C2F00001C2BF51EF5F
:1002980001F04FEF01F054EF01F00B0EF4EF09F00D
:1002A800D890C135D96EC235DA6E7E0ED926010EC8
:1002B800DA22DECFDBF0DDCFDCF0DB51DC11D8A4B5
:1002C80068EF01F06AEF01F06DEF01F00C0EF4EF4A
:1002D80009F084C0D9FF85C0DAFFDBC0DEFFDCC0CF
:1002E800DDFFDBC0D9FFDCC0DAFFDF50D8B47FEF19
:1002F80001F081EF01F0A8EF01F020EE01F0DB51F1
:10030800D926DC51DA22DF505DEC6FF00001CD6FA9
:10031800CDB191EF01F093EF01F0A8EF01F0885112
:10032800D8B499EF01F09BEF01F0A5EF01F0CDA54E
:10033800A0EF01F0A2EF01F0A5EF01F00A0EF4EF33
:1003480009F0000EF4EF09F0DBC0D9FFDCC0DAFFDA
:10035800000EDF6E20EE01F0DB51D926DC51DA22E7
:10036800C1C0DFFF20EE01F0DB51D926DC51DA22D3
:10037800DF5090EC48F00001CD6FCDA1C6EF01F041
:10038800C8EF01F0CBEF01F0030EF4EF09F088514C
:10039800D8B4D1EF01F0D3EF01F0DCEF01F0CDA537
:1003A800D8EF01F0DAEF01F0DCEF01F0A2EF01F095
:1003B800000ED46F000ED56F000ED66F000ED76FEB
:1003C800DBC060F0DCC061F0000E626F000E636F8E
:1003D800000E646F000E656F57EC4BF00001DA6F8A
:1003E800DA05D8B4FAEF01F0FCEF01F0FEEF01F006
:1003F8001AEF03F0000ED96F000ED86FD95109E13A
:10040800040ED85DD8A00BEF02F00DEF02F00FEF4D
:1004180002F0B7EF02F0D8C089F0D9C08AF0893B62
:100428008A3BF00E8A1789510F0B8A13F00E891731
:10043800DBC08BF0DCC08CF089518B278A518C2370
:10044800EC0E8B25CE6F010E8C21CF6F20EE04F0C1
:10045800CE51D926CF51DA22DF50D8A436EF02F098
:1004680038EF02F042EF02F0000EB36F000EB46FE7
:10047800000EB56F000EB66F9BEF02F020EE09F08C
:10048800CE51D926CF51DA22DF50896F89518B6F2F
:100498008A6B20EE0AF0CE51D926CF51DA22DF50EE
:1004A8008C6F8CC08DF08E6B8F6B906B8EC090F0C4
:1004B8008DC08FF08E6B8D6B20EE0BF0CE51D92650
:1004C800CF51DA22DF50916F91C092F0936B946B09
:1004D800956B92C095F0946B936B926B8D519211C2
:1004E800966F8E519311976F8F519411986F905109
:1004F8009511996F8A5196119A6F8B5197119B6F2D
:10050800000E98119C6F000E99119D6F20EE08F057
:10051800CE51D926CF51DA22DF509E6F9E519A11C3
:10052800B36F9B51B46F9C51B56F9D51B66FA30EBD
:10053800896F000E8A6FD890D835D96ED935DA6EA2
:10054800D890D936DA368951D9268A51DA22B3C0F9
:10055800DEFFB4C0DEFFB5C0DEFFB6C0DEFFD84B9D
:10056800D92B02EF02F0000ED96F000ED86FD851C8
:10057800D911D8B4C2EF02F0C4EF02F0C7EF02F00D
:10058800D807D8A0D907A30E896F000E8A6FD89014
:10059800D835D96ED935DA6ED890D936DA36895148
:1005A800D9268A51DA22DECFD4F0DECFD5F0DECFDD
:1005B800D6F0DECFD7F0D451D511D611D711D8A4A3
:1005C800E8EF02F0EAEF02F0F0EF02F0000EB86F89
:1005D800020EB76F03EF03F0DBC060F0DCC061F020
:1005E800D4C062F0D5C063F0D6C064F0D7C065F05F
:1005F80057EC4BF00001896F8951B76FB86BB7C0E2
:10060800DAF0DA51D8B40BEF03F00DEF03F01AEF7C
:1006180003F0D84BD92BD95109E1040ED85DD8A0E5
:1006280018EF03F01AEF03F0C7EF02F0030EDA1920
:10063800D8A421EF03F023EF03F026EF03F0010E17
:10064800F4EF09F0DA51D8B42CEF03F02EEF03F0F1
:1006580031EF03F00D0EF4EF09F020EE3AF0DB5124
:10066800D926DC51DA22DF50896F89518B6F8A6B6A
:1006780020EE39F0DB51D926DC51DA22DF508C6FBD
:100688008C518A13000E8B13020E8B198A11D8B461
:1006980050EF03F052EF03F054EF03F02EEF03F0A6
:1006A80020EE45F0DB51D926DC51DA22DF50896F84
:1006B80089518B6F8A6B20EE44F0DB51D926DC51CF
:1006C800DA22DF508C6F8C518A13000E8B138AC08C
:1006D800D0F08BC0D1F0D26BD36BD051D111D211E5
:1006E800D311D8A47AEF03F07CEF03F0D5EF03F031
:1006F80020EE53F0DB51D926DC51DA22DF50896F26
:1007080089518B6F8A6B20EE54F0DB51D926DC516E
:10071800DA22DF508C6F8CC08DF08E6B8F6B906BF4
:100728008EC090F08DC08FF08E6B8D6B20EE55F0E3
:10073800DB51D926DC51DA22DF50916F91C092F05B
:10074800936B946B956B92C095F0946B936B926BD3
:100758008D519211966F8E519311976F8F519411FD
:10076800986F90519511996F8A5196119A6F8B5184
:1007780097119B6F000E98119C6F000E99119D6F39
:1007880020EE52F0DB51D926DC51DA22DF509E6F81
:100798009E519A11D06F9B51D16F9C51D26F9D5130
:1007A800D36F20EE16F0DB51D926DC51DA22D0C007
:1007B800DEFFD1C0DEFFD2C0DEFFD3C0DEFF20EEF9
:1007C8003EF0DB51D926DC51DA2210EE03F0DB5182
:1007D800E126DC51E222DFCFE7FF20EE03F0DB5118
:1007E800D926DC51DA22DE04D8B4FDEF03F0FFEF9E
:1007F80003F010EF04F020EE03F0DB51D926DC51B2
:10080800DA22020EDE18D8B40CEF04F00EEF04F072
:1008180010EF04F02EEF03F0D0C00CF0D1C00DF0B3
:10082800D2C00EF0D3C00FF020EE03F0DB51D92672
:10083800DC51DA22DF50896F8951106E116A126A11
:10084800136A1AEC6AF00CC0D0F00DC0D1F00EC0DB
:10085800D2F00FC0D3F0000120EE3BF0DB51D926D7
:10086800DC51DA2210EE02F0DB51E126DC51E22203
:10087800DFCFE7FF20EE02F0DB51D926DC51DA2288
:10088800DF50D8B44AEF04F04CEF04F02EEF03F039
:10089800FF0E896FFF0E8A6F20EE02F0DB51D9261A
:1008A800DC51DA22DF508B6F8C6B89518B278A5190
:1008B8008C2320EE02F0DB51D926DC51DA22DF50FE
:1008C8008D6F8D518B17000E8C178B518C11D8B4EE
:1008D80070EF04F072EF04F074EF04F02EEF03F001
:1008E80020EE40F0DB51D926DC51DA22DF50896F47
:1008F80089518B6F8A6B20EE3FF0DB51D926DC5192
:10090800DA22DF508C6F8C518A13000E8B1320EE85
:1009180008F0DB51D926DC51DA228AC0DEFF8BC011
:10092800DDFF20EE08F0DB51D926DC51DA22DECFDC
:1009380089F0DDCF8AF00F0E8917000E8A178951CA
:100948008A11D8B4AAEF04F0ACEF04F0AEEF04F0CB
:100958002EEF03F020EE42F0DB51D926DC51DA22EB
:10096800DF50896F89518B6F8A6B20EE41F0DB5124
:10097800D926DC51DA22DF508C6F8C518A13000E95
:100988008B138AC0C5F08BC0C6F0C76BC86BC55146
:10099800C611C711C811D8A4D4EF04F0D6EF04F0DB
:1009A8002FEF05F020EE4FF0DB51D926DC51DA228B
:1009B800DF50896F89518B6F8A6B20EE50F0DB51C5
:1009C800D926DC51DA22DF508C6F8CC08DF08E6B0B
:1009D8008F6B906B8EC090F08DC08FF08E6B8D6B8F
:1009E80020EE51F0DB51D926DC51DA22DF50916F2D
:1009F80091C092F0936B946B956B92C095F0946B49
:100A0800936B926B8D519211966F8E519311976FD4
:100A18008F519411986F90519511996F8A51961131
:100A28009A6F8B5197119B6F000E98119C6F000E57
:100A380099119D6F20EE4EF0DB51D926DC51DA2258
:100A4800DF509E6F9E519A11C56F9B51C66F9C5186
:100A5800C76F9D51C86F20EE3CF0DB51D926DC51A1
:100A6800DA22DF50896F20EE3DF0DB51D926DC51C8
:100A7800DA22DF508A6F8951C36F8AC0C4F0C3512C
:100A8800C411D8A44AEF05F04CEF05F04EEF05F07D
:100A98002EEF03F020EE08F0DB51D926DC51DA22E4
:100AA800DECF89F0DDCF8AF0040E8B6FD8908A33C1
:100AB80089338B2F5AEF05F0C35189258C6FC451A8
:100AC8008A218D6F8E6BD8B08E2B8F6BD0518C2571
:100AD800BD6FD1518D21BE6FD2518E21BF6FD351C1
:100AE8008F21C06FBD51C55DBE51C659BF51C75991
:100AF800C051C859D8B083EF05F085EF05F087EFEE
:100B080005F02EEF03F0BD51C55D0C6EBE51C65900
:100B18000D6EBF51C7590E6EC051C8590F6E20EEE9
:100B280002F0DB51D926DC51DA22DF50896F895176
:100B3800106E116A126A136A30EC67F00CC0C9F0C3
:100B48000DC0CAF00EC0CBF00FC0CCF00001C951E7
:100B5800CA11CB11CC11D8A4B4EF05F0B6EF05F04B
:100B6800B8EF05F02EEF03F0010EDA6FCC51CB1180
:100B78000BE1F60EC95D0F0ECA59D8A0C6EF05F0F5
:100B8800C8EF05F0CAEF05F0020EDA6FCC51CB11B1
:100B98000BE1F60EC95DFF0ECA59D8A0D6EF05F0D5
:100BA800D8EF05F0DAEF05F0030EDA6F020EC9256B
:100BB800896F000ECA218A6F000ECB218B6F000E41
:100BC800CC218C6F20EE12F0DB51D926DC51DA22D1
:100BD80089C0DEFF8AC0DEFF8BC0DEFF8CC0DEFF6F
:100BE80020EE1AF0DB51D926DC51DA22D4C0DEFF20
:100BF800D5C0DEFFD6C0DEFFD7C0DEFFC351D42587
:100C0800896FC451D5218A6F000ED6218B6F000ED3
:100C1800D7218C6F20EE1EF0DB51D926DC51DA2269
:100C280089C0DEFF8AC0DEFF8BC0DEFF8CC0DEFF1E
:100C3800BD51D425896FBE51D5218A6FBF51D621A8
:100C48008B6FC051D7218C6F20EE26F0DB51D9264F
:100C5800DC51DA2289C0DEFF8AC0DEFF8BC0DEFFEE
:100C68008CC0DEFF030EDA19D8A43DEF06F03FEF83
:100C780006F0D8EF06F020EE08F0DB51D926DC515B
:100C8800DA22DE50DE10D8B44CEF06F04EEF06F054
:100C980050EF06F02EEF03F020EE5BF0DB51D92683
:100CA800DC51DA22DF50896F89518B6F8A6B20EE15
:100CB8005CF0DB51D926DC51DA22DF508C6F8CC016
:100CC8008DF08E6B8F6B906B8EC090F08DC08FF017
:100CD8008E6B8D6B20EE5DF0DB51D926DC51DA226C
:100CE800DF50916F91C092F0936B946B956B92C0AB
:100CF80095F0946B936B926B8D519211966F8E5108
:100D08009311976F8F519411986F90519511996F16
:100D18008A5196119A6F8B5197119B6F000E9811FB
:100D28009C6F000E99119D6F20EE5AF0DB51D92669
:100D3800DC51DA22DF509E6F9E519A119F6F9B51B2
:100D4800A06F9C51A16F9D51A26F20EE22F0DB5144
:100D5800D926DC51DA229FC0DEFFA0C0DEFFA1C089
:100D6800DEFFA2C0DEFF20EE12F0DB51D926DC51F7
:100D7800DA22DECF89F0DECF8AF0DECF8BF0DECF4D
:100D88008CF0020ED89089378A378B378C37E82E4B
:100D9800C6EF06F089C0B9F08AC0BAF08BC0BBF0C4
:100DA8008CC0BCF077EF07F020EE08F0DB51D926B5
:100DB800DC51DA22DE50DE10D8A4E5EF06F0E7EFCA
:100DC80006F0E9EF06F02EEF03F020EE1EF0DB51FF
:100DD800D926DC51DA22DECF89F0DECF8AF0DECFE9
:100DE8008BF0DECF8CF0D05189258D6FD1518A21BF
:100DF8008E6FD2518B218F6FD3518C21906F20EE43
:100E080022F0DB51D926DC51DA228DC0DEFF8EC0FC
:100E1800DEFF8FC0DEFF90C0DEFF020EDA19D8B405
:100E280018EF07F01AEF07F060EF07F020EE12F066
:100E3800DB51D926DC51DA22DECF89F0DECF8AF009
:100E4800DECF8BF0DECF8CF0010E89158D6F000E92
:100E58008A158E6F000E8B158F6F000E8C15906F94
:100E680020EE12F0DB51D926DC51DA22DECF0CF06D
:100E7800DECF0DF0DECF0EF0DECF0FF0030E106EDA
:100E8800000E116E000E126E000E136E1AEC6AF050
:100E9800D8900F320E320D320C3200018D510C24D5
:100EA800B96F8E510D20BA6F8F510E20BB6F9051C4
:100EB8000F20BC6F77EF07F020EE12F0DB51D92638
:100EC800DC51DA22DECF89F0DECF8AF0DECF8BF07C
:100ED800DECF8CF0D8908935B96F8A35BA6F8B35EB
:100EE800BB6F8C35BC6FFF0EB925896F010EBA2117
:100EF8008A6F000EBB218B6F000EBC218C6F0A0E0F
:100F08008BEF07F0D8908C338B338A338933E82EF4
:100F180086EF07F020EE16F0DB51D926DC51DA22F5
:100F28008951DE5C8A51DE588B51DE588C51DE586F
:100F3800D8B0A1EF07F0A3EF07F0A5EF07F02EEF69
:100F480003F020EE0EF0DB51D926DC51DA22FF0E39
:100F5800DE6EFF0EDE6EFF0EDE6EFF0EDD6EDD5204
:100F6800DD5210EE0AF0DB51E126DC51E222DECF41
:100F7800E6FFDECFE6FFDECFE6FFDECFE6FF20EEC0
:100F880005F0DB51D926DC51DA22800EDF6E030E24
:100F9800DA19D8A4D2EF07F0D4EF07F0DEEF09F0A2
:100FA80020EE5FF0DB51D926DC51DA22DF50896F61
:100FB80089518B6F8A6B20EE5EF0DB51D926DC51AC
:100FC800DA22DF508C6F8C518A13000E8B138A053E
:100FD8008B11D8A4F2EF07F0F4EF07F0DEEF09F079
:100FE800DBC03AF0DCC03BF0010ED4253C6E000EAD
:100FF800D5213D6E000ED6213E6E000ED7213F6EE4
:10100800AFEC64F00009D8A40CEF08F00EEF08F07C
:10101800DEEF09F0000120EE05F0DB51D926DC51A6
:10102800DA22000EDF6E22EE2DF0DB51D926DC51DC
:10103800DA22DF50896F89518B6F8A6B22EE2CF090
:10104800DB51D926DC51DA22DF508C6F8C518A13A0
:10105800000E8B13550E8A1907E1AA0E8B19D8A416
:1010680038EF08F03AEF08F0DEEF09F020EE2FF045
:10107800DB51D926DC51DA22DF50896F89518B6F19
:101088008A6B20EE30F0DB51D926DC51DA22DF50B2
:101098008C6F8CC08DF08E6B8F6B906B8EC090F0C8
:1010A8008DC08FF08E6B8D6B20EE31F0DB51D92621
:1010B800DC51DA22DF50916F91C092F0936B946B00
:1010C800956B92C095F0946B936B926B8D519211C6
:1010D800966F8E519311976F8F519411986F90510D
:1010E8009511996F8A5196119A6F8B5197119B6F31
:1010F800000E98119C6F000E99119D6F20EE2EF036
:10110800DB51D926DC51DA22DF509E6F9E519A11AD
:101118009F6F9B51A06F9C51A16F9D51A26F520E62
:101128009F190DE1520EA0190AE1610EA11907E1FC
:10113800410EA219D8A4A3EF08F0A5EF08F0DEEF3E
:1011480009F022EE13F0DB51D926DC51DA22DF5008
:10115800896F89518B6F8A6B22EE14F0DB51D92687
:10116800DC51DA22DF508C6F8CC08DF08E6B8F6B68
:10117800906B8EC090F08DC08FF08E6B8D6B22EED1
:1011880015F0DB51D926DC51DA22DF50916F91C07E
:1011980092F0936B946B956B92C095F0946B936BF4
:1011A800926B8D519211966F8E519311976F8F514B
:1011B8009411986F90519511996F8A5196119A6F61
:1011C8008B5197119B6F000E98119C6F000E99110F
:1011D8009D6F22EE12F0DB51D926DC51DA22DF5066
:1011E8009E6F9E519A119F6F9B51A06F9C51A16F4A
:1011F8009D51A26F720E9F190DE1720EA0190AE19E
:10120800410EA11907E1610EA219D8A40EEF09F049
:1012180010EF09F0DEEF09F022EE17F0DB51D926C6
:10122800DC51DA22DF50896F89518B6F8A6B22EE8D
:1012380018F0DB51D926DC51DA22DF508C6F8CC0D4
:101248008DF08E6B8F6B906B8EC090F08DC08FF091
:101258008E6B8D6B22EE19F0DB51D926DC51DA2228
:10126800DF50916F91C092F0936B946B956B92C025
:1012780095F0946B936B926B8D519211966F8E5182
:101288009311976F8F519411986F90519511996F91
:101298008A5196119A6F8B5197119B6F000E981176
:1012A8009C6F000E99119D6F22EE16F0DB51D92626
:1012B800DC51DA22DF509E6F9E519A119F6F9B512D
:1012C800A06F9C51A16F9D51A26F20EE0EF0DB51D3
:1012D800D926DC51DA229FC0DEFFA0C0DEFFA1C004
:1012E800DEFFA2C0DEFF22EE1BF0DB51D926DC5167
:1012F800DA22DF50896F89518B6F8A6B22EE1CF0DE
:10130800DB51D926DC51DA22DF508C6F8CC08DF08E
:101318008E6B8F6B906B8EC090F08DC08FF08E6B44
:101328008D6B22EE1DF0DB51D926DC51DA22DF501D
:10133800916F91C092F0936B946B956B92C095F0FE
:10134800946B936B926B8D519211966F8E51931192
:10135800976F8F519411986F90519511996F8A5189
:1013680096119A6F8B5197119B6F000E98119C6F75
:10137800000E99119D6F22EE1AF0DB51D926DC512F
:10138800DA22DF509E6F9E519A119F6F9B51A06F7A
:101398009C51A16F9D51A26F20EE0AF0DB51D92616
:1013A800DC51DA229FC0DEFFA0C0DEFFA1C0DEFF55
:1013B800A2C0DEFFDBC0D9FFDCC0DAFFDAC0DFFF86
:1013C80001017C4B7D2B000120EE06F0DB51D92674
:1013D800DC51DA227CC1DEFF7DC1DDFFA5EF01F023
:1013E8001200000E01019D6F000E966F070E8C6EA5
:1013F800010EE26F000E9C6F0F0E0F01596F000E69
:10140800116F000E196F000E216F000E266F000E6F
:101418002E6F886889688A688A8E88908892838205
:10142800020E536E39EC6EF088948384889C839CFA
:10143800889E839E8B6889689D0E00018A6FF60ED0
:101448008B6FCD0E8C6FFF0E8D6FFB0E8E6FFE0EA9
:101458008F6F3A0E906FFF0E916F4EEC6FF01EEC8F
:101468006EF04DEF0AF0A30E00018A6FFE0E8B6F2F
:101478008FCF8CF08D6B4EEC6FF0290E0101DD6F74
:10148800960EDC6F7F0EE82EFED7DC2FFCD7DD2F03
:10149800FAD78FB252EF0AF054EF0AF037EF0AF09A
:1014A80038EC6DF001019D6F6D0E00018A6FFB0E27
:1014B8008B6F9DC18CF08D6B4EEC6FF00400290E84
:1014C8000101DD6F960EDC6F7F0EE82EFED7DC2F54
:1014D800FCD7DD2FFAD7D250F00B0109D26ED09E7F
:1014E8000E01C691CF0ECF16CF82CF80C2890F01D1
:1014F800138113891489F28E0E01BA8911EC65F0F3
:10150800839283948380040078EC42F0C6EC57F011
:10151800EAEC6EF001019551D8B495EF0AF097EF17
:101528000AF090EF0BF0A40E00018A6FFD0E8B6F8E
:101538004EEC6FF04EEC62F023C0A9F324C0AAF37E
:1015480025C0ABF326C0ACF3000E0301B76F000E45
:10155800B66FD90E00018A6FFF0E8B6FA90E0301BB
:10156800B625D96E030EB721DA6EDF500101DC6FA4
:10157800DC5100018C6F8D6B4EEC6FF00301B64BA4
:10158800B72BB7BFD1EF0AF0B75109E1040EB65D2A
:10159800D8A0D1EF0AF0D3EF0AF0ADEF0AF0850E2C
:1015A80000018A6FFC0E8B6F4EEC6FF0C10E0001CC
:1015B8008A6FFA0E8B6F4EEC6FF022EE04F000EE9D
:1015C800CBF01F0EDBCFEBFFE806FCE2D10E0001EB
:1015D800EB6FFF0EEC6F9DEC45F0CBC058F1CCC023
:1015E80059F1CDC05AF1CEC05BF1010158515911E2
:1015F8005A115B11D8B403EF0BF005EF0BF090EF25
:101608000BF0A70E00018A6FFA0E8B6F58C18CF091
:1016180059C18DF05AC18EF05BC18FF04EEC6FF05E
:10162800040E0001A46F020EA56F58C1DDF159C167
:10163800DEF15AC1DFF10101DC6B000EDC2500018F
:10164800A66F010E0101DD210001A76F000E010147
:10165800DE210001A86F000E0101DF210001A96F42
:10166800CDEC17F0040E00018C6F020E8D6F340E56
:101678008E6F0B0E8F6F000E916F080E906FB30E6A
:10168800926F030E936FD0EC1EF0000E0301B96F3A
:10169800000EB86FB9BF5AEF0BF0B95109E1080E47
:1016A800B85DD8A05AEF0BF05CEF0BF05EEF0BF0D3
:1016B80078EF0BF0D50E00018A6FFF0E8B6F340E9A
:1016C8000301B825D96E0B0EB921DA6EDF5001017E
:1016D800DC6FDC5100018C6F8D6B4EEC6FF00301F9
:1016E800B84BB92B4EEF0BF034CBDCF10101DC51D8
:1016F8000301A16FA26BA36BA46B7A0E00018A6F22
:10170800FE0E8B6FA1C38CF0A2C38DF0A3C38EF025
:10171800A4C38FF04EEC6FF001019CAF96EF0BF075
:1017280098EF0BF0ABEF0BF08A6883928382290E57
:101738000101DD6F960EDC6F7F0EE82EFED7DC2FE1
:10174800FCD7DD2FFAD7F6EC49F099EF0BF0E25110
:10175800D8B4B1EF0BF0B3EF0BF0C1EF0BF0C40E40
:1017680000018A6FFD0E8B6F4EEC6FF0020E0101C7
:101778009B6F220E9A6FCDEF0BF0B40E00018A6FAB
:10178800FD0E8B6F4EEC6FF0010E01019B6F040E86
:101798009A6F000E0301B06F000EAF6F000EBD6FA1
:1017A800839E000EBC6F010EBB6FBCBFE5EF0BF054
:1017B800BC5109E1040EBB5DD8A0E5EF0BF0E7EFE3
:1017C8000BF0E9EF0BF05AEF0CF0BBC30CF0BCC305
:1017D8000DF0000E0F6E0F0E0E6E8EEC6EF0240ED6
:1017E8000C24126E0E0E0D20136EDFEC6BF01350EE
:1017F80009E1030E125CD8A004EF0CF006EF0CF020
:1018080055EF0CF0BBC30CF0BCC30DF0000E0F6E0F
:101818000F0E0E6E8EEC6EF0240E0C240301A76FD3
:101828000E0E0D20A86F120E00018A6FFE0E8B6F30
:10183800A7C38CF0A8C38DF04EEC6FF0BBC3DCF1EE
:10184800BCC3DDF1050ED8900101DC37DD37E82E89
:1018580027EF0CF0040EDC250001DD6F020E0101FC
:10186800DD210001DE6FBBC30CF0BCC30DF0000E20
:101878000F6E0F0E0E6E8EEC6EF0240E0C2400010F
:10188800DF6F0E0E0D20E06F030EE16F12EC28F0F3
:101898000101DE6FDE510301B16FB26BB1512CEC67
:1018A80069F00301BB4BBC2BD9EF0BF0020E010111
:1018B8009719D8A462EF0CF064EF0CF07AEF0EF0F1
:1018C8000F01108B070E2D6F7AEF0EF038EC6DF0CC
:1018D8000101966F9751D8B474EF0CF076EF0CF0C5
:1018E800D4EF0CF09D519619D8B47DEF0CF07FEF32
:1018F8000CF0D4EF0CF0838E000E0301AE6F000ED7
:10190800AD6F96C1A5F3A66BD00E0101DC6FC90EB1
:10191800E82EFED7DC2FFCD700D038EC6DF00101A3
:10192800966F9651DC6FDD6B0301A5510101DC193F
:1019380009E10301A6510101DD19D8A4A6EF0CF0B5
:10194800A8EF0CF0ABEF0CF00301AD4BAE2B03018D
:10195800AEBFB8EF0CF0AE5109E1650EAD5DD8A091
:10196800B8EF0CF0BAEF0CF085EF0CF096C19DF1D2
:10197800290E0101DD6F960EDC6F7F0EE82EFED773
:10198800DC2FFCD7DD2FFAD7740E00018A6FFC0E0E
:101998008B6F9DC18CF08D6B4EEC6FF0A4EF0EF049
:1019A8008EB8D9EF0CF0DBEF0CF0DCEF0CF089947B
:1019B80072EC6FF00C500D10D8B4E5EF0CF0E7EFB7
:1019C8000CF07AEF0EF0BDC3B5F3BA0E0C6E030E31
:1019D8000D6E2CEC66F00301BD6F430E00018A6F9B
:1019E800FF0E8B6FBDC38CF08D6B8DB0FEEF0CF0CE
:1019F80003EF0DF00101DC6BDC2B05EF0DF00101AD
:101A0800DC6BDC5100018E6F8F6B4EEC6FF00301C5
:101A1800BAA911EF0DF013EF0DF071EF0DF0600E94
:101A2800BD19D8A41AEF0DF01CEF0DF071EF0DF0F1
:101A38005F0EB519D8A423EF0DF025EF0DF071EF67
:101A48000DF0B00E00018A6FFC0E8B6FBDC38CF0D9
:101A58008D6BB5C38EF08F6B8EB235EF0DF03AEF0C
:101A68000DF00101DC6BDC2B3CEF0DF00101DC6BB0
:101A7800DC510001906F916B8EB445EF0DF04AEF89
:101A88000DF00101DD6BDD2B4CEF0DF00101DD6B7D
:101A9800DD510001926F936B4EEC6FF053500209C9
:101AA800536E2BEE34F09BC1DFFF2BEE35F09AC15D
:101AB800DFFF8384000E246E020E236E45EC3DF09A
:101AC80083945350FD0B536E000E506E68EC6EF00D
:101AD800000E0301BD6F7AEF0EF00101E251D8B498
:101AE80078EF0DF07AEF0DF0ECEF0DF00301BA513D
:101AF800100B0001B06F000EB16F0301BD5171EC06
:101B080039F0B0C0BEF3B1C0BFF3080E0301BE196F
:101B1800BF11D8A492EF0DF094EF0DF095EF0DF0F2
:101B280000F0070E0301BE19BF11D8A49EEF0DF0F7
:101B3800A0EF0DF0A2EF0DF017EC68F00301BE0561
:101B4800BF11D8A4AAEF0DF0ACEF0DF0AEEF0DF079
:101B5800CFEC67F0020E0301BE19BF11D8A4B7EF8E
:101B68000DF0B9EF0DF0BBEF0DF01FEC4FF0030EC9
:101B78000301BE19BF11D8A4C4EF0DF0C6EF0DF0D4
:101B8800CCEF0DF065EC37F0E2C0AFF3E3C0B0F393
:101B9800050E0301BE19BF11D8A4D5EF0DF0D7EF7C
:101BA8000DF0DDEF0DF014EC44F0EDC0AFF3EEC036
:101BB800B0F3090E0301BE19BF11D8A4E6EF0DF06A
:101BC800E8EF0DF07AEF0EF06BEC6FF07AEF0EF0B5
:101BD8000301BA51100B236E000E246EBD516CEC3C
:101BE8001BF023C0BEF324C0BFF3070E0301BE19C8
:101BF800BF11D8A402EF0EF004EF0EF006EF0EF0BE
:101C0800C7EC6EF0020E0301BE19BF11D8A40FEF86
:101C18000EF011EF0EF013EF0EF0A9EC69F00301CE
:101C2800BE05BF11D8A41BEF0EF01DEF0EF01FEF7D
:101C38000EF071EC53F0030E0301BE19BF11D8A4C6
:101C480028EF0EF02AEF0EF02CEF0EF043EC5CF0CC
:101C5800040E0301BE19BF11D8A435EF0EF037EFFB
:101C68000EF039EF0EF075EC6CF0050E0301BE199D
:101C7800BF11D8A442EF0EF044EF0EF046EF0EF07D
:101C88001EEC56F0060E0301BE19BF11D8A44FEF83
:101C98000EF051EF0EF053EF0EF0FCEC6CF0080E66
:101CA8000301BE19BF11D8A45CEF0EF05EEF0EF071
:101CB80060EF0EF0E0EC4DF0090E0301BE19BF1104
:101CC800D8A469EF0EF06BEF0EF06DEF0EF088EC14
:101CD8006FF00A0E0301BE19BF11D8A476EF0EF0FB
:101CE80078EF0EF07AEF0EF0EDEC5CF08FB27FEF4C
:101CF8000EF081EF0EF0A4EF0EF0050E0301AF1900
:101D0800B011D8A48AEF0EF08CEF0EF06AEF0CF049
:101D1800A4EF0EF0A30E00018A6FFE0E8B6F8FCF1B
:101D28008CF08D6B4EEC6FF0290E0101DD6F960E75
:101D3800DC6F7F0EE82EFED7DC2FFCD7DD2FFAD71D
:101D48008FB2A9EF0EF0ABEF0EF08EEF0EF0290E6A
:101D58000101DD6F960EDC6F7F0EE82EFED7DC2FBB
:101D6800FCD7DD2FFAD7000E5DEC6FF00101936F01
:101D7800880E00018A6FFC0E8B6F93C18CF08D6BFF
:101D88004EEC6FF0290E0101DD6F960EDC6F7F0EB1
:101D9800E82EFED7DC2FFCD7DD2FFAD78394839269
:101DA800000E0001DD6F000EDE6F870EDF6FFC0E88
:101DB800E06F000EE16FFAEC60F087EF0AF035EFA4
:101DC80001F0406E000E3F6ECEEF12F04050D8A4E6
:101DD800F0EF0EF0F2EF0EF011EF0FF00001FE51F0
:101DE800D8B4F9EF0EF0FBEF0EF011EF0FF0F80E8C
:101DF8008A6FFB0E8B6FCECF8CF08D6BCDCF8EF0B4
:101E08008F6B4EEC6FF0000E3F6E000E0101756F88
:101E18000A0E746F839071EF13F0020E4018D8A465
:101E280018EF0FF01AEF0FF039EF0FF00001FE5125
:101E3800D8B421EF0FF023EF0FF039EF0FF0CA0EEF
:101E48008A6FFB0E8B6FCECF8CF08D6BCDCF8EF063
:101E58008F6B4EEC6FF0000E3F6E000E0101756F38
:101E6800140E746F839071EF13F01F0E40643FEFF0
:101E78000FF041EF0FF09FEF0FF0300E406047EF8B
:101E88000FF049EF0FF09FEF0FF00001FE51D8B4AB
:101E980050EF0FF052EF0FF09FEF0FF04050E00FB0
:101EA800FF6FB50E8A6FF90E8B6FCECF8CF08D6BEE
:101EB800CDCF8EF08F6BFFC090F0916B4EEC6FF032
:101EC800000E3F6E0001FF51200D0E0EF324D96E57
:101ED800020EF420DA6EDE50DE10DE10DE10D8B40A
:101EE80078EF0FF07AEF0FF082EF0FF0030EFF6537
:101EF80080EF0FF082EF0FF097EF0FF0010E4D6EAD
:101F0800FF51140D130EF324D96E010EF420DA6E6E
:101F1800FF51140D130EF324E16E010EF420E26E4E
:101F2800E7500409DF6E000E0101756F000E746F33
:101F3800839071EF13F03F0E4064A5EF0FF0A7EF09
:101F48000FF0E6EF0FF0500E4060ADEF0FF0AFEF7F
:101F58000FF0E6EF0FF00001FE51D8B4B6EF0FF026
:101F6800B8EF0FF0E6EF0FF0FF51140D000EF32459
:101F7800D96E010EF420DA6E4050C00FDF6E3D0EB0
:101F88008A6FF90E8B6FCECF8CF08D6BCDCF8EF024
:101F98008F6BFF51140D000EF324D96E010EF4203F
:101FA800DA6EDF50236E2350906F916B4EEC6FF01A
:101FB800000E3F6E000E0101756F000E746F839066
:101FC80071EF13F0340E4018D8A4EDEF0FF0EFEFD7
:101FD8000FF00EEF10F00001FE51D8B4F6EF0FF03D
:101FE800F8EF0FF00EEF10F0230E8A6FFC0E8B6FD8
:101FF800CECF8CF08D6BCDCF8EF08F6B4EEC6FF01B
:10200800000E0101756F000E746F000E3F6E839015
:1020180071EF13F0350E4018D8A415EF10F017EF34
:1020280010F036EF10F00001FE51D8B41EEF10F09A
:1020380020EF10F036EF10F0730E8A6FFA0E8B6FE8
:10204800CECF8CF08D6BCDCF8EF08F6B4EEC6FF0CA
:10205800000E3F6E0D0E0101756FAC0E746F83900C
:1020680071EF13F0370E4018D8A43DEF10F03FEF92
:1020780010F04FEF10F00001FE51D8B446EF10F009
:1020880048EF10F04FEF10F00E0E0101756F750E4E
:10209800746F71EF13F00D0E4018D8A456EF10F0BE
:1020A80058EF10F078EF10F00001FE51D8B45FEF50
:1020B80010F061EF10F078EF10F0000E3F6E020E96
:1020C8000101756FBC0E746F8390240E00018A6F36
:1020D800FA0E8B6FCECF8CF08D6BCDCF8EF08F6BD1
:1020E8004EEC6FF071EF13F0100E4018D8A47FEF8C
:1020F80010F081EF10F091EF10F00001FE51D8B40C
:1021080088EF10F08AEF10F091EF10F0030E010144
:10211800756FE90E746F71EF13F0180E4018D8A49C
:1021280098EF10F09AEF10F0AAEF10F00001FE51AE
:10213800D8B4A1EF10F0A3EF10F0AAEF10F0070E3B
:102148000101756F090E746F71EF13F03E0E4018A0
:10215800D8A4B1EF10F0B3EF10F0C3EF10F0000106
:10216800FE51D8B4BAEF10F0BCEF10F0C3EF10F086
:102178000F0E0101756F3D0E746F71EF13F0D20EE3
:1021880000018A6FF90E8B6FCECF8CF08D6BCDCF9F
:102198008EF08F6B40C090F0916B4EEC6FF071EF4A
:1021A80013F00001FF51140D010EF324D96E010E36
:1021B800F420DA6E40C0DFFF030E0101756FEA0EEE
:1021C800746F71EF13F00001FF51140D020EF32428
:1021D800D96E010EF420DA6E40C0DFFF030E010154
:1021E800756FEB0E746F71EF13F00001FF51140D52
:1021F800030EF324D96E010EF420DA6E40C0DFFF1F
:10220800030E0101756FEC0E746F71EF13F000018E
:10221800FF51140D040EF324D96E010EF420DA6E6A
:1022280040C0DFFF030E0101756FED0E746F71EF93
:1022380013F00001FF51140D050EF324D96E010EA1
:10224800F420DA6E40C0DFFF030E0101756FEE0E59
:10225800746F71EF13F00001FF51140D060EF32493
:10226800D96E010EF420DA6E40C0DFFFFF51140D65
:10227800060EF324D96E010EF420DA6EDF50236EB9
:1022880023C024F0256A266A276A26C027F025C0BD
:1022980026F024C025F0246AFF51140D050EF324FE
:1022A800D96E010EF420DA6EDF50286E28C029F0AE
:1022B8002A6A2B6A2C6A2AC02CF029C02BF02A6AB9
:1022C800296AFF51140D040EF324D96E010EF4206F
:1022D800DA6EDF502D6E2DC02EF02F6A306A316A0B
:1022E8002EC031F0306A2F6A2E6AFF51140D030E8A
:1022F800F324D96E010EF420DA6EDF50326E3250BC
:102308002E24336E000E2F20346E000E3020356ED2
:10231800000E3120366E29503324376E2A5034206F
:10232800386E2B503520396E2C5036203A6E24509A
:1023380037243B6E255038203C6E265039203D6EA0
:1023480027503A203E6EFF51140D070EF324D96E24
:10235800010EF420DA6E3BC0DEFF3CC0DEFF3DC05C
:10236800DEFF3EC0DEFF5C0E8A6FF80E8B6FCECFAD
:102378008CF08D6BCDCF8EF08F6BFF51140D070E47
:10238800F324D96E010EF420DA6EDECF90F0DECFA2
:1023980091F0DECF92F0DECF93F04EEC6FF0000EAE
:1023A8000101756F000E746F71EF13F00001FF519A
:1023B800140D120EF324D96E010EF420DA6E40C00B
:1023C800DFFF070E0101756F0A0E746F71EF13F0CE
:1023D8000001FF51140D110EF324D96E010EF420E3
:1023E800DA6E40C0DFFF070E0101756F0B0E746FC8
:1023F80071EF13F00001FF51140D100EF324D96E84
:10240800010EF420DA6E40C0DFFF070E0101756F80
:102418000C0E746F71EF13F00001FF51140D0F0EC5
:10242800F324D96E010EF420DA6E40C0DFFFDE0E11
:102438008A6FF80E8B6FCECF8CF08D6BCDCF8EF070
:102448008F6BFF51140D0F0EF324D96E010EF4207B
:10245800DA6EDECF90F0DECF91F0DECF92F0DECFF5
:1024680093F04EEC6FF0D3EF11F040C050F10F0E27
:102478000101756F3E0E746F71EF13F040C051F19A
:102488000F0E0101756F3F0E746F71EF13F040C0AE
:1024980052F10F0E0101756F400E746F71EF13F05A
:1024A80040C053F10F0E0101756F410E746F71EF4B
:1024B80013F040C054F10F0E0101756F420E746F96
:1024C80071EF13F040C055F10F0E0101756F430E07
:1024D800746F71EF13F040C056F10F0E0101756F64
:1024E800440E746F71EF13F040C057F1320E0001C3
:1024F8008A6FF60E8B6FCECF8CF08D6BCDCF8EF0B2
:102508008F6B50C190F0916B51C192F0936B52C197
:1025180094F0956B53C196F0976B54C198F0996BF2
:1025280055C19AF09B6B56C19CF09D6B57C19EF0AC
:102538009F6B4EEC6FF0D3EF11F0230E00018A6F02
:10254800FC0E8B6FCECF8CF08D6BCDCF8EF08F6B5A
:102558004EEC6FF0D3EF11F00E0E0101756F760E91
:10256800746F71EF13F0090E00018A6FFA0E8B6F0A
:10257800CECF8CF08D6BCDCF8EF08F6B4EEC6FF095
:10258800000E0101756F000E746F090E3F6E839087
:1025980071EF13F074C123F075C124F02450000AC0
:1025A800D8B4F5EF12F0030AD8B4FCEF12F0040A1D
:1025B800D8B417EF13F00A0AD8B42AEF13F0030AB5
:1025C800D8B435EF13F0010AD8B440EF13F0130A6A
:1025D800D8B463EF13F03B0AD8B46AEF13F071EF85
:1025E80013F02350000AD8B4EAEF0EF071EF13F09D
:1025F8002350E90AD8B4D5EF10F0030AD8B4E7EFAE
:1026080010F0010AD8B4F9EF10F0070AD8B40BEFAC
:1026180011F0010AD8B41DEF11F0030AD8B42FEF56
:1026280011F071EF13F02350090AD8B4DAEF11F062
:10263800030AD8B4ECEF11F0010AD8B4FEEF11F098
:10264800070AD8B410EF12F071EF13F02350480ABC
:10265800D8B4A1EF12F0E40AD8B471EF13F071EF17
:1026680013F02350750AD8B4B0EF12F0030AD8B4A7
:10267800B7EF12F071EF13F023503D0AD8B439EFD9
:1026880012F0030AD8B442EF12F0010AD8B44BEFA3
:1026980012F07F0AD8B454EF12F0010AD8B45DEFF3
:1026A80012F0030AD8B466EF12F0010AD8B46FEF3B
:1026B80012F0070AD8B478EF12F071EF13F0235034
:1026C8002A0AD8B471EF13F071EF13F023500F0AF0
:1026D800D8B471EF13F071EF13F03F501200A6C099
:1026E800B9F0A7C0BAF0AAC0D9FFABC0DAFF000E94
:1026F800DE6E000EDD6EA4C00DF0A5C00EF085ECF8
:1027080063F00001B86FB851D8B48DEF13F08FEFB4
:1027180013F092EF13F0B851CCEF17F020EE05F05C
:10272800A451D926A551DA22DF50D8B49EEF13F070
:10273800A0EF13F0A9EF13F020EE05F0A451D9266D
:10274800A551DA22DF50CCEF17F020EE04F0A451A7
:10275800D926A551DA22DFB2B4EF13F0B6EF13F0A1
:10276800B9EF13F0070ECCEF17F020EE06F0A451E6
:10277800D926A551DA2210EE06F0A451E126A5517A
:10278800E222E6CFB0F0E6CFB1F0E6CFB2F0E6CF86
:10279800B3F0A851B025B46FA951B121B56F000E9F
:1027A800B221B66F000EB321B76FDE50B45DDE50B4
:1027B800B559DE50B659DE50B759D8B0E6EF13F028
:1027C800E8EF13F08BEF17F0000EA96F000EA86F5B
:1027D8008BEF17F020EE06F0A451D926A551DA2286
:1027E800FF0EDE14AC6F010EDE14AD6F000EDE14AA
:1027F800AE6F000EDE14AF6FAC51AD11AE11AF115C
:10280800D8A409EF14F00BEF14F0DEEF16F020EE69
:1028180006F0A451D926A551DA22DECFACF0DECFDE
:10282800ADF0DECFAEF0DECFAFF00A0E21EF14F040
:10283800D890AF33AE33AD33AC33E82E1CEF14F081
:10284800A4C0D9FFA5C0DAFF10EE02F0DE50E126E1
:10285800DD50E222E750B06FB005AC15BB6FBB513D
:10286800D8A439EF14F03BEF14F00BEF15F020EE7D
:1028780006F0A451D926A551DA22DE50DE10DE106A
:10288800DE10D8A44AEF14F04CEF14F081EF14F0E6
:1028980020EE0EF0A451D926A551DA22DECFC2F0DF
:1028A800DECFC3F0DECFC4F0DECFC5F0C251C31116
:1028B800C411C511D8A463EF14F065EF14F0A1EFAB
:1028C80014F0A4C0D9FFA5C0DAFFDECF91F0DDCFA8
:1028D80092F0000E936F000E946F000E956F000E2D
:1028E800966F66EC3BF091C0C2F092C0C3F093C003
:1028F800C4F094C0C5F0A1EF14F0A4C0D9FFA5C0DE
:10290800DAFFDECF91F0DDCF92F020EE12F0A45185
:10291800D926A551DA22DECF93F0DECF94F0DECFB0
:1029280095F0DECF96F066EC3BF091C0C2F092C015
:10293800C3F093C0C4F094C0C5F00001C251C311E4
:10294800C411C511D8A4ABEF14F0ADEF14F0AFEF7C
:1029580014F094EF17F0C205C311C411C511D8A41F
:10296800B8EF14F0BAEF14F0C5EF14F020EE05F04C
:10297800A451D926A551DA22020EDF6E020ECCEF41
:1029880017F0C2290AE1C32908E1C42906E1C529CB
:10299800D8A4D1EF14F0D3EF14F0DEEF14F020EE4A
:1029A80005F0A451D926A551DA22010EDF6E010ED9
:1029B800CCEF17F020EE12F0A451D926A551DA2257
:1029C800C2C0DEFFC3C0DEFFC4C0DEFFC5C0DEFF7D
:1029D80020EE0EF0A451D926A551DA22DE50DE10E1
:1029E800DE10DE10D8A4FBEF14F0FDEF14F00BEFAF
:1029F80015F020EE0EF0A451D926A551DA22C2C056
:102A0800DEFFC3C0DEFFC4C0DEFFC5C0DEFF20EEB0
:102A180016F0A451D926A551DA22A4C0E1FFA5C019
:102A2800E2FF00EE2AF0E650E926E550EA22DE5001
:102A3800EE180DE1DE50EE180AE1DE50EE1807E15F
:102A4800DE50EE18D8A42BEF15F02DEF15F04AEF55
:102A580015F0A4C0D9FFA5C0DAFFDECF25F0DDCF81
:102A680026F015EC5AF00009D8B43DEF15F03FEF09
:102A780015F04AEF15F0000120EE05F0A451D92613
:102A8800A551DA22010EDF6EDBEF14F0A4C0D9FFE6
:102A9800A5C0DAFFDECF18F0DDCF19F0000120EE77
:102AA80012F0A451D926A551DA22DECF1AF0DECFD2
:102AB8001BF0DECF1CF0DECF1DF04CEC64F018C02C
:102AC800BEF019C0BFF01AC0C0F01BC0C1F00001B1
:102AD800BE51BF11C011C111D8A475EF15F077EF21
:102AE80015F081EF15F020EE05F0A451D926A55177
:102AF800DA22020EDF6EC2EF14F0BB51BE27000EC1
:102B0800BF23C023C123A8C0ACF0A9C0ADF0090EF3
:102B1800AE6FD890AD33AC33AE2F8DEF15F0ACC09F
:102B2800BCF0ADC0BDF0BC51BD11D8B49EEF15F0DE
:102B3800A0EF15F085EF16F0BB51BC25AC6F000E69
:102B4800BD21AD6FA4C0D9FFA5C0DAFF10EE02F019
:102B5800DE50E126DD50E222E750AE6FAF6BAC519C
:102B6800AE5DAD51AF59D8B0BCEF15F0BEEF15F062
:102B7800D0EF15F0A4C0D9FFA5C0DAFF10EE02F01F
:102B8800DE50E126DD50E222E750AC6FBB51AC5D70
:102B9800BC6FBD6BD8A0BD07B9C01BF0BAC01CF094
:102BA800BEC01DF0BFC01EF0C0C01FF0C1C020F0E5
:102BB800BCC021F0BDC022F0A4C0D9FFA5C0DAFF77
:102BC80010EE01F0DE50E126DD50E222E750F2EC93
:102BD80056F00009D8B4F3EF15F0F5EF15F000EF53
:102BE80016F0000120EE05F0A451D926A551DA22ED
:102BF800010EDF6EDBEF14F00001BC51AC6FBD516C
:102C0800AD6FAE6BAF6BA4C0D9FFA5C0DAFF10EEF5
:102C18002AF0DE50E126DD50E222E6CFB0F0E6CF22
:102C2800B1F0E6CFB2F0E6CFB3F0BE51B05DB46F0D
:102C3800BF51B159B56FC051B259B66FC151B359EF
:102C4800B76FAC51B45DAD51B559AE51B659AF512E
:102C5800B759D8B032EF16F034EF16F073EF16F01C
:102C6800A4C0D9FFA5C0DAFFDECFACF0DDCFADF050
:102C78002E0EAC250C6E000EAD210D6EA4C0D9FF32
:102C8800A5C0DAFF10EE2AF0DE50E126DD50E22280
:102C9800E6CFAEF0E5CFAFF0BE51AE5FBF51AF5B50
:102CA800090ED890AE37AF37E82E55EF16F0AE5173
:102CB800B9250E6EAF51BA210F6E020E116E000EBD
:102CC800106E07EC6CF0A4C0D9FFA5C0DAFF10EEB7
:102CD80004F0DE50E126DD50E222000EE76EBCC0B3
:102CE800ACF0BDC0ADF0090ED8900001AC37AD37DF
:102CF800E82E78EF16F0ACC0C6F0ADC0C7F06DEFA7
:102D080017F020EE0AF0A451D926A551DA2210EEC8
:102D180006F0A451E126A551E222DE50E65CDE5021
:102D2800E658DE50E658DE50E658D8A09EEF16F07A
:102D3800A0EF16F0CFEF16F0A4C0D9FFA5C0DAFFB8
:102D4800DECF25F0DDCF26F015EC5AF00009D8B417
:102D5800B0EF16F0B2EF16F0BDEF16F0000120EE5E
:102D680005F0A451D926A551DA22010EDF6EDBEF5A
:102D780014F0A4C0D9FFA5C0DAFF10EE2AF0DE5087
:102D8800E126DD50E222BEC0E6FFBFC0E6FFC0C0BC
:102D9800E6FFC1C0E6FF000120EE16F0A451D926D7
:102DA800A551DA22BEC0DEFFBFC0DEFFC0C0DEFF15
:102DB800C1C0DEFFFF0EAC6F010EAD6F20EE06F056
:102DC800A451D926A551DA22DECFAEF0DDCFAFF07F
:102DD800AC51AE17AD51AF17AE510008C66FAF5129
:102DE800D8A0E82A0208C76FC651A85DC751A959DB
:102DF800D8B001EF17F003EF17F007EF17F0A8C0EE
:102E0800C6F0A9C0C7F0A4C0D9FFA5C0DAFFDECFBD
:102E18003AF0DDCF3BF020EE16F0A451D926A551AB
:102E2800DA22DECF3CF0DECF3DF0DECF3EF0DECF63
:102E38003FF0AFEC64F00009D8B425EF17F027EFA6
:102E480017F032EF17F0000120EE05F0A451D92653
:102E5800A551DA22010EDF6EDBEF14F0FF0E000140
:102E6800AC6F010EAD6F20EE06F0A451D926A55126
:102E7800DA22DECFAEF0DDCFAFF0AC51AE17AD51F8
:102E8800AF17A4C0D9FFA5C0DAFFDECFB0F0DDCF01
:102E9800B1F0AE51B027AF51B1232E0EB0250C6E54
:102EA800000EB1210D6EB9C00EF0BAC00FF0C6C049
:102EB80010F0C7C011F007EC6CF0A4C0D9FFA5C092
:102EC800DAFF10EE04F0DE50E126DD50E222010EBA
:102ED800E76E0001C651B927C751BA2320EE06F0A4
:102EE800A451D926A551DA22C651DE26C751DE22C1
:102EF800000EDE22DE22AAC0D9FFABC0DAFFC6511F
:102F0800DE26C751DD22C651A85FC751A95BA8516B
:102F1800A911D8A492EF17F094EF17F0EEEF13F081
:102F280020EE06F0A451D926A551DA2210EE0AF0B7
:102F3800A451E126A551E222DE50E65CDE50E658B7
:102F4800DE50E658DE50E658D8B0ADEF17F0AFEFD8
:102F580017F0C3EF17F020EE06F0A451D926A551BB
:102F6800DA2210EE0AF0A451E126A551E222DECFC2
:102F7800E6FFDECFE6FFDECFE6FFDECFE6FF20EEA0
:102F880004F0A451D926A551DA22000EDB8A000EDE
:102F98001200A4C00DF0A5C00EF085EC63F000018E
:102FA800BE6FBE51D8B4DBEF17F0DDEF17F0E0EFDE
:102FB80017F0BE516BEF1BF020EE05F0A451D92697
:102FC800A551DA22DF50D8B4ECEF17F0EEEF17F086
:102FD800F7EF17F020EE05F0A451D926A551DA2213
:102FE800DF506BEF1BF020EE0AF0A451D926A55153
:102FF800DA22A651DE5CA751DE58A851DE58A95145
:10300800DE58D8B00AEF18F00CEF18F027EF18F0D8
:1030180020EE04F0A451D926A551DA22DFB217EF29
:1030280018F019EF18F027EF18F020EE0AF0A45165
:10303800D926A551DA22DECFA6F0DECFA7F0DECF63
:10304800A8F0DECFA9F020EE06F0A451D926A551AC
:10305800DA22DECFBAF0DECFBBF0DECFBCF0DECFB7
:10306800BDF0000EBF6F000EC06F000EC16F000EE6
:10307800C26F20EE06F0A451D926A551DA22BFC0AE
:10308800DEFFC0C0DEFFC1C0DEFFC2C0DEFFA6514A
:10309800A711A811A911D8B454EF18F056EF18F0D9
:1030A800EFEF1AF0A4C0D9FFA5C0DAFF10EE02F0C6
:1030B800DE50E126DD50E222E750AA6FAAC0ABF04D
:1030C800AC6BAD6BAE6B090ED890AB37AC37AD3788
:1030D800AE37E82E68EF18F0ABC0C3F0ACC0C4F050
:1030E800ADC0C5F0AEC0C6F0BA51BB11BC11BD1120
:1030F800D8B481EF18F083EF18F020EF19F0FF0E25
:10310800A6250C6EFF0EA7210D6EFF0EA8210E6ED0
:10311800FF0EA9210F6EC3C010F0C4C011F0C5C0C6
:1031280012F0C6C013F030EC67F00CC0AAF00DC066
:10313800ABF00EC0ACF00FC0ADF0FF0E0001BA2529
:103148000C6EFF0EBB210D6EFF0EBC210E6EFF0E26
:10315800BD210F6EC3C010F0C4C011F0C5C012F07D
:10316800C6C013F030EC67F00C500001AA5D0D509A
:10317800AB590E50AC590F50AD59D8A0C6EF18F046
:10318800C8EF18F020EF19F0FF0EC325AA6FFF0E45
:10319800C421AB6FFF0EC521AC6FFF0EC621AD6F0A
:1031A800AA1DAE6FAB1DAF6FAC1DB06FAD1DB16F7B
:1031B800FF0EBA25B26FFF0EBB21B36FFF0EBC2105
:1031C800B46FFF0EBD21B56FAE51B215B66FAF51DA
:1031D800B315B76FB051B415B86FB151B515B96F14
:1031E80020EE06F0A451D926A551DA22B6C0DEFF9A
:1031F800B7C0DEFFB8C0DEFFB9C0DEFF20EE06F0C4
:10320800A451D926A551DA22DE50A65FDE50A75B6D
:10321800DE50A85BDD50A95B20EE12F0A451D92640
:10322800A551DA22DECFC7F0DECFC8F0DECFC9F075
:10323800DECFCAF09FEF19F020EE0EF0A451D92688
:10324800A551DA22DECFC7F0DECFC8F0DECFC9F055
:10325800DECFCAF0C751C811C911CA11D8A437EFB7
:1032680019F039EF19F091EF19F0A4C0D9FFA5C0F2
:10327800DAFFDECF91F0DDCF92F0000E936F000EF3
:10328800946F000E956F000E966F66EC3BF091C040
:10329800C7F092C0C8F093C0C9F094C0CAF000014A
:1032A800C705C811C911CA11D8A45DEF19F05FEF9D
:1032B80019F06AEF19F020EE05F0A451D926A551AE
:1032C800DA22020EDF6E020E6BEF1BF0C7290AE14D
:1032D800C82908E1C92906E1CA29D8A476EF19F056
:1032E80078EF19F083EF19F020EE05F0A451D926F4
:1032F800A551DA22010EDF6E010E6BEF1BF020EEF6
:103308000EF0A451D926A551DA22C7C0DEFFC8C0E5
:10331800DEFFC9C0DEFFCAC0DEFF20EE12F0A451F6
:10332800D926A551DA22C7C0DEFFC8C0DEFFC9C052
:10333800DEFFCAC0DEFFC751C811C911CA11D8B40F
:10334800A8EF19F0AAEF19F0EFEF1AF070EF1AF0E2
:1033580020EE04F0A451D926A551DA22DFA2B7EF56
:1033680019F0B9EF19F0E9EF19F0A4C0D9FFA5C019
:10337800DAFFDECF91F0DDCF92F0C7C093F0C8C07E
:1033880094F0C9C095F0CAC096F066EC3BF091C0C5
:10339800C7F092C0C8F093C0C9F094C0CAF0000149
:1033A800C751C811C911CA11D8A4DDEF19F0DFEF50
:1033B80019F003EF1AF0C3C0A6F0C4C0A7F0C5C047
:1033C800A8F0C6C0A9F07FEF1AF0A4C0D9FFA5C025
:1033D800DAFFDECF60F0DDCF61F0C7C062F0C8C0B1
:1033E80063F0C9C064F0CAC065F072EC30F060C028
:1033F800C7F061C0C8F062C0C9F063C0CAF000017C
:10340800C7290AE1C82908E1C92906E1CA29D8A4B7
:1034180010EF1AF012EF1AF01CEF1AF020EE05F078
:10342800A451D926A551DA22010EDF6E80EF19F0DA
:10343800CA51C911C81109E1020EC75DD8A027EF0A
:103448001AF029EF1AF042EF1AF0A4C0D9FFA5C06C
:10345800DAFF10EE12F0DE50E126DD50E222E650EF
:10346800C75DE650C859E650C959E650CA59D8A0B0
:1034780040EF1AF042EF1AF04CEF1AF020EE05F088
:10348800A451D926A551DA22020EDF6E67EF19F092
:1034980020EE12F0A451D926A551DA22C7C0DEFFCA
:1034A800C8C0DEFFC9C0DEFFCAC0DEFF20EE06F0DE
:1034B800A451D926A551DA22C351DE26C451DE22F1
:1034C800C551DE22C651DE22C351A65FC451A75B97
:1034D800C551A85BC651A95BA651C35DA751C45984
:1034E800A851C559A951C659D8A07DEF1AF07FEF48
:1034F8001AF0ACEF19F020EE06F0A451D926A55128
:10350800DA22A651DE26A751DE22A851DE22A951D1
:10351800DE22FF0EA615AA6F010EA715AB6F000ECF
:10352800A815AC6F000EA915AD6FAA51AB11AC115F
:10353800AD11D8B4A2EF1AF0A4EF1AF0EFEF1AF019
:10354800A4C0D9FFA5C0DAFFDECF18F0DDCF19F08F
:10355800C7C01AF0C8C01BF0C9C01CF0CAC01DF013
:103568004CEC64F018C0BFF019C0C0F01AC0C1F02C
:103578001BC0C2F00001BF51C011C111C211D8A4B3
:10358800C8EF1AF0CAEF1AF0D4EF1AF020EE05F0DF
:10359800A451D926A551DA22020EDF6E67EF19F081
:1035A800A6C0AAF0A7C0ABF0A8C0ACF0A9C0ADF007
:1035B8000A0EE4EF1AF0D890AD33AC33AB33AA332C
:1035C800E82EDFEF1AF0AA51BF27AB51C023AC5148
:1035D800C123AD51C22320EE06F0A451D926A5512E
:1035E800DA22FF0EDE14AA6F010EDE14AB6F000E96
:1035F800DE14AC6F000EDE14AD6FAA51AB11AC1126
:10360800AD11D8B40AEF1BF00CEF1BF032EF1BF032
:1036180020EE16F0A451D926A551DA22BF51DE18A2
:103628000FE1C051DE180CE1C151DE1809E1C251A9
:10363800DE18D8B422EF1BF024EF1BF032EF1BF09A
:1036480020EE16F0A451D926A551DA22BFC0DEFF1C
:10365800C0C0DEFFC1C0DEFFC2C0DEFF20EE06F044
:10366800A451D926A551DA2210EE0AF0A451E12678
:10367800A551E222DE50E65CDE50E658DE50E65800
:10368800DE50E658D8B04BEF1BF04DEF1BF0DDEFE6
:1036980017F020EE06F0A451D926A551DA2210EE33
:1036A8000AF0A451E126A551E222DECFE6FFDECFE3
:1036B800E6FFDECFE6FFDECFE6FF20EE04F0A45102
:1036C800D926A551DA22000EDB8ADDEF17F01200A9
:1036D800286E2450D8B473EF1BF075EF1BF077EF0A
:1036E8001BF0EAEC6EF0000E276E550E00018A6F93
:1036F800FF0E8B6F28C08CF08D6B83B086EF1BF0AC
:103708008AEF1BF0256A252A8BEF1BF0256A2550C6
:1037180000018E6F8F6B4EEC6FF02350D8B497EF8B
:103728001BF099EF1BF041EF1EF028507F0B286E1D
:10373800040E2818D8B4A3EF1BF0A5EF1BF0AEEFCA
:103748001BF0140E2818D8A4ACEF1BF0AEEF1BF03A
:10375800B9EF1BF0000E0101736F000E726F000EBF
:10376800246E070E236ECFEF1EF03F0E2818D8A444
:10377800C0EF1BF0C2EF1BF0CFEF1BF0000E0101F2
:103788008C6F000E736F000E726F000E246E000EA9
:10379800236ECFEF1EF05F0E2818D8A4D6EF1BF0CB
:1037A800D8EF1BF0E5EF1BF0000E01018D6F000E46
:1037B800736F000E726F000E246E000E236ECFEF33
:1037C8001EF03F0E2864EBEF1BF0EDEF1BF000EF4F
:1037D8001CF05F0E2860F3EF1BF0F5EF1BF000EF15
:1037E8001CF0400E2818D8B4FCEF1BF0FEEF1BF0BD
:1037F80000EF1CF0D8EF1BF0400E2818D8A407EFF4
:103808001CF009EF1CF018EF1CF0010E01018D6F80
:10381800000E8C6F000E736F000E726F000E246E18
:10382800000E236ECFEF1EF0200E2818D8A41FEF2D
:103838001CF021EF1CF041EF1EF0010E01018C6F0E
:10384800000E736F000E726F000E246E000E236E52
:10385800CFEF1EF0600E2818D8A435EF1CF037EF14
:103868001CF054EF1CF001018D51D8B43EEF1CF050
:1038780040EF1CF054EF1CF08A51D8B446EF1CF00E
:1038880048EF1CF04CEF1CF0080E276E4EEF1CF0B2
:10389800030E276E000E736F000E726FCCEF1EF0D2
:1038A800600E2818D8A45BEF1CF05DEF1CF076EFD3
:1038B8001CF001018C51D8B464EF1CF066EF1CF0C9
:1038C80076EF1CF08A51D8B46CEF1CF06EEF1CF048
:1038D80072EF1CF0090E276E4EEF1CF0050E276ED6
:1038E8004EEF1CF0680E2818D8A47DEF1CF07FEF6F
:1038F8001CF08FEF1CF001018C51D8B486EF1CF03E
:1039080088EF1CF08FEF1CF01A0E736F900E726F19
:103918008380CCEF1EF0680E2818D8A496EF1CF010
:1039280098EF1CF0AAEF1CF001018D51D8B49FEF5D
:103938001CF0A1EF1CF0AAEF1CF0020E276E000E7F
:103948000101736F000E726FCCEF1EF06A0E28181B
:10395800D8A4B1EF1CF0B3EF1CF0C3EF1CF00101C9
:103968008C51D8B4BAEF1CF0BCEF1CF0C3EF1CF0BC
:103978001A0E736FF40E726F8380CCEF1EF06C0E0C
:103988002818D8A4CAEF1CF0CCEF1CF0DCEF1CF010
:1039980001018C51D8B4D3EF1CF0D5EF1CF0DCEF4B
:1039A8001CF01A0E736F2C0E726F8380CCEF1EF012
:1039B800700E2818D8A4E3EF1CF0E5EF1CF0F7EF21
:1039C8001CF001018D51D8B4ECEF1CF0EEEF1CF0A7
:1039D800F7EF1CF0040E276E000E736F000E726F67
:1039E8008380CCEF1EF0700E2818D8A4FEEF1CF0D0
:1039F80000EF1DF0CCEF1EF001018C51D8B407EF99
:103A08001DF009EF1DF0CCEF1EF01B0E736F620E58
:103A1800726F8380CCEF1EF0020E2818D8A417EF1F
:103A28001DF019EF1DF01EEF1DF01A0E0101736F46
:103A3800920E726F050E2818D8A425EF1DF027EFF7
:103A48001DF02CEF1DF01A0E0101736FAE0E726F90
:103A5800070E2818D8A433EF1DF035EF1DF03AEF04
:103A68001DF01A0E0101736FB80E726F030E28183D
:103A7800D8B441EF1DF043EF1DF04BEF1DF028289F
:103A8800D8A449EF1DF04BEF1DF056EF1DF08380D1
:103A9800000E276E8390000E0101736F000E726F87
:103AA800CCEF1EF0160E2818D8A45DEF1DF05FEFBE
:103AB8001DF0CCEF1EF01A0E0101736FA40E726F89
:103AC800CCEF1EF0050E2818D8A46DEF1DF06FEF8F
:103AD8001DF0CCEF1EF01A0E0101736FF50E726F18
:103AE800CCEF1EF01A0E0101736F9B0E726FCCEFB4
:103AF8001EF028C049F01A0E0101736F9C0E726FF8
:103B0800CCEF1EF028C04AF01A0E0101736F9D0E0B
:103B1800726FCCEF1EF028C04BF01A0E0101736FC4
:103B28009E0E726FCCEF1EF028C04CF0000E010103
:103B3800736F000E726F010E276ECCEF1EF01A0E17
:103B48000101736FB90E726F8380CCEF1EF01A0EED
:103B58000101736FBA0E726FCCEF1EF01A0E0101DD
:103B6800736FBB0E726FCCEF1EF0000E0101736F06
:103B7800000E726F960E00018A6FFE0E8B6F4EEC70
:103B88006FF08390CCEF1EF0000E0101736F000EF2
:103B9800726F060E276ECCEF1EF0000E01018A6FC1
:103BA8001A0E736FF70E726F020ED9EC6EF08390D7
:103BB800CCEF1EF01A0E0101736FF70E726FCCEF87
:103BC8001EF08390270E0101736F0F0E726F030EA4
:103BD800D9EC6EF0CCEF1EF0180E2818D8A4F7EF29
:103BE8001DF0F9EF1DF0CCEF1EF01A0E0101736FF6
:103BF8002D0E726FCCEF1EF01A0E0101736F2E0E90
:103C0800726FCCEF1EF01A0E0101736F2F0E726FD8
:103C1800CCEF1EF01A0E0101736F300E726FCCEFED
:103C28001EF0000E0101736F000E726F0A0E276EF0
:103C38008390CCEF1EF0040E276E270E0101736FE0
:103C48000F0E726F8380CCEF1EF08380000E01018F
:103C5800736F000E726F000E276ECCEF1EF083900C
:103C6800010E01018A6F080E276E000E736F000E99
:103C7800726F000E276ECCEF1EF072C125F073C173
:103C880026F02650000AD8B458EF1EF01A0AD8B405
:103C98005FEF1EF0010AD8B4BAEF1EF03C0AD8B4A0
:103CA800C5EF1EF0CCEF1EF02550000AD8B42EEF59
:103CB8001CF0CCEF1EF025502C0AD8B4F0EF1DF004
:103CC800010AD8B400EF1EF0030AD8B407EF1EF0BB
:103CD800010AD8B40EEF1EF01F0AD8B415EF1EF073
:103CE800A00AD8B410EF1DF0020AD8B476EF1DF080
:103CF800090AD8B47DEF1DF0070AD8B486EF1DF085
:103D0800010AD8B48FEF1DF0030AD8B498EF1DF05C
:103D18003A0AD8B4C8EF1DF00A0AD8B433EF1EF037
:103D2800160AD8B4A3EF1DF0010AD8B4ABEF1DF002
:103D3800030AD8B4B2EF1DF0010AD8B4B9EF1DF0E8
:103D4800790AD8B4A1EF1CF0360AD8B466EF1DF092
:103D5800010AD8B4D1EF1DF0030AD8B4DEEF1DF084
:103D6800010AD8B4E5EF1DF0CCEF1EF02550580A33
:103D7800D8B41FEF1EF03A0AD8B429EF1EF0CCEFE2
:103D88001EF025500F0AD8B4CCEF1EF0CCEF1EF071
:103D980027C023F0246A12008EC0A9F08FC0AAF0B1
:103DA80092C0D9FF93C0DAFF000EDE6E000EDD6E02
:103DB8008CC00DF08DC00EF085EC63F00001A46F8F
:103DC800A451D8B4EAEF1EF0ECEF1EF0EFEF1EF0AE
:103DD800A45120EF22F020EE05F08C51D9268D5108
:103DE800DA22DF50D8B4FBEF1EF0FDEF1EF006EF2D
:103DF8001FF020EE05F08C51D9268D51DA22DF50C4
:103E080020EF22F020EE04F08C51D9268D51DA22D1
:103E1800DFB011EF1FF013EF1FF016EF1FF0070EC2
:103E280020EF22F020EE06F08C51D9268D51DA22AF
:103E3800DECF94F0DECF95F0DECF96F0DECF97F0B0
:103E480020EE0AF08C51D9268D51DA22DECF98F077
:103E5800DECF99F0DECF9AF0DECF9BF09451985DDB
:103E6800A06F95519959A16F96519A59A26F975180
:103E78009B59A36F9051946F9151956F966B976B67
:103E88009451A05D9551A1599651A2599751A359A2
:103E9800D8B051EF1FF053EF1FF016EF22F0A0C07B
:103EA80090F0A1C091F016EF22F020EE06F08C51B0
:103EB800D9268D51DA22FF0EDE14946F010EDE141E
:103EC800956F000EDE14966F000EDE14976F9451F6
:103ED800951196119711D8A474EF1FF076EF1FF083
:103EE80075EF21F020EE06F08C51D9268D51DA229B
:103EF800DECF94F0DECF95F0DECF96F0DECF97F0F0
:103F08000A0E8CEF1FF0D89097339633953394337D
:103F1800E82E87EF1FF08CC0D9FF8DC0DAFF10EEB6
:103F280002F0DE50E126DD50E222E750986F980556
:103F38009415AB6FAB51D8A4A4EF1FF0A6EF1FF0F8
:103F480027EF20F020EE06F08C51D9268D51DA2289
:103F5800DE50DE10DE10DE10D8A4B5EF1FF0B7EF8C
:103F68001FF0C7EF1FF020EE0EF08C51D9268D51AF
:103F7800DA22DECFA5F0DECFA6F0DECFA7F0DECFC7
:103F8800A8F0E7EF1FF08CC0D9FF8DC0DAFFDECFB5
:103F980060F0DDCF61F020EE12F08C51D9268D5102
:103FA800DA22DECF62F0DECF63F0DECF64F0DECF60
:103FB80065F072EC30F060C0A5F061C0A6F062C098
:103FC800A7F063C0A8F00001A851A711A61107E146
:103FD800020EA55DD8B0F3EF1FF0F5EF1FF000EF6C
:103FE80020F020EE05F08C51D9268D51DA22020EF0
:103FF800DF6E020E20EF22F0A5290AE1A62908E1CA
:10400800A72906E1A829D8A40CEF20F00EEF20F08C
:1040180019EF20F020EE05F08C51D9268D51DA22C7
:10402800010EDF6E010E20EF22F020EE12F08C510F
:10403800D9268D51DA22A5C0DEFFA6C0DEFFA7C0B3
:10404800DEFFA8C0DEFF8CC0D9FF8DC0DAFFDECF4F
:1040580018F0DDCF19F020EE12F08C51D9268D51D1
:10406800DA22DECF1AF0DECF1BF0DECF1CF0DECF77
:104078001DF04CEC64F018C0ACF019C0ADF01AC0DB
:10408800AEF01BC0AFF00001AC51AD11AE11AF11D5
:10409800D8A451EF20F053EF20F05DEF20F020EE90
:1040A80005F08C51D9268D51DA22020EDF6EFDEF14
:1040B8001FF0AB51AC27000EAD23AE23AF2390C049
:1040C80094F091C095F0090E966FD890953394337B
:1040D800962F69EF20F094C0B0F095C0B1F0B051C0
:1040E800B111D8B47AEF20F07CEF20F067EF21F01F
:1040F800AB51B025946F000EB121956F8CC0D9FFDC
:104108008DC0DAFF10EE02F0DE50E126DD50E2222B
:10411800E750966F976B9451965D95519759D8B023
:1041280098EF20F09AEF20F0ACEF20F08CC0D9FF88
:104138008DC0DAFF10EE02F0DE50E126DD50E222FB
:10414800E750946FAB51945DB06FB16BD8A0B107D5
:10415800A9C01BF0AAC01CF0ACC01DF0ADC01EF079
:10416800AEC01FF0AFC020F0B0C021F0B1C022F047
:104178008CC0D9FF8DC0DAFF10EE01F0DE50E126C9
:10418800DD50E222E75034EC5EF00009D8B4CFEFFE
:1041980020F0D1EF20F0DCEF20F0000120EE05F058
:1041A8008C51D9268D51DA22010EDF6E16EF20F0E0
:1041B8008CC0D9FF8DC0DAFF10EE04F0DE50E12686
:1041C800DD50E222E750D8B4ECEF20F0EEEF20F01B
:1041D80055EF21F00001B051946FB151956F966B76
:1041E800976B8CC0D9FF8DC0DAFF10EE2AF0DE5035
:1041F800E126DD50E222E6CF98F0E6CF99F0E6CF4F
:104208009AF0E6CF9BF0AC51985D9C6FAD519959EF
:104218009D6FAE519A599E6FAF519B599F6F9451A4
:104228009C5D95519D5996519E5997519F59D8B06B
:1042380020EF21F022EF21F055EF21F08CC0D9FFBB
:104248008DC0DAFF10EE2AF0DE50E126DD50E222C2
:10425800E6CF94F0E5CF95F0AC51945FAD51955B06
:10426800090ED89094379537E82E35EF21F0945100
:10427800A9250C6E9551AA210D6E8CC0D9FF8DC051
:10428800DAFFDECF96F0DDCF97F02E0E96250E6E74
:10429800000E97210F6E020E116E000E106E07ECC5
:1042A8006CF0B0C094F0B1C095F0090ED890000140
:1042B80094379537E82E5AEF21F094C0B2F095C0A4
:1042C800B3F0F8EF21F020EE16F08C51D9268D517D
:1042D800DA22ACC0DEFFADC0DEFFAEC0DEFFAFC08D
:1042E800DEFFFF0E946F010E956F20EE06F08C51E5
:1042F800D9268D51DA22DECF96F0DDCF97F0945192
:1043080096179551971796510008B26F9751D8A0F4
:10431800E82A0208B36FB251905DB3519159D8B0F1
:1043280098EF21F09AEF21F09EEF21F090C0B2F0C3
:1043380091C0B3F08CC0D9FF8DC0DAFFDECF3AF060
:10434800DDCF3BF020EE16F08C51D9268D51DA22C4
:10435800DECF3CF0DECF3DF0DECF3EF0DECF3FF0EB
:10436800AFEC64F00009D8B4BCEF21F0BEEF21F047
:10437800C9EF21F0000120EE05F08C51D9268D51AE
:10438800DA22010EDF6E16EF20F0A9C00CF0AAC0E9
:104398000DF0FF0E0001946F010E956F20EE06F0F0
:1043A8008C51D9268D51DA22DECF96F0DDCF97F0E9
:1043B80094519617955197178CC0D9FF8DC0DAFF85
:1043C800DECF98F0DDCF99F0965198279751992331
:1043D8002E0E98250E6E000E99210F6EB2C010F0A9
:1043E800B3C011F007EC6CF00001B251A927B3512A
:1043F800AA2320EE06F08C51D9268D51DA22B2512B
:10440800DE26B351DE22000EDE22DE2292C0D9FF64
:1044180093C0DAFFB251DE26B351DD22B251905F6C
:10442800B351915B90519111D8A41DEF22F01FEF69
:1044380022F059EF1FF0000E12002B6E1CC042F044
:104448001DC043F02B50D8B42CEF22F02EEF22F0F1
:1044580031EF22F0040E1AEF25F0010E406E51A044
:1044680038EF22F03AEF22F0EAEF24F0030E1AEFC9
:1044780025F053EC6EF00009D8B445EF22F047EF71
:1044880022F017EF25F0000E406E17EF25F0000E12
:10449800156E000E166E000E176E000E186E090EC1
:1044A8000FEC6BF00009D8A45CEF22F05EEF22F06D
:1044B80017EF25F02C0E0C6E000E0D6E000E0F6E11
:1044C800100E0E6E82EC67F00009D8B46EEF22F081
:1044D80070EF22F017EF25F02C44E846030BE806AE
:1044E800D8A479EF22F07BEF22F0CBEF22F033C093
:1044F8001EF03F0E1E161EC01FF0206A216A226A97
:1045080020C022F01FC021F0206A1F6A3450246E98
:10451800236A3550256E266A2350252624502622E4
:1045280025501F24276E26502020286E000E21209B
:10453800296E000E22202A6E010E27243C6E000EE2
:1045480028203D6E000E29203E6E000E2A203F6E68
:104558003CC01EF03DC01FF03EC020F03FC021F01F
:104568000A0ED8901E361F3620362136E82EB5EFB3
:1045780022F01CC0D9FF1DC0DAFF1EC0DEFF1FC01D
:10458800DEFF20C0DEFF21C0DEFF47EF22F01E6AFB
:1045980036AE01D01E2A010E1E1631C01FF00F0EB6
:1045A8001F163550030B020DF3501F241E24020F53
:1045B800416E3250030B1E6E1F6A0A0ED8901E36CB
:1045C8001F36E82EE2EF22F03350206E216AD89091
:1045D80020362136D890203621363444E846030B5D
:1045E800226E236A20502226215023221E50222682
:1045F8001F502322010E2226000E232222C03CF047
:1046080023C03DF03E6A3F6A41C01EF0F70E1E26E9
:104618003CC01FF03DC020F03EC021F03FC022F05A
:104628001E2A1CEF23F0D8901F362036213622365A
:104638001E2E17EF23F01CC0D9FF1DC0DAFF1FC0C4
:10464800DEFF20C0DEFF21C0DEFF22C0DEFF47EF15
:1046580022F04EA432EF23F034EF23F08DEF23F055
:10466800000E156E000E166E000E176E000E186EF8
:104678008D0E0FEC6BF00009D8A445EF23F047EF3F
:1046880023F017EF25F00CEC6FF02C0E0C6E000EDB
:104698000D6E000E0F6E100E0E6E82EC67F00009A4
:1046A800D8B459EF23F05BEF23F017EF25F0300E65
:1046B800416E62EF23F00CEC6FF041064150D8A434
:1046C80068EF23F06AEF23F05FEF23F036C01EF0A7
:1046D8001E3A0F0E1E16100E1F6E206A216A226ADD
:1046E8001E2A7CEF23F0D8901F362036213622363A
:1046F8001E2E77EF23F01CC0D9FF1DC0DAFF1FC0A4
:10470800DEFF20C0DEFF21C0DEFF22C0DEFF47EF54
:1047180022F0000E156E000E166E000E176E000EBB
:10472800186E090E0FEC6BF00009D8A49EEF23F069
:10473800A0EF23F017EF25F02C0E0C6E000E0D6E77
:10474800000E0F6E100E0E6E82EC67F00009D8B4E2
:10475800B0EF23F0B2EF23F017EF25F04EA2B7EF3A
:1047680023F0B9EF23F0F6EF23F039C01EF0060E60
:104778001F6ED8901E321F2EBDEF23F0FF0E1E268F
:1047880036503F0B206E216AD89020362136226A97
:1047980037AE01D0222A010E221622502026000E02
:1047A8002122010E2026000E21221E2ADFEF23F0EF
:1047B800D890203621361E2EDCEF23F02050236EB1
:1047C8002150246E256A266A1CC0D9FF1DC0DAFF55
:1047D80023C0DEFF24C0DEFF25C0DEFF26C0DEFFCB
:1047E80047EF22F036C01EF0D8901E32D8901E3205
:1047F8001F0E1E16010E1E240C6E0D6A000E0D22D1
:104808003750030B1F6E206AD8901F362036D89079
:104818001F362036D8901F36203637C021F0050EB7
:10482800226ED8902132222E15EF24F0070E211681
:1048380021501F26000E2022010E1F240E6E000E8E
:1048480020200F6E8EEC6EF00C50236E0D50246EEF
:10485800256A266A1CC0D9FF1DC0DAFF23C0DEFF07
:1048680024C0DEFF25C0DEFF26C0DEFF47EF22F0B2
:1048780042C0D9FF43C0DAFF4EC0DFFF47EF22F046
:10488800000E156E000E166E000E176E000E186ED6
:10489800090E0FEC6BF00009D8A455EF24F057EF80
:1048A80024F017EF25F042C00CF043C00DF0000EC5
:1048B8000F6E100E0E6E82EC67F00009D8B467EF29
:1048C80024F069EF24F017EF25F047EF22F0000EEF
:1048D800156E000E166E000E176E000E186E0A0E7C
:1048E8000FEC6BF00009D8A47CEF24F07EEF24F0E5
:1048F80017EF25F042C00CF043C00DF0000E0F6E0C
:10490800100E0E6E82EC67F00009D8B48EEF24F01A
:1049180090EF24F017EF25F047EF22F0000E156E08
:10492800000E166E000E176E000E186E3A0E0FEC83
:104938006BF00009D8A4A3EF24F0A5EF24F017EF3B
:1049480025F0040E416EB3EF24F00CEC6FF042C07A
:10495800D9FF43C0DAFFDF6E424A432A410641507D
:10496800D8A4B9EF24F0BBEF24F0A9EF24F047EF67
:1049780022F0000E156E000E166E000E176E000E59
:10498800186E8D0E0FEC6BF00009D8A4CEEF24F052
:10499800D0EF24F017EF25F00CEC6FF042C00CF0CC
:1049A80043C00DF0000E0F6E400E0E6E82EC67F0E5
:1049B8000009D8B4E2EF24F0E4EF24F017EF25F073
:1049C80047EF22F0040E406E17EF25F01B501E6EC5
:1049D8001F6A1F50000AD8B4F4EF24F0E6EF24F061
:1049E8001E50000AD8B43DEF22F0010AD8B44BEFAC
:1049F80022F0020AD8B42DEF23F0090AD8B43CEF0C
:104A080024F0010AD8B444EF24F0070AD8B46BEFB5
:104A180024F0010AD8B492EF24F0030AD8B4BDEF09
:104A280024F0E6EF24F077EC6FF04050120019C044
:104A3800F6FF1AC0F7FF0800F5CF89F0194A1A2ABD
:104A480000018951D8A42BEF25F02DEF25F02FEF89
:104A580025F011EF28F0250E8919D8B436EF25F086
:104A680038EF25F03DEF25F089511DEC6FF01BEF75
:104A780025F0000E856F000E846F19C0F6FF1AC06E
:104A8800F7FF0800F5CF89F0194A1A2A300E89195C
:104A9800D8A451EF25F053EF25F062EF25F0000E72
:104AA800856F010E846F19C0F6FF1AC0F7FF080062
:104AB800F5CF89F0194A1A2A71EF25F02D0E8919B8
:104AC800D8A469EF25F06BEF25F071EF25F0000E03
:104AD800856F020E846F57EF25F0000E7D6F000E74
:104AE8007C6F95EF25F07CC00CF07DC00DF0000EBA
:104AF8000F6E0A0E0E6E8EEC6EF0000189510C26B8
:104B0800000E0D22D00E0C247C6FFF0E0D207D6F41
:104B180019C0F6FF1AC0F7FF0800F5CF89F0194A47
:104B28001A2A2F0E89659BEF25F09DEF25F0A5EF3A
:104B380025F0390E8965A3EF25F0A5EF25F077EF6D
:104B480025F06C0E8919D8B4ACEF25F0AEEF25F03E
:104B5800B7EF25F04C0E8919D8A4B5EF25F0B7EFBB
:104B680025F0C1EF25F0848519C0F6FF1AC0F7FFBC
:104B78000800F5CF89F0194A1A2A8951D8A4C7EF35
:104B880025F0C9EF25F0CBEF25F011EF28F089C00B
:104B980088F0600E8865D3EF25F0D5EF25F084EF17
:104BA80026F0200E885F84EF26F01BC0D9FF1CC0BA
:104BB800DAFFDFCF1DF0020EDE26DFCF1EF0000E7B
:104BC800DD221DC0D9FF1EC0DAFFDECF78F0DDCFB1
:104BD80079F0000E7F6F000E7E6FF6EF25F0000172
:104BE8007E4B7F2B7E5178251D6E7F5179211E6E5D
:104BF8001DC0F6FF1EC0F7FF000EF86E0E0EF7641C
:104C080003D00800F55005D0F6CFE9FFF7CFEAFF4B
:104C1800EF500009D8A413EF26F015EF26F0F3EFB4
:104C280025F01AEF26F0200E1DEC6FF0000184B37A
:104C380020EF26F022EF26F033EF26F07E511D6E8E
:104C48007F511E6E7E4B7F2B7C511D5C7D511E5803
:104C5800D8A031EF26F033EF26F017EF26F078C012
:104C68000DF079C00EF080EC6AF03EEF26F0200ED1
:104C78001DEC6FF000017E511D6E7F511E6E7E4B44
:104C88007F2B7C511D5C7D511E58D8A04EEF26F01D
:104C980050EF26F03BEF26F01BEF25F01BC0D9FFA5
:104CA8001CC0DAFFDFCF1DF0020EDE26DFCF1EF0BC
:104CB800000EDD221DC0D9FF1EC0DAFFDF501DEC3B
:104CC8006FF01BEF25F0000E7B6F020E7A6FADEFD1
:104CD80026F0000E7B6F080E7A6FADEF26F0000EFF
:104CE8007B6F0A0E7A6FADEF26F0000E7B6F100E09
:104CF8007A6FADEF26F089511DEC6FF01BEF25F0B0
:104D080088511D6E1E6A1E50000AD8B48EEF26F018
:104D18007FEF26F01D50420AD8B467EF26F0010A4B
:104D2800D8B452EF26F0070AD8B473EF26F00B0A6E
:104D3800D8B46DEF26F01C0AD8B4D9EF25F0060ACE
:104D4800D8B473EF26F00D0AD8B479EF26F07FEFC8
:104D580026F084B5B2EF26F0B4EF26F0FCEF26F08B
:104D6800440E8819D8B4BBEF26F0BDEF26F0D9EF72
:104D780026F01BC0D9FF1CC0DAFFDFCF1DF0020EE2
:104D8800DE26DFCF1EF0000EDD221DC0D9FF1EC0BB
:104D9800DAFFDECF1FF0DDCF20F01FC070F020C09B
:104DA80071F0726B736BF2EF26F01BC0D9FF1CC059
:104DB800DAFFDFCF1DF0020EDE26DFCF1EF0000E79
:104DC800DD221DC0D9FF1EC0DAFFDECF70F0DDCFB7
:104DD80071F0000E71BFFF0E726F736F70C080F0BC
:104DE80071C081F072C082F073C083F014EF27F0B5
:104DF8001BC0D9FF1CC0DAFFDFCF1DF0040EDE2672
:104E0800DFCF1EF0000EDD221DC0D9FF1EC0DAFF65
:104E1800DECF80F0DECF81F0DECF82F0DECF83F010
:104E2800440E8819D8A41BEF27F01DEF27F02EEFAA
:104E380027F083AF22EF27F024EF27F02EEF27F09B
:104E4800806D811FD8B0812B821FD8B0822B000EB5
:104E580083578487000E876F000E866F80C00CF022
:104E680081C00DF082C00EF083C00FF07AC010F040
:104E78007BC011F0126A136AA6EC68F00C500001AE
:104E8800886F80C00CF081C00DF082C00EF083C026
:104E98000FF07AC010F07BC011F0126A136A30EC80
:104EA80067F00CC080F00DC081F00EC082F00FC01A
:104EB80083F0090E0001886564EF27F066EF27F09C
:104EC8007BEF27F0780E8919D8B46DEF27F06FEFD4
:104ED80027F075EF27F0000E756F070E746F79EFE6
:104EE80027F0000E756F270E746F74518827600EB7
:104EF8008625D96E000E8721DA6E8851300FDF6E55
:104F0800864B872B8051811182118311D8B48FEF82
:104F180027F091EF27F09CEF27F0875109E1100E59
:104F2800865DD8A09AEF27F09CEF27F032EF27F0A4
:104F380084A7A1EF27F0A3EF27F0ADEF27F0600ECD
:104F48008625D96E000E8721DA6E2D0EDF6E864B10
:104F5800872B86C07EF087C07FF084B1B6EF27F03C
:104F6800B8EF27F0BEEF27F0000E776F200E766FB0
:104F7800C2EF27F0000E776F300E766F76C088F09C
:104F8800C9EF27F088511DEC6FF0000184B3CFEF13
:104F980027F0D1EF27F0E2EF27F07E511D6E7F5109
:104FA8001E6E7E4B7F2B7C511D5C7D511E58D8A0F8
:104FB800E0EF27F0E2EF27F0C6EF27F08607D8A04A
:104FC8008707600E8625D96E000E8721DA6EDF50BE
:104FD8001DEC6FF0000186518711D8A4F6EF27F079
:104FE800F8EF27F0E2EF27F0FDEF27F0200E1DEC99
:104FF8006FF000017E511D6E7F511E6E7E4B7F2B20
:105008007C511D5C7D511E58D8A00DEF28F00FEF84
:1050180028F0FAEF27F01BEF25F012000001DD5110
:10502800DE11D8A41AEF28F01CEF28F01FEF28F0A3
:10503800090EFCEF2AF0DDC0D9FFDEC0DAFF000E52
:10504800DE6E000EDD6E7EC1C0F17FC1C1F11F0EA4
:10505800E117C00E846F010E856FDF0E866F000E9C
:10506800876FE151FE0B886F37EC01F00101BD6FCE
:10507800BD51D8A442EF28F044EF28F0FAEF2AF007
:10508800A90ED46F010ED56FC00E0001BD6F010EC1
:10509800BE6FDFC0BFF0E0C0C0F073EC52F001019A
:1050A800BD6FD2C1BEF1D3C1BFF1BD51D8A45FEF6E
:1050B80028F061EF28F06CEF28F0BE51BF11D8A49A
:1050C80068EF28F06AEF28F06CEF28F0060EBD6F45
:1050D800E1C0E2F01C0E0001E217D8B476EF28F028
:1050E80078EF28F0C4EF29F00101BD51D8B47FEF63
:1050F80028F081EF28F09BEF28F0040EBD19D8A402
:1051080088EF28F08AEF28F093EF28F0C00E00010E
:10511800C16F010EC26F85EC60F00101BD6F000127
:10512800E187D2C1BEF1D3C1BFF1BCEF28F020EEB8
:105138000BF0BE51D926BF51DA22DF500001E26FD1
:10514800110EE217D8B4ABEF28F0ADEF28F0B2EFAC
:1051580028F0070E0101BD6FBCEF28F0E1A5B7EFFD
:1051680028F0B9EF28F0BCEF28F0080E0101BD6F58
:105178000101BD51D8A4C3EF28F0C5EF28F0F6EF20
:1051880029F00001E1A7CBEF28F0CDEF28F0F6EFEA
:1051980029F0010120EE0EF0BE51D926BF51DA22C6
:1051A800000EDF6E20EE0FF0BE51D926BF51DA2275
:1051B800000EDF6E20EE10F0BE51D926BF51DA2264
:1051C800210EDF6E20EE11F0BE51D926BF51DA2232
:1051D800460EDF6E20EE16F0BE51D926BF51DA22F8
:1051E800000EDF6E20EE17F0BE51D926BF51DA222D
:1051F800000EDF6E20EE18F0BE51D926BF51DA221C
:10520800210EDF6E20EE19F0BE51D926BF51DA22E9
:10521800460EDF6E20EE0BF0BE51D926BF51DA22C2
:10522800000EDF6E20EE1CF0BE51D926BF51DA22E7
:10523800000EDF6E20EE1DF0BE51D926BF51DA22D6
:10524800000EDF6E20EE1EF0BE51D926BF51DA22C5
:10525800000EDF6E20EE1FF0BE51D926BF51DA22B4
:10526800000EDF6EC0C10CF0C1C10DF0BEC10EF062
:10527800BFC10FF0B9EC62F00CC0B5F10DC0B6F1CA
:105288000EC0B7F10FC0B8F1BEC10CF0BFC10DF030
:10529800000E0E6E000E0F6E000E106E000E116ED8
:1052A800DBEC6CF0010120EE04F0C051D926C151AD
:1052B800DA22010EDF6EB551B611B711B811D8B4A4
:1052C80068EF29F06AEF29F0F6EF29F020EE2AF0CE
:1052D800C051D926C151DA22DECFB9F1DECFBAF1F9
:1052E800DECFBBF1DECFBCF1C0C191F0C1C192F0FD
:1052F800B5C193F0B6C194F0B7C195F0B8C196F0B6
:1053080048EC55F00101BD6FBD51D8A48EEF29F0CE
:1053180090EF29F0F6EF29F0FF0EB5250001E26FB6
:10532800FF0E0101B6210001E36FFF0E0101B72155
:105338000001E46FFF0E0101B8210001E56F0101D2
:1053480020EE0AF0C051D926C151DA22E2C0DEFFB0
:10535800E3C0DEFFE4C0DEFFE5C0DEFFC0C13AF017
:10536800C1C13BF0B9C13CF0BAC13DF0BBC13EF090
:10537800BCC13FF0AFEC64F00101BD6FF6EF29F05E
:105388000101BD51D8A4CBEF29F0CDEF29F0F6EFFC
:1053980029F020EE0BF0BE51D926BF51DA22DFA842
:1053A800D8EF29F0DAEF29F0DEEF29F0040EBD6F0F
:1053B800F6EF29F00001E1A3E4EF29F0E6EF29F088
:1053C800F6EF29F0010120EE0BF0BE51D926BF51AE
:1053D800DA22DFA0F2EF29F0F4EF29F0F6EF29F056
:1053E800070EBD6F0101BD51D8A4FDEF29F0FFEFF5
:1053F80029F028EF2AF00001E1A705EF2AF007EFCE
:105408002AF008EF2AF0E18B010120EE2AF0C051C2
:10541800D926C151DA22000110EE1AF0DD51E12639
:10542800DE51E222DECFE6FFDECFE6FFDECFE6FF8B
:10543800DECFE6FF20EE1EF0DD51D926DE51DA225E
:10544800BEC1DEFFBFC1DDFF0101BD51D8A42FEFF2
:105458002AF031EF2AF0FAEF2AF0000120EE04F0EA
:10546800DD51D926DE51DA22E1C0DFFF20EE05F05A
:10547800DD51D926DE51DA22000EDF6EC0C10CF0F4
:10548800C1C10DF0BEC10EF0BFC10FF0B9EC62F0A2
:10549800000120EE0EF0DD51D926DE51DA220CC0D3
:1054A800DEFF0DC0DEFF0EC0DEFF0FC0DEFF010114
:1054B80020EE1DF0BE51D926BF51DA22DF5000017F
:1054C800E26FE251E46FE36B010120EE1EF0BE5182
:1054D800D926BF51DA22DF500001E56FE5C0E6F0BA
:1054E800E76BE86BE96BE7C0E9F0E6C0E8F0E76B6B
:1054F800E66B010120EE1FF0BE51D926BF51DA221A
:10550800DF500001EA6FEAC0EBF0EC6BED6BEE6B7D
:10551800EBC0EEF0ED6BEC6BEB6BE651EB11EF6F64
:10552800E751EC11F06FE851ED11F16FE951EE110F
:10553800F26FE351EF11F36FE451F011F46F000EC5
:10554800F111F56F000EF211F66F010120EE1CF05B
:10555800BE51D926BF51DA22DF500001F76FF7514B
:10556800F311F86FF451F96FF551FA6FF651FB6FBB
:1055780020EE0AF0DD51D926DE51DA22F8C0DEFF2E
:10558800F9C0DEFFFAC0DEFFFBC0DEFF20EE06F04A
:10559800DD51D926DE51DA22DE6ADE6ADE6ADD6A8C
:1055A80020EE16F0DD51D926DE51DA22DE6ADE6AF7
:1055B800DE6ADD6ADDC0D9FFDEC0DAFFC0C1DEFF0A
:1055C800C1C1DDFFDDC0D9FFDEC0DAFF10EE06F095
:1055D800DE50E126DD50E22220EE02F0DD51D92630
:1055E800DE51DA22E6CFDEFFE5CFDDFF0101BD5156
:1055F8001200000165516411631109E1020E625D38
:10560800D8A009EF2BF00BEF2BF020EF2BF020EEBA
:1056180012F06051D9266151DA22DE50625DDE5007
:105628006359DE506459DE506559D8A01EEF2BF03F
:1056380020EF2BF0B8EF2DF0020E8E6FD5EF2DF086
:1056480062C08CF063C08DF0D8908D316B6F8C3157
:105658006A6F6A518C276B518D2360C03AF061C024
:105668003BF020EE1EF06051D9266151DA22DECFE0
:105678006AF0DECF6BF0DECF6CF0DECF6DF08CC061
:105688006EF08DC06FF0090E706FD8906F336E3367
:10569800702F49EF2BF06E516A253C6E6F516B21CC
:1056A8003D6E000E6C213E6E000E6D213F6EAFEC1C
:1056B80064F000018E6F8E51D8B465EF2BF067EF60
:1056C8002BF069EF2BF0D5EF2DF0FF0E6A6F010E6E
:1056D8006B6F8CC06CF08DC06DF06A516C176B519C
:1056E8006D1760C06EF061C06FF06C516E276D5120
:1056F8006F232E0E6E258F6F000E6F21906F8C4BCF
:105708008D2B62B18AEF2BF08CEF2BF091EF2BF001
:1057180066C088F0896BABEF2BF066516A6F6B6BD4
:105728006A3B6B3BF00E6B176A510F0B6B13F00E55
:105738006A178FC0D9FF90C0DAFFDF500F0B6C6F6C
:105748006D6B6A516C11886F6B516D11896F8FC0C9
:10575800D9FF90C0DAFF88C0DFFF20EE04F0605167
:10576800D9266151DA22010EDF6E60C03AF061C0BD
:105778003BF020EE1EF06051D9266151DA22DECFCF
:105788006AF0DECF6BF0DECF6CF0DECF6DF08CC050
:105798006EF08DC06FF0090E706FD8906F336E3356
:1057A800702FD1EF2BF06E516A253C6E6F516B2133
:1057B8003D6E000E6C213E6E000E6D213F6EAFEC0B
:1057C80064F000018E6F8E51D8B4EDEF2BF0EFEF3F
:1057D8002BF0F1EF2BF0D5EF2DF0FF0E6A6F010ED5
:1057E8006B6F8CC06CF08DC06DF06A516C176B518B
:1057F8006D1760C06EF061C06FF06C516E276D510F
:105808006F232E0E6E258F6F000E6F21906F62B181
:1058180010EF2CF012EF2CF030EF2CF066C06AF08D
:1058280067C06BF068C06CF069C06DF06BC06AF05F
:105838006CC06BF06DC06CF06D6B0F0E6A178FC08B
:10584800D9FF90C0DAFFDF50F00B6A116E6F6E510E
:105858008A6F8B6B46EF2CF066C06AF067C06BF0FE
:1058680068C06CF069C06DF0050E40EF2CF0D89060
:105878006D336C336B336A33E82E3BEF2CF06A518F
:105888008A6F8B6B8FC0D9FF90C0DAFF8AC0DFFFA9
:1058980020EE04F06051D9266151DA22010EDF6E44
:1058A800D5EF2DF060C03AF061C03BF020EE1EF05D
:1058B8006051D9266151DA22DECF6AF0DECF6BF073
:1058C800DECF6CF0DECF6DF062C06EF063C06FF0BB
:1058D80064C070F065C071F06FC06EF070C06FF09A
:1058E80071C070F0716B6A516E253C6E6B516F21FF
:1058F8003D6E6C5170213E6E6D5171213F6EAFEC63
:1059080064F000018E6F8E51D8B48DEF2CF08FEFBC
:105918002CF091EF2CF0D5EF2DF0FF0E6A6F010EF1
:105928006B6F62C06CF063C06DF0D8906C376D37E8
:105938006A516C176B516D1760C06EF061C06FF0E3
:105948006C516E276D516F232E0E6E258F6F000ED2
:105958006F21906F8FC0D9FF90C0DAFF66C0DFFF5C
:1059680020EE01F08F51D9269051DA226751DF6E6F
:1059780020EE04F06051D9266151DA22010EDF6E63
:10598800D5EF2DF060C03AF061C03BF020EE1EF07C
:105998006051D9266151DA22DECF6AF0DECF6BF092
:1059A800DECF6CF0DECF6DF062C06EF063C06FF0DA
:1059B80064C070F065C071F0080EE8EF2CF0D89064
:1059C800713370336F336E33E82EE3EF2CF06A5186
:1059D8006E253C6E6B516F213D6E6C5170213E6E91
:1059E8006D5171213F6EAFEC64F000018E6F8E51E6
:1059F800D8B401EF2DF003EF2DF005EF2DF0D5EF22
:105A08002DF0FF0E6A6F010E6B6F62C06CF063C001
:105A18006DF0D8906C376D37D8906C376D376A5108
:105A28006C176B516D1760C06EF061C06FF06C51F0
:105A38006E276D516F232E0E6E258F6F000E6F210E
:105A4800906F20EE01F08F51D9269051DA22DF5065
:105A58006A6F6A516C6F6B6B20EE02F08F51D9261A
:105A68009051DA22DF506D6F6DC06EF06F6B706B06
:105A7800716B6FC071F06EC070F06F6B6E6B20EE63
:105A880003F08F51D9269051DA22DF50726F72C01D
:105A980073F0746B756B766B73C076F0756B746BA3
:105AA800736B6E517311776F6F517411786F7051FA
:105AB8007511796F715176117A6F6B5177117B6F10
:105AC8006C5178117C6F000E79117D6F000E7A1180
:105AD8007E6F8FC0D9FF90C0DAFFDF507F6F7F5194
:105AE8007B11806F7C51816F7D51826F7E51836FF6
:105AF800000E8015846F000E8115856F000E8215CB
:105B0800866FF00E8315876F84516613855167136E
:105B180086516813875169138FC0D9FF90C0DAFF87
:105B280066C0DFFF20EE01F08F51D9269051DA22AE
:105B38006751DF6E20EE02F08F51D9269051DA229C
:105B480068C0DFFF20EE03F08F51D9269051DA228A
:105B580069C0DFFF20EE04F06051D9266151DA22D6
:105B6800010EDF6ED5EF2DF060C0D9FF61C0DAFFFE
:105B7800DF506A6F6B6B6B51000AD8B4C6EF2DF01B
:105B880020EF2BF06A51010AD8B424EF2BF0030A56
:105B9800D8B456EF2CF0010AD8B4C6EF2CF020EF99
:105BA8002BF08E511200040E00018C6F020E8D6FC7
:105BB800340E8E6F0B0E8F6F020E916F000E906F6A
:105BC800E50E926F000E936FD0EC1EF04F6EE40E50
:105BD80000018A6FFD0E8B6FE5C08CF0E6C08DF07A
:105BE8004EEC6FF0000E0001E86F000EE76F000E3C
:105BF800E26F000EE16F000EEA6F000EE96FC30E50
:105C0800E925D96E000EEA21DA6E000EDF6ED20E9B
:105C1800E925D96E000EEA21DA6E000EDF6EE94B37
:105C2800EA2BEABF21EF2EF0EA5109E10F0EE95DF8
:105C3800D8A021EF2EF023EF2EF003EF2EF0000E68
:105C4800EC6F000EEB6FDAEF2FF0340EEB25D96E08
:105C58000B0EEC21DA6E0D0EDE18D8A436EF2EF0FE
:105C680038EF2EF077EF2FF0930E0C6EFF0E0D6EBF
:105C7800C30E0E6E000E0F6ECFEC65F00C500D10BB
:105C8800D8A449EF2EF04BEF2EF054EF2EF0D20EA1
:105C9800136E000E146E8CEC58F013500101E26F75
:105CA8008D0E0C6EFF0E0D6EC30E0E6E000E0F6E77
:105CB800CFEC65F00C500D10D8A465EF2EF067EF0F
:105CC8002EF070EF2EF0D20E136E000E146E8CECC8
:105CD80058F0135001019C6F720E0C6EFF0E0D6E82
:105CE800C30E0E6E000E0F6ECFEC65F00C500D104B
:105CF800D8A481EF2EF083EF2EF08CEF2EF0D20E89
:105D0800136E000E146E8CEC58F013500101976F4F
:105D1800D10E0C6EFF0E0D6EC30E0E6E000E0F6EC2
:105D2800CFEC65F00C500D10D8A49DEF2EF09FEF2E
:105D38002EF0A8EF2EF0D20E136E000E146E8CEC1F
:105D480058F013500101956F000E0001EE6F000E20
:105D5800ED6FB40E826F000E836F790E846FFF0EA5
:105D6800856FEDC086F0EEC087F065EC6BF0B40E81
:105D78000C6E000E0D6EC30E0E6E000E0F6ECFEC85
:105D880065F00C500D10D8A4CCEF2EF0CEEF2EF00D
:105D9800E8EF2EF0EDC00CF0EEC00DF0000E0F6E27
:105DA8000F0E0E6E8EEC6EF0340E0C24126E0D0E6D
:105DB8000D20136ED20E146E000E156E000E176EA7
:105DC8000F0E166EEAEC68F00001ED4BEE2BEEBFFD
:105DD800F7EF2EF0EE5109E1100EED5DD8A0F7EFC8
:105DE8002EF0F9EF2EF0ADEF2EF0000EEE6F010E53
:105DF800ED6FB40E826F000E836F800E846FFF0EFE
:105E0800856FEDC086F0EEC087F065EC6BF0B40EE0
:105E18000C6E000E0D6EC30E0E6E000E0F6ECFECE4
:105E280065F00C500D10D8A41CEF2FF01EEF2FF0CA
:105E380038EF2FF0EDC00CF0EEC00DF0000E0F6E35
:105E48000F0E0E6E8EEC6EF0240E0C24126E0E0EDB
:105E58000D20136ED20E146E000E156E000E176E06
:105E68000F0E166EEAEC68F00001ED4BEE2BEEBF5C
:105E780047EF2FF0EE5109E1040EED5DD8A047EF92
:105E88002FF049EF2FF0FDEF2EF0000EEA6F000E15
:105E9800E96FC30EE925D96E000EEA21DA6E000E0D
:105EA800DF6ED20EE925D96E000EEA21DA6E000EF9
:105EB800DF6EE94BEA2BEABF6BEF2FF0EA5109E1FD
:105EC8000F0EE95DD8A06BEF2FF06DEF2FF04DEFBF
:105ED8002FF0000EE26F000EE16F000EE86F000E6B
:105EE800E76FD8EF2FF0340EEB25D96E0B0EEC21AF
:105EF800DA6E0A0EDE18D8A484EF2FF086EF2FF0A2
:105F080088EF2FF0D8EF2FF0340EEB25D96E0B0E5B
:105F1800EC21DA6E200EDE18D8A495EF2FF097EF5B
:105F28002FF0A1EF2FF0000EE26F010EE16F000ECF
:105F3800E86F000EE76FD8EF2FF0E151E211D8B407
:105F4800A8EF2FF0AAEF2FF0BAEF2FF0340EEB25C1
:105F5800D96E0B0EEC21DA6ED20EE725E16E000E3B
:105F6800E821E26EDFCFE7FFC8EF2FF0340EEB2514
:105F7800D96E0B0EEC21DA6EC30EE725E16E000E2A
:105F8800E821E26EDFCFE7FFE8BFD6EF2FF0E85158
:105F980007E10F0EE75DD8B0D4EF2FF0D6EF2FF062
:105FA800D8EF2FF0E74BE82BEB4BEC2BE551EB5DF3
:105FB800E651EC59D8A0E3EF2FF0E5EF2FF029EFE9
:105FC8002EF0D40E8A6FFD0E8B6F97C18CF08D6BFF
:105FD8004EEC6FF0300E00018A6FFE0E8B6FE2C13F
:105FE8008CF08D6B4EEC6FF0210E00018A6FFE0E67
:105FF8008B6F9CC18CF08D6B4EEC6FF0000E000126
:10600800EE6F000EED6FEDC00CF0EEC00DF0000E5F
:106018000F6E0F0E0E6E8EEC6EF0340E0C24000117
:10602800E36F0D0E0D20E46F520E8A6FFD0E8B6F1D
:10603800EDC08CF0EEC08DF0E3C08EF0E4C08FF0C0
:106048004EEC6FF00001ED4BEE2BEEBF35EF30F06C
:10605800EE5109E1100EED5DD8A035EF30F037EFC5
:1060680030F007EF30F0000EEC6F010EEB6FEBC075
:106078000CF0ECC00DF0000E0F6E0F0E0E6E8EECD5
:106088006EF0240E0C240001E36F0E0E0D20E46F59
:10609800630E8A6FFD0E8B6FEBC08CF0ECC08DF039
:1060A800E3C08EF0E4C08FF04EEC6FF00001EB4BD4
:1060B800EC2BECBF69EF30F0EC5109E1040EEB5D1D
:1060C800D8A069EF30F06BEF30F03BEF30F0850E81
:1060D8008A6FFC0E8B6F4EEC6FF012000001655159
:1060E8006411631109E1020E625DD8A07EEF30F001
:1060F80080EF30F095EF30F020EE12F06051D926A5
:106108006151DA22DE50625DDE506359DE50645917
:10611800DE506559D8A093EF30F095EF30F09FEF3F
:1061280030F0010E846F000E856F000E866F000E32
:10613800876FDFEF32F08469856986698769C2EF06
:1061480032F062C088F063C089F0D8908931676FF7
:106158008831666F665188276751892360C03AF095
:1061680061C03BF020EE1EF06051D9266151DA2261
:10617800DECF66F0DECF67F0DECF68F0DECF69F005
:1061880088C06AF089C06BF0090E6C6FD8906B33C9
:106198006A336C2FCAEF30F06A5166253C6E6B513A
:1061A80067213D6E000E68213E6E000E69213F6E2C
:1061B800AFEC64F00009D8B4E4EF30F0E6EF30F06B
:1061C800E8EF30F0DFEF32F0FF0E0001666F010EEE
:1061D800676F88C068F089C069F0665168176751B1
:1061E800691760C06AF061C06BF068516A2769512D
:1061F8006B232E0E6A25D96E000E6B21DA6EDF50E6
:106208006C6F6C51826F836B884B892B60C03AF03E
:1062180061C03BF020EE1EF06051D9266151DA22B0
:10622800DECF66F0DECF67F0DECF68F0DECF69F054
:1062380088C06AF089C06BF0090E6C6FD8906B3318
:106248006A336C2F22EF31F06A5166253C6E6B5130
:1062580067213D6E000E68213E6E000E69213F6E7B
:10626800AFEC64F00009D8B43CEF31F03EEF31F008
:1062780040EF31F0DFEF32F0FF0E0001666F010EE4
:10628800676F88C068F089C069F066516817675100
:10629800691760C06AF061C06BF068516A2769517C
:1062A8006B232E0E6A25D96E000E6B21DA6EDF5035
:1062B8006C6F6C516E6F6D6B6D5182136E518313E1
:1062C80062B169EF31F06BEF31F073EF31F0FF0E2F
:1062D8008215806F0F0E8315816F83EF31F082C0B6
:1062E80066F083C067F0040E686FD8906733663332
:1062F800682F79EF31F066C080F067C081F080C008
:1063080084F081C085F0866B876BDFEF32F060C068
:106318003AF061C03BF020EE1EF06051D926615181
:10632800DA22DECF66F0DECF67F0DECF68F0DECFB0
:1063380069F062C06AF063C06BF064C06CF065C05D
:106348006DF06BC06AF06CC06BF06DC06CF06D6B7B
:1063580066516A253C6E67516B213D6E68516C2110
:106368003E6E69516D213F6EAFEC64F00009D8B400
:10637800C0EF31F0C2EF31F0C4EF31F0DFEF32F0AF
:10638800FF0E0001666F010E676F62C068F063C0A0
:1063980069F0D89068376937665168176751691787
:1063A80060C06AF061C06BF068516A2769516B235D
:1063B8002E0E6A258A6F000E6B218B6F20EE01F07E
:1063C8008A51D9268B51DA22DF50666F6651686F81
:1063D800676B8AC0D9FF8BC0DAFFDF50696F6951DC
:1063E8006713000E681367C084F068C085F0866B79
:1063F800876BDFEF32F060C03AF061C03BF020EE0F
:106408001EF06051D9266151DA22DECF66F0DECF68
:1064180067F0DECF68F0DECF69F062C06AF063C073
:106428006BF064C06CF065C06DF0080E21EF32F0BF
:10643800D8906D336C336B336A33E82E1CEF32F02F
:1064480066516A253C6E67516B213D6E68516C211F
:106458003E6E69516D213F6EAFEC64F00009D8B40F
:1064680038EF32F03AEF32F03CEF32F0DFEF32F053
:10647800FF0E0001666F010E676F62C068F063C0AF
:1064880069F0D89068376937D890683769376651A6
:1064980068176751691760C06AF061C06BF068518E
:1064A8006A2769516B232E0E6A258A6F000E6B21AD
:1064B8008B6F20EE01F08A51D9268B51DA22DF50FA
:1064C800666F6651686F676B20EE02F08A51D926B5
:1064D8008B51DA22DF50696F69C06AF06B6B6C6BA5
:1064E8006D6B6BC06DF06AC06CF06B6B6A6B20EE05
:1064F80003F08A51D9268B51DA22DF506E6F6EC0B5
:106508006FF0706B716B726B6FC072F0716B706B48
:106518006F6B6A516F11736F6B517011746F6C519F
:106528007111756F6D517211766F67517311776FB5
:1065380068517411786F000E7511796F000E76111D
:106548007A6F8AC0D9FF8BC0DAFFDF507B6F7B512F
:1065580077117C6F78517D6F79517E6F7A517F6F9B
:10656800FF0E7C15846FFF0E7D15856FFF0E7E155F
:10657800866F0F0E7F15876FDFEF32F060C0D9FF8F
:1065880061C0DAFFDF50666F676B6751000AD8B4E5
:10659800D0EF32F095EF30F06651010AD8B4A5EF8C
:1065A80030F0030AD8B48BEF31F0010AD8B4FFEF0A
:1065B80031F095EF30F084C060F085C061F086C09E
:1065C80062F087C063F01200000120EE04F0A451CD
:1065D800D926A551DA22DECFA8F0DDCFA9F0010E29
:1065E800A825B16F000EA921B26FB151B211D8B46C
:1065F80000EF33F002EF33F013EF33F020EE0EF03C
:10660800A451D926A551DA22DE50DE10DE10DE10A4
:10661800D8A411EF33F013EF33F016EF33F0040E74
:106628004CEF35F00F0EB115A86F000EB215A96F1B
:10663800A851A911D8A423EF33F025EF33F01AEFAE
:1066480035F020EE0EF0A451D926A551DA22DE2A23
:10665800000EDE22DE22DE2220EE0AF0A451D92628
:10666800A551DA22DE50DE10DE10DE10D8A43FEF8E
:1066780033F041EF33F058EF33F0A4C0D9FFA5C091
:10668800DAFF10EE08F0DE50E126DD50E222E65097
:10669800B15DE650B259D8A054EF33F056EF33F05D
:1066A8001AEF35F013EF33F0B1C0A8F0B2C0A9F07B
:1066B800040EAA6FD890A933A833AA2F5EEF33F03F
:1066C800FF0EAB6FFF0EAC6FA4C0D9FFA5C0DAFFF9
:1066D80010EE02F0DE50E126DD50E222E750AD6F09
:1066E800AE6BAB51AD27AC51AE23A851AD17A95134
:1066F800AE17AD51AE11D8A484EF33F086EF33F066
:106708001AEF35F0A4C0D9FFA5C0DAFFDECF60F0DC
:10671800DDCF61F020EE0AF0A451D926A551DA2286
:10672800DECF62F0DECF63F0DECF64F0DECF65F05F
:1067380072EC30F060C0B3F061C0B4F062C0B5F084
:1067480063C0B6F00001B651B511B41107E1020EED
:10675800B35DD8B0B2EF33F0B4EF33F0B7EF33F046
:10676800020E4CEF35F0B3290AE1B42908E1B52946
:1067780006E1B629D8A4C3EF33F0C5EF33F0C8EF6C
:1067880033F0010E4CEF35F0A4C0D9FFA5C0DAFFF5
:1067980010EE12F0DE50E126DD50E222E650B35D45
:1067A800E650B459E650B559E650B659D8A0DFEFCF
:1067B80033F0E1EF33F0EBEF34F0A651A711D8A492
:1067C800E8EF33F0EAEF33F0ECEF33F013EF33F0A8
:1067D800A4C0D9FFA5C0DAFFDECF91F0DDCF92F0DB
:1067E80020EE0AF0A451D926A551DA22DECF93F083
:1067F800DECF94F0DECF95F0DECF96F066EC3BF07E
:1068080091C0B3F092C0B4F093C0B5F094C0B6F0A4
:106818000001B351B411B511B611D8A416EF34F074
:1068280018EF34F01BEF34F0070E4CEF35F0B305DA
:10683800B411B511B611D8A424EF34F026EF34F012
:1068480028EF34F0B4EF33F0B3290AE1B42908E1B2
:10685800B52906E1B629D8A434EF34F036EF34F080
:1068680038EF34F0C5EF33F0A4C0D9FFA5C0DAFF84
:10687800DECF25F0DDCF26F015EC5AF00009D8B4AC
:1068880048EF34F04AEF34F04CEF34F0C5EF33F012
:10689800A4C0D9FFA5C0DAFFDECFA8F0DDCFA9F0EC
:1068A8002E0E0001A8250C6E000EA9210D6E000EFB
:1068B8000F6E000E0E6E020E116E000E106E92EC30
:1068C8006DF0A4C0D9FFA5C0DAFFDECF18F0DDCF88
:1068D80019F0B3C01AF0B4C01BF0B5C01CF0B6C0B4
:1068E8001DF04CEC64F0A4C0D9FFA5C0DAFF10EE8F
:1068F8002AF0DE50E126DD50E22218C0E6FF19C07A
:10690800E6FF1AC0E6FF1BC0E6FF000E0001B06FED
:10691800000EAF6FC2EF34F0A4C0D9FFA5C0DAFFF4
:1069280010EE04F0DE50E126DD50E222010EE76EA3
:10693800A4C0D9FFA5C0DAFFDECF25F0DDCF26F051
:1069480015EC5AF00009D8B4ACEF34F0AEEF34F0DF
:10695800B0EF34F0C5EF33F0A4C0D9FFA5C0DAFF1B
:1069680010EE2AF0DE50E126DD50E222E62A000E83
:10697800E622E622E6220001AF4BB02BA4C0D9FFE5
:10698800A5C0DAFF10EE02F0DE50E126DD50E2226B
:10699800E750A86FA96BA851AF5DA951B059D8A00D
:1069A800D8EF34F0DAEF34F090EF34F0A4C0D9FF28
:1069B800A5C0DAFF10EE2AF0DE50E126DD50E22213
:1069C800AF51E65EB051E65A000EE65AE65A20EE9E
:1069D8000AF0A451D926A551DA22B3C0DEFFB4C00B
:1069E800DEFFB5C0DEFFB6C0DEFFA4C0D9FFA5C07C
:1069F800DAFFDECF18F0DDCF19F0B3C01AF0B4C05B
:106A08001BF0B5C01CF0B6C01DF04CEC64F00001E2
:106A180020EE0EF0A451D926A551DA2218C0DEFFC7
:106A280019C0DEFF1AC0DEFF1BC0DEFF20EE04F037
:106A3800A451D926A551DA22B1C0DEFFB2C0DDFFCC
:106A48000F0EB115A86F000EB215A96F050ED890DC
:106A5800A837A937E82E2BEF35F0A4C0D9FFA5C079
:106A6800DAFFDECFAAF0DDCFABF0A851AA27A951F3
:106A7800AB232E0EAA27000EAB2320EE12F0A45152
:106A8800D926A551DA22AAC0DEFFABC0DDFF000E71
:106A9800120016C0D9FF17C0DAFFDECF24F0DDCF11
:106AA80025F059EF35F0244A252A24C0F6FF25C0E1
:106AB800F7FF000EF86E0E0EF76403D00800F550CD
:106AC80005D0F6CFE9FFF7CFEAFFEF502F0AD8B489
:106AD80070EF35F072EF35F057EF35F024C0F6FF60
:106AE80025C0F7FF000EF86E0E0EF76403D00800FD
:106AF800F55005D0F6CFE9FFF7CFEAFFEF505C0A73
:106B0800D8B489EF35F08BEF35F057EF35F020EE3C
:106B180014F01450D9261550DA22DECF26F0DDCF36
:106B280027F026C00CF027C00DF0000E0F6E200EC7
:106B38000E6E000E116E0B0E106E92EC6DF0000EC4
:106B4800206E20C028F0296A28C01EF029C01FF036
:106B5800000E226E080E216E1E502424186E1F503F
:106B68002520196E18C0F6FF19C0F7FF000EF86E41
:106B78000E0EF76403D00800F55005D0F6CFE9FFF4
:106B8800F7CFEAFFEF502A6E1E4A1F2A200E2A640A
:106B9800D0EF35F0D2EF35F0F7EF36F02F0E2A1898
:106BA800D8B4D9EF35F0DBEF35F0F7EF36F05C0EFF
:106BB8002A18D8A4E2EF35F0E4EF35F0E6EF35F027
:106BC800F7EF36F02E0E2A18D8B4EDEF35F0EFEFC8
:106BD80035F0FAEF35F02150285C22502958D8A01A
:106BE800F8EF35F0FAEF35F01EEF36F0080E211801
:106BF8002210D8A402EF36F004EF36F00DEF36F08D
:106C08002E0E2A18D8B40BEF36F00DEF36F010EF31
:106C180036F0060E64EF37F0000E296E080E286E67
:106C2800000E226E0B0E216ED8902036D89020369A
:106C3800B0EF35F07F0E2A6424EF36F026EF36F0F9
:106C480028EF36F0030E2012800E2A642EEF36F05D
:106C580030EF36F038EF36F09F0E2A6436EF36F014
:106C680038EF36F048EF36F0DF0E2A643EEF36F0A4
:106C780040EF36F0B1EF36F0FD0E2A6046EF36F001
:106C880048EF36F0B1EF36F01E502424186E1F502E
:106C98002520196E18C0F6FF19C0F7FF000EF86E10
:106CA8000E0EF76403D00800F55005D0F6CFE9FFC3
:106CB800F7CFEAFFEF50236E1E4A1F2A3F0E2364C8
:106CC80068EF36F06AEF36F072EF36F07E0E236426
:106CD80070EF36F072EF36F082EF36F07F0E2364F5
:106CE80078EF36F07AEF36F00DEF36F0FD0E2360D0
:106CF80080EF36F082EF36F00DEF36F0FF0E186EAB
:106D0800FF0E196E21C01AF022C01BF018501A2667
:106D180019501B221A50285C1B502958D8A097EFED
:106D280036F099EF36F09BEF36F00DEF36F028503D
:106D38002624D96E29502720DA6E2AC0DFFF284A78
:106D4800292A28502624D96E29502720DA6E23C0F4
:106D5800DFFF284A292AB0EF35F0030E0C6EFE0E2D
:106D68000D6E2AC00EF00F6AB1EC6AF00C500D10CF
:106D7800D8B4C1EF36F0C3EF36F0C5EF36F00DEFFB
:106D880036F0400E2A64CBEF36F0CDEF36F0D8EF70
:106D980036F05B0E2A60D3EF36F0D5EF36F0D8EF39
:106DA80036F02082EBEF36F0600E2A64DEEF36F024
:106DB800E0EF36F0EBEF36F07B0E2A60E6EF36F0C8
:106DC800E8EF36F0EBEF36F02080200E2A5E2850F0
:106DD8002624D96E29502720DA6E2AC0DFFF284AD8
:106DE800292AB0EF35F01E502424186E1F50252094
:106DF800196E16C0D9FF17C0DAFF18C0DEFF19C018
:106E0800DDFF200E2A640BEF37F00DEF37F013EF9C
:106E180037F0000E1D6E000E1C6E17EF37F0000ED7
:106E28001D6E040E1C6E1CC02AF028502910D8A410
:106E380020EF37F022EF37F024EF37F00DEF36F080
:106E480026C0D9FF27C0DAFFE50EDE18D8A42FEF39
:106E580037F031EF37F037EF37F026C0D9FF27C0CA
:106E6800DAFF050EDF6E080E21182210D8A43FEFB6
:106E780037F041EF37F045EF37F0D8902036D8900B
:106E880020362050030BE806D8A44DEF37F04FEF1B
:106E980037F050EF37F02A8820500C0B040AD8A49A
:106EA80058EF37F05AEF37F05BEF37F02A8620EECD
:106EB8000BF02650D9262750DA222AC0DFFF000E11
:106EC800120083803B0E00018A6FF80E8B6FCECFC5
:106ED8008CF08D6BCDCF8EF08F6BFF51140D070E9C
:106EE800F324D96E010EF420DA6EDECF90F0DECFF7
:106EF80091F0DECF92F0DECF93F0FF51140D070E24
:106F0800F324D96E010EF420DA6EDECF94F0DECFD2
:106F180095F0DECF96F0DECF97F04EEC6FF062EC96
:106F280051F0CBC0EEF0CCC0EFF00001EE51EF1104
:106F3800D8B4A1EF37F0A3EF37F0BEEF37F0FF5129
:106F4800140D130EF324D96E010EF420DA6EFF51DE
:106F5800140D130EF324E16E010EF420E26EE750D7
:106F68000409DF6E1AEC6DF0EEC0E2F0EFC0E3F05A
:106F780070EF39F0FF51140D0F0EF324D96E010E86
:106F8800F420DA6EDECFE4F0DECFE5F0DECFE6F017
:106F9800DECFE7F0E5C0E4F0E6C0E5F0E7C0E6F0F4
:106FA800E76BE4C0E8F0E5C0E9F0FF51140D0F0EFF
:106FB800F324D96E010EF420DA6EDECFE4F0DDCFD3
:106FC800E5F0E451F06FF16B5350FD0B536E000E7A
:106FD800ED6F000EEC6F000EEB6F000EEA6FAFEF77
:106FE80038F0FF0EE46FFF0EE56FE8C0E6F0E9C089
:106FF800E7F0E451E627E551E723EA51E61907E10E
:10700800EB51E719D8A40BEF38F00DEF38F019EF72
:1070180038F0F051F111D8A414EF38F016EF38F029
:1070280019EF38F053500209536EFF51200D040E2A
:10703800F3248C6F020EF4208D6F340E8E6F0B0EBE
:107048008F6F010E916F000E906FF30E926F000E0E
:10705800936FD0EC1EF00001F26FB30E8A6FF70E3B
:107068008B6FCECF8CF08D6BCDCF8EF08F6BF2C047
:1070780090F0916BF3C092F0F4C093F04EEC6FF087
:107088000001F251D8B44BEF38F04DEF38F04FEF24
:1070980038F0A3EF37F0F3C023F0F4C024F045EC48
:1070A8003DF00001F351EC25EC6FF451ED21ED6F4B
:1070B800FF51140D070EF324D96E010EF420DA6E79
:1070C800000EDE24E46F010EDE20E56F000EDE20E8
:1070D800E66F000EDE20E76FFF51140D070EF32454
:1070E800D96E010EF420DA6EE4C0DEFFE5C0DEFFE3
:1070F800E6C0DEFFE7C0DEFF980E8A6FF90E8B6FE1
:10710800CECF8CF08D6BCDCF8EF08F6BFF51140DE1
:10711800070EF324D96E010EF420DA6EDECF90F05C
:10712800DECF91F0DECF92F0DECF93F0FF51140D59
:10713800070EF324D96E010EF420DA6EDECF94F038
:10714800DECF95F0DECF96F0DECF97F04EEC6FF005
:107158000001EA4BEB2BE851EA5DEB51800AE46F42
:10716800E951800AE459D8A0BCEF38F0BEEF38F0F6
:10717800F5EF37F0F1BFC9EF38F0F15108E1F0054C
:10718800D8A0C9EF38F0CBEF38F055EF39F0FF5100
:10719800200D040EF3248C6F020EF4208D6F340E34
:1071A8008E6F0B0E8F6FF0C090F0F1C091F0F30E60
:1071B800926F000E936FD0EC1EF00001F26F590E23
:1071C8008A6FFA0E8B6FF2C08CF08D6BF3C08EF065
:1071D800F4C08FF04EEC6FF00001F251D8B4F7EF25
:1071E80038F0F9EF38F0FBEF38F0A3EF37F05350F1
:1071F8000209536EF0C023F0F1C024F045EC3DF0D5
:107208000001F351EC25EC6FF451ED21ED6FFF51C6
:10721800140D070EF324D96E010EF420DA6E000E59
:10722800DE24E46F010EDE20E56F000EDE20E66F3F
:10723800000EDE20E76FFF51140D070EF324D96E00
:10724800010EF420DA6EE4C0DEFFE5C0DEFFE6C022
:10725800DEFFE7C0DEFF600E8A6FFC0E8B6FFF510A
:10726800140D070EF324D96E010EF420DA6EDECF6A
:107278008CF0DECF8DF0DECF8EF0DECF8FF0FF51B9
:10728800140D070EF324D96E010EF420DA6EDECF4A
:1072980090F0DECF91F0DECF92F0DECF93F04EEC9F
:1072A8006FF05350FD0B536E8D0E00018A6FFA0E6E
:1072B8008B6FCECF8CF08D6BCDCF8EF08F6BECC0FB
:1072C80090F0EDC091F04EEC6FF0000E4D6E839093
:1072D8004DC0E2F00001E36B1200446E0001B151B1
:1072E800D8B479EF39F07BEF39F07DEF39F0C6EC9F
:1072F80057F0000E436E0001B051D8B486EF39F054
:1073080088EF39F03BEF3BF0040E4418D8B48FEF08
:1073180039F091EF39F09AEF39F0140E4418D8A4E7
:1073280098EF39F09AEF39F0A8EF39F0000E010123
:107338008E6F000E756F000E746F000E0001B16F36
:10734800070EB06F65EF3BF03F0E4418D8A4AFEFBF
:1073580039F0B1EF39F0BDEF39F0000EFE6F000ED5
:1073680001018E6F000E0001B16F000EB06F65EF66
:107378003BF05F0E4418D8A4C4EF39F0C6EF39F0DB
:10738800D2EF39F0000E01018F6F000E8E6F000EE4
:107398000001B16F000EB06F65EF3BF03F0E446423
:1073A800D8EF39F0DAEF39F0EDEF39F05F0E4460DD
:1073B800E0EF39F0E2EF39F0EDEF39F0400E441824
:1073C800D8B4E9EF39F0EBEF39F0EDEF39F0C6EF6B
:1073D80039F0400E4418D8A4F4EF39F0F6EF39F03C
:1073E80002EF3AF0010E01018F6F000E8E6F000E52
:1073F8000001B16F000EB06F65EF3BF0200E44182E
:10740800D8A409EF3AF00BEF3AF01EEF3AF0010E6C
:10741800FE6F000E01018E6F870E00018A6FFF0E4E
:107428008B6F4EEC6FF0000E0001B16F000EB06F65
:1074380065EF3BF0650E4418D8A425EF3AF027EF26
:107448003AF03DEF3AF0FE51D8B42DEF3AF02FEF75
:107458003AF03DEF3AF0000E0101756F000E746FBF
:10746800010E8E6F000E0001B16F000EB06F65EF58
:107478003BF06E0E4418D8A444EF3AF046EF3AF0C9
:1074880049EF3AF0020E01018E6F700E4418D8A42D
:1074980050EF3AF052EF3AF061EF3AF001018F51B4
:1074A800D8B459EF3AF05BEF3AF061EF3AF0000EDA
:1074B800756F000E746F030E8E6F700E4418D8A48B
:1074C80068EF3AF06AEF3AF082EF3AF00001FE51C5
:1074D800D8B471EF3AF073EF3AF082EF3AF0838064
:1074E800000E0101756F000E746F040E8E6F000E92
:1074F8000001B16F000EB06F65EF3BF0720E4418DB
:10750800D8A489EF3AF08BEF3AF03BEF3BF000015B
:10751800FE51D8B492EF3AF094EF3AF03BEF3BF0DB
:1075280083801C0E0101756F2A0E746F050E8E6F15
:10753800000E0001B16F000EB06F65EF3BF04450D4
:10754800E5EC0EF0436E61EF3BF083804450DCECD9
:1075580066F0436E000E01018E6F61EF3BF0838091
:107568005C0E00018A6FF90E8B6FCECF8CF08D6B9D
:10757800CDCF8EF08F6B4DC090F0916B4EEC6FF0CD
:10758800340E0C6E0B0E0D6E000E0F6E000E0E6E8E
:10759800010E116E000E106ED9EC5AF0535002090C
:1075A800536E2BEE34F04DC0DFFF410E00018A6FA1
:1075B800FD0E8B6F000E8D6F010E8C6F4EEC6FF011
:1075C800340E236E0B0E246E000E266E010E256EF1
:1075D8006B0E276EFF0E286E9FEC4CF0000E246E8B
:1075E800010E236E45EC3DF05350FD0B536E080E13
:1075F800436EAEEF3AF08390000E436EFE0E00012C
:107608008A6FF80E8B6FCECF8CF08D6BCDCF8EF04E
:107618008F6B44C090F0916B4EEC6FF061EF3BF0D4
:10762800080E4418D8A41BEF3BF01DEF3BF061EFA8
:107638003BF07D0E00018A6FF80E8B6FCECF8CF079
:107648008D6BCDCF8EF08F6B44C090F0916B4EEC6C
:107658006FF08390000E436E000E4D6E000E010118
:107668008E6F000E756F000E746F61EF3BF00101B5
:107678008E51416E426A4250000AD8B446EF3BF040
:1076880061EF3BF04150000AD8B461EF3BF0010ACA
:10769800D8B4A3EF3AF0030AD8B4A9EF3AF0010A34
:1076A800D8B4B3EF3AF0070AD8B4FFEF3AF0010ABA
:1076B800D8B414EF3BF061EF3BF043C0B0F00001E9
:1076C800B16B120000019351941195119611D8A431
:1076D80070EF3BF072EF3BF0AAEF3BF020EE0AF0C0
:1076E8009151D9269251DA22DECF98F0DECF99F067
:1076F800DECF9AF0DECF9BF0985199119A119B1129
:10770800D8B489EF3BF08BEF3BF0A0EF3BF020EED5
:1077180012F09151D9269251DA22DE50985DDE504E
:107728009959DE509A59DE509B59D8A09EEF3BF0EC
:10773800A0EF3BF00FEF3CF0010E986F000E996F31
:10774800000E9A6F000E9B6F0FEF3CF091C060F037
:1077580092C061F093C062F094C063F095C064F089
:1077680096C065F072EC30F060C0A0F061C0A1F086
:1077780062C0A2F063C0A3F00001A351A211A1113D
:1077880007E1020EA05DD8B0CCEF3BF0CEEF3BF0A6
:10779800D8EF3BF0010E916F000E926F000E936FC1
:1077A800000E946F44EF3DF0A0290AE1A12908E1F9
:1077B800A22906E1A329D8A4E4EF3BF0E6EF3BF0C9
:1077C800F0EF3BF0A0C091F0A1C092F0A2C093F0FE
:1077D800A3C094F044EF3DF020EE12F09151D92669
:1077E8009251DA22DE50A05DDE50A159DE50A25936
:1077F800DE50A359D8B003EF3CF005EF3CF007EF9B
:107808003CF0E6EF3BF093C098F094C099F095C037
:107818009AF096C09BF098C09CF099C09DF09AC0D1
:107828009EF09BC09FF0010E9C27000E9D239E2377
:107838009F2320EE12F09151D9269251DA22DE5080
:107848009C5DDE509D59DE509E59DE509F59D8A050
:1078580030EF3CF032EF3CF051EF3CF0020E9C6F01
:10786800000E9D6F000E9E6F000E9F6F9B519A1128
:10787800991107E1020E985DD8B045EF3CF047EF4B
:107888003CF051EF3CF0000E916F000E926F000E2D
:10789800936F000E946F44EF3DF091C060F092C07A
:1078A80061F09CC062F09DC063F09EC064F09FC010
:1078B80065F072EC30F060C0A0F061C0A1F062C069
:1078C800A2F063C0A3F00001A051A111A211A3115D
:1078D800D8A471EF3CF073EF3CF075EF3CF0A4EFE7
:1078E8003CF0A0290CE1A1290AE1A22908E1A32979
:1078F800D8B481EF3CF083EF3CF0E6EF3BF0A00515
:10790800A111A211A311D8A48CEF3CF08EEF3CF08A
:1079180090EF3CF0E6EF3BF098519C190DE199513E
:107928009D190AE19A519E1907E19B519F19D8A404
:10793800A0EF3CF0A2EF3CF017EF3CF047EF3CF033
:1079480091C060F092C061F09CC062F09DC063F08D
:107958009EC064F09FC065F0FF0E666FFF0E676FF4
:10796800FF0E686F0F0E696FFDEC2AF00001976F2C
:107978009751D8A4C2EF3CF0C4EF3CF0E7EF3CF0DD
:107988009351941195119611D8B4CDEF3CF0CFEFE7
:107998003CF0E7EF3CF091C060F092C061F093C01A
:1079A80062F094C063F095C064F096C065F09CC026
:1079B80066F09DC067F09EC068F09FC069F0FDEC5E
:1079C8002AF00001976F9751D8A4EDEF3CF0EFEF44
:1079D8003CF026EF3DF020EE0AF09151D926925165
:1079E800DA229CC0DEFF9DC0DEFF9EC0DEFF9FC086
:1079F800DEFF20EE0EF09151D9269251DA22DE28D0
:107A08000CE1DE280AE1DE2808E1DE28D8B40FEF11
:107A18003DF011EF3DF03CEF3DF020EE0EF09151BE
:107A2800D9269251DA22DE06000EDE5ADE5ADE5AD6
:107A380020EE05F09151D9269251DA22000EDB8012
:107A48003CEF3DF09705D8B42CEF3DF02EEF3DF01C
:107A580038EF3DF0010E9C6F000E9D6F000E9E6F7B
:107A6800000E9F6F3CEF3DF09C699D699E699F6980
:107A78009CC091F09DC092F09EC093F09FC094F07E
:107A88001200000E0101A16F000E836F000E826FBD
:107A9800898689808982898489888B688490849280
:107AA80084948498838E83B45CEF3DF05EEF3DF060
:107AB80072EF3DF052A663EF3DF065EF3DF06CEFDD
:107AC8003DF0470E00018A6FF70E8B6F4EEC6FF09A
:107AD800000E246E000E236E12EF3FF00F0113917B
:107AE800350EE82EFED700F0F4EF3EF08EB87FEFAB
:107AF8003DF081EF3DF0AEEF3DF08EBA86EF3DF000
:107B080088EF3DF0AEEF3DF0CA0E00018A6FFE0E21
:107B18008B6F8DB092EF3DF096EF3DF0256A252AE8
:107B280097EF3DF0256A255000018C6F8D6B83B06F
:107B3800A0EF3DF0A4EF3DF0266A262AA5EF3DF020
:107B4800266A265000018E6F8F6BA1C190F0916B51
:107B58004EEC6FF08EB8B3EF3DF0B5EF3DF0BEEFF1
:107B68003DF08B680F01138182C123F083C124F09B
:107B780012EF3FF08EB8C3EF3DF0C5EF3DF0D1EF07
:107B88003DF05D0E00018A6FFE0E8B6F4EEC6FF0BC
:107B9800630E0101A16F05EF3FF0100E0101646F44
:107BA800270E656F000E666F000E676FC7EF3EF019
:107BB8008EA2E1EF3DF0E3EF3DF001EF3EF08EA441
:107BC800E8EF3DF0EAEF3DF001EF3EF06407000E0C
:107BD800655B665B675B64290AE1652908E16629DC
:107BE80006E16729D8A4FBEF3DF0FDEF3DF0F4EF87
:107BF8003EF0620EA16FF4EF3EF0010EA16FF4EFBC
:107C08003EF08EA80AEF3EF00CEF3EF0F4EF3EF0A7
:107C1800020EA16FF4EF3EF0FF0E256EFF0E266EEA
:107C280023C027F024C028F02550272626502822D4
:107C38008251271807E183512818D8A426EF3EF06F
:107C480028EF3EF030EF3EF053A22DEF3EF02FEF3D
:107C58003EF030EF3EF0899A340E8225D96E0B0E35
:107C68008321DA6EDF50FF0A866E824B832B000E6B
:107C78008B6E030EA16F100E646F270E656F000EDA
:107C8800666F000E676FF4EF3EF08EB24EEF3EF077
:107C980050EF3EF063EF3EF06407000E655B665BF5
:107CA800675B64290AE1652908E1662906E1672915
:107CB800D8A461EF3EF063EF3EF065EF3EF0040EAE
:107CC800A16F8EA26AEF3EF06CEF3EF0F4EF3EF04B
:107CD800040EA16FF4EF3EF08990050EA16F100E0F
:107CE800646F270E656F000E666F000E676FF4EF06
:107CF8003EF089848EB483EF3EF085EF3EF098EF36
:107D08003EF06407000E655B665B675B64290AE109
:107D1800652908E1662906E16729D8A496EF3EF0AF
:107D280098EF3EF09AEF3EF0060EA16F8EA49FEFFB
:107D38003EF0A1EF3EF0F4EF3EF0060EA16FF4EF37
:107D48003EF0898A89808B682350825D8351800A3E
:107D5800256E2450800A2558D8B0B5EF3EF0B7EF0D
:107D68003EF0B9EF3EF001EF3EF0630E0101A16F66
:107D7800F4EF3EF09F0E00018A6FFF0E8B6F4EEC02
:107D88006FF0B9EF3EF0A151256E266A2650000A21
:107D9800D8B4D1EF3EF0F4EF3EF02550000AD8B445
:107DA800DCEF3DF0010AD8B405EF3EF0030AD8B481
:107DB80010EF3EF0010AD8B449EF3EF0070AD8B4F4
:107DC80070EF3EF0010AD8B47DEF3EF0030AD8B454
:107DD800A5EF3EF0640AD8B4BEEF3EF0F4EF3EF0F3
:107DE800630E0101A119D8B4FCEF3EF0FEEF3EF09E
:107DF80005EF3FF08EBC03EF3FF005EF3FF07AEF61
:107E08003DF08980898289848988898A8B68839EE4
:107E18000F01138182C123F083C124F0120044C0F2
:107E280025F045C026F015EC5AF0466E4650D8A409
:107E380020EF3FF022EF3FF0D2EF40F044C0D9FFEF
:107E480045C0DAFF030EDE18D8A42DEF3FF02FEF60
:107E58003FF0B9EF40F020EE05F04450D9264550E8
:107E6800DA22DE04D8A43BEF3FF03DEF3FF0B9EF54
:107E780040F02E0E44240C6E000E45200D6E000EB0
:107E88000F6E000E0E6E020E116E000E106E92EC4A
:107E98006DF022EE2CF04450D9264550DA22550ECA
:107EA800DF6E22EE2DF04450D9264550DA22AA0E74
:107EB800DF6E20EE2EF04450D9264550DA22520EBD
:107EC800DF6E20EE2FF04450D9264550DA22520EAC
:107ED800DF6E20EE30F04450D9264550DA22610E8C
:107EE800DF6E20EE31F04450D9264550DA22410E9B
:107EF800DF6E22EE12F04450D9264550DA22720E77
:107F0800DF6E22EE13F04450D9264550DA22720E65
:107F1800DF6E22EE14F04450D9264550DA22410E85
:107F2800DF6E22EE15F04450D9264550DA22610E54
:107F3800DF6E20EE0EF04450D9264550DA2212EEBC
:107F480016F04450E1264550E222DFCFE7FF22EE4B
:107F580017F04450D9264550DA2210EE0EF044505E
:107F6800E1264550E222E6CF60F0E5CF61F061C03E
:107F780060F00001616B6051DF6E22EE18F0445032
:107F8800D9264550DA2210EE0EF04450E12645502D
:107F9800E222E6CF60F0E6CF61F0E6CF62F0E6CF0E
:107FA80063F0110EDDEF3FF0D89063336233613335
:107FB8006033E82ED8EF3FF06051DF6E22EE19F003
:107FC8004450D9264550DA2210EE0EF04450E126EE
:107FD8004550E222E6CF60F0E6CF61F0E6CF62F0EE
:107FE800E6CF63F0190EFEEF3FF0D89063336233AB
:107FF80061336033E82EF9EF3FF06051DF6E20EE19
:108008000AF04450D9264550DA2212EE1AF04450AC
:10801800E1264550E222DFCFE7FF22EE1BF0445075
:10802800D9264550DA2210EE0AF04450E126455090
:10803800E222E6CF60F0E5CF61F061C060F0616BED
:108048006051DF6E22EE1CF04450D9264550DA22EA
:1080580010EE0AF04450E1264550E222E6CF60F0E7
:10806800E6CF61F0E6CF62F0E6CF63F0110E42EFA3
:1080780040F0D8906333623361336033E82E3DEFCC
:1080880040F06051DF6E22EE1DF04450D926455075
:10809800DA2210EE0AF04450E1264550E222E6CFFB
:1080A80060F0E6CF61F0E6CF62F0E6CF63F0190E3C
:1080B80063EF40F0D8906333623361336033E82E66
:1080C8005EEF40F06051DF6E20EE1AF04450D92682
:1080D8004550DA22DECF60F0DECF61F0DECF62F00D
:1080E800DECF63F0010E6025646F000E6121656FBD
:1080F800000E6221666F000E6321676F20EE2AF082
:108108004450D9264550DA2264C0DEFF65C0DEFF40
:1081180066C0DEFF67C0DEFF2E0E44241B6E000E15
:1081280045201C6E20EE2AF04450D9264550DA220C
:10813800DECF1DF0DECF1EF0DECF1FF0DECF20F049
:10814800000E226E010E216E20EE01F04450D92659
:108158004550DA22DF50F2EC56F020EE05F044509C
:10816800D9264550DA22000EDF6E000E1B6E000E77
:108178001C6E000E1D6E20EE01F04450D9264550AD
:10818800DA22DF5021EC22F00009D8B4CEEF40F01B
:10819800D0EF40F0D2EF40F0010E466E465012008C
:1081A80020EE04F04550D9264650DA2247C0DEFFBB
:1081B80048C0DDFF20EE06F04550D9264650DA22A9
:1081C800DECF99F0DECF9AF0DECF9BF0DECF9CF0C9
:1081D800000199059A119B119C11D8B4F6EF40F053
:1081E800F8EF40F011EF41F045C0D9FF46C0DAFF83
:1081F80010EE12F0DE50E126DD50E222E650995DE5
:10820800E6509A59E6509B59E6509C59D8A00FEF72
:1082180041F011EF41F014EF41F0020E77EF42F018
:1082280099519A119B119C11D8A41DEF41F01FEF91
:1082380041F046EF41F045C0D9FF46C0DAFFDECF36
:108248008CF0DDCF8DF08CC0D9FF8DC0DAFF030E26
:10825800DE18D8A432EF41F034EF41F046EF41F098
:1082680045C0D9FF46C0DAFF10EE22F0DE50E12605
:10827800DD50E222E6CF99F0E6CF9AF0E6CF9BF008
:10828800E6CF9CF099519A119B119C11D8A44FEFFD
:1082980041F051EF41F07CEF41F045C0D9FF46C0B5
:1082A800DAFF10EE08F0DE50E126DD50E222E6505B
:1082B800475CE6504858D8A064EF41F066EF41F0BB
:1082C80068EF41F011EF41F045C0D9FF46C0DAFF31
:1082D80010EE22F0DE50E126DD50E222E6CF95F0E6
:1082E800E6CF96F0E6CF97F0E6CF98F00DEF42F0A4
:1082F80045C0D9FF46C0DAFF10EE02F0DE50E12695
:10830800DD50E222E7508C6F8C51100DF3CF93F0C3
:10831800F4CF94F0E8EF41F045C0D9FF46C0DAFF4A
:10832800DECF60F0DDCF61F099C062F09AC063F0F3
:108338009BC064F09CC065F072EC30F060C099F0AE
:1083480061C09AF062C09BF063C09CF0000199295B
:108358000AE19A2908E19B2906E19C29D8A4B7EFEC
:1083680041F0B9EF41F0BCEF41F0010E77EF42F078
:108378009C519B119A1109E1020E995DD8A0C7EF93
:1083880041F0C9EF41F011EF41F045C0D9FF46C0B7
:10839800DAFF10EE12F0DE50E126DD50E222E65060
:1083A800995DE6509A59E6509B59E6509C59D8A0D9
:1083B800E0EF41F0E2EF41F0E4EF41F011EF41F07E
:1083C8009351475E9451485A9351475C9451485889
:1083D800D8B0F1EF41F0F3EF41F090EF41F045C034
:1083E800D9FF46C0DAFFDECF18F0DDCF19F099C00B
:1083F8001AF09AC01BF09BC01CF09CC01DF04CECFE
:1084080064F018C095F019C096F01AC097F01BC018
:1084180098F020EE0AF04550D9264650DA2299C045
:10842800DEFF9AC0DEFF9BC0DEFF9CC0DEFF0001BE
:108438009551961197119811D8A425EF42F027EF7E
:1084480042F029EF42F011EF41F047C08CF048C0EC
:108458008DF0040E8E6FD8908D338C338E2F2FEFC6
:1084680042F08C5195258F6F8D519621906F000E9B
:108478009721916F000E9821926F20EE0EF04550D3
:10848800D9264650DA228FC0DEFF90C0DEFF91C0A9
:10849800DEFF92C0DEFF0F0E47148C6F000E4814EB
:1084A8008D6F050ED8908C378D37E82E56EF42F039
:1084B80045C0D9FF46C0DAFFDECF8EF0DDCF8FF0A2
:1084C8008C518E278D518F232E0E8E27000E8F23D1
:1084D80020EE12F04550D9264650DA228EC0DEFF33
:1084E8008FC0DDFF000E1200000E0101DB6F0A0EC7
:1084F800DA6F000ED96F050ED86F01EF44F0000E49
:10850800DB6F140EDA6FF3EF43F09C0E0D6EFC0E6A
:108518000E6E80EC6AF08FB294EF42F096EF42F064
:108528009BEF42F0000E0101DB6F1E0EDA6F290E81
:108538000101D76F960ED66F7F0EE82EFED7D62F85
:10854800FCD7D72FFAD7F3EF43F0EF0E0D6EFE0EE0
:108558000E6E80EC6AF0060E0001DD6F090EDE6F0C
:10856800870EDF6FFC0EE06F000EE16FFAEC60F033
:108578004F6E4F502CEC69F04F50D8A4C6EF42F024
:10858800C8EF42F09BEF42F0000E0101DB6F230EB3
:10859800DA6F9BEF42F03F0E0D6EFE0E0E6E80EC12
:1085A8006AF0040E0001DD6F020EDE6F120EDF6F3F
:1085B800FF0EE06F010EE16F12EC28F04F6E4F5086
:1085C8002CEC69F04F50D8A4ECEF42F0EEEF42F0FB
:1085D800F8EF42F0D7EC2DF0040E0001736F020E95
:1085E800746F3BEC6BF04F6E4F502CEC69F0000E43
:1085F8000101DB6F280EDA6F9751D8A406EF43F01C
:1086080008EF43F017EF43F0000E9D6F340E0001A2
:10861800826F0D0E836FB00E846FFE0E856F65EC52
:108628006BF024EF43F07A0E00018A6FF90E8B6F1E
:1086380097C18CF08D6B9DC18EF08F6B4EEC6FF0F7
:108648004E0E00018A6FFE0E8B6F01019D510F0DBA
:10865800340EF32400018C6F0D0EF4208D6F4EEC58
:108668006FF09BEF42F0E10E00018A6FFB0E8B6FFB
:1086780001019D510F0D340EF32400018C6F0D0E76
:10868800F4208D6F4EEC6FF0040E0001DD6F020ECA
:10869800DE6F01019D510F0D340EF3240001DF6FD1
:1086A8000D0EF420E06F030EE16F12EC28F04F6E10
:1086B8004F50D8A462EF43F064EF43F069EF43F002
:1086C800000E0101DB6F3C0EDA6F040E4F18D8A4C0
:1086D80070EF43F072EF43F09BEF42F0000E0101A0
:1086E800DB6F320EDA6F9BEF42F00D0E00018A6FDE
:1086F800FD0E8B6F01019D510F0D340EF324000107
:108708008C6F0D0EF4208D6F4EEC6FF0040E00018F
:10871800DD6F020EDE6F01019D510F0D340EF32443
:108728000001DF6F0D0EF420E06F070EE16F12EC11
:1087380028F04F6E4F50D8A4A4EF43F0A6EF43F0B3
:108748009BEF42F0000E0101DB6F3C0EDA6F9BEFEE
:1087580042F0C40E00018A6FFC0E8B6F01019D511F
:108768000F0D340EF32400018C6F0D0EF4208D6F65
:108778004EEC6FF0000E0001FD6F010EFC6F13EF61
:1087880044F0DAC1D6F1DBC1D7F1D751000AD8B429
:10879800D0EF43F0F3EF43F0D6510A0AD8B483EF91
:1087A80042F01E0AD8B489EF42F00A0AD8B4A9EFF9
:1087B80042F03D0AD8B4CFEF42F00B0AD8B437EFF5
:1087C80043F0050AD8B4F3EF43F01F0AD8B479EFA1
:1087D80043F00E0AD8B4ADEF43F0F3EF43F0140EB4
:1087E8000101DA19DB11D8B4FCEF43F0FEEF43F0D6
:1087F80001EF44F0D807D8A0D907D9BF0EEF44F04D
:10880800D95106E1D805D8B00CEF44F00EEF44F08A
:10881800C5EF43F0000E0001FD6F000EFC6F120063
:108828008380000E4D6ED60E00018A6FF70E8B6F97
:10883800CECF8CF08D6BCDCF8EF08F6BFF51140D9A
:10884800070EF324D96E010EF420DA6EDECF90F015
:10885800DECF91F0DECF92F0DECF93F0FF51140D12
:10886800070EF324D96E010EF420DA6EDECF94F0F1
:10887800DECF95F0DECF96F0DECF97F04EEC6FF0BE
:1088880062EC51F0CBC0ADF1CCC0AEF10101AD51FD
:10889800AE11D8B452EF44F054EF44F05AEF44F01C
:1088A800ADC1EDF0AEC1EEF09CEF45F0000EAF6F3C
:1088B800000EB06F000EB16F000EB26F000EAB6FFE
:1088C800010EAA6F000EB56F6FEF45F0000EB46F82
:1088D800000EB36FA1EF44F072EC6FF00C500D1066
:1088E800D8B479EF44F07BEF44F08EEF44F0B50E46
:1088F8000C6E010E0D6E2CEC66F00101A96F000ED6
:108908005024D96EDA6A040EDA22A9C1DFFF502A90
:10891800B34BB42B0101B5AB94EF44F096EF44F0A0
:1089280098EF44F0ACEF44F08EBC9DEF44F09FEF1D
:1089380044F0A1EF44F0ACEF44F0B4BFAAEF44F028
:10894800B405D8A0AAEF44F0ACEF44F070EF44F0BF
:10895800B3C1EFF0B4C1F0F0000E0001F0BFFF0E9C
:10896800F16FF26F0101AF510001EF250101AF6F07
:10897800B0510001F0210101B06FB1510001F121A6
:108988000101B16FB2510001F2210101B26F000182
:10899800FF51140D0F0EF324D96E010EF420DA6E78
:1089A800DE500101AF5DDE50B059DE50B159DE50E6
:1089B800B259D8A0E2EF44F0E4EF44F0E8EF44F015
:1089C800000EAB6F000EAA6FB5ABEDEF44F0EFEF02
:1089D80044F0F3EF44F0000EAB6F000EAA6F8EBCAC
:1089E800F8EF44F0FAEF44F0FEEF44F0000EAB6FFE
:1089F800000EAA6F5050D8B404EF45F006EF45F0CA
:108A080014EF45F00D0E00018A6FFB0E8B6FADC1A0
:108A18008CF0AEC18DF050C08EF08F6B4EEC6FF0C5
:108A28000101B4BF20EF45F0B405D8B01EEF45F002
:108A380020EF45F03CEF45F0000E50240C6E0D6A17
:108A4800040E0D22FF0E5024D96EDA6A030EDA22C4
:108A5800DF500001EF6FEF510E6E0F6A50500008A3
:108A6800106E000ED8A0E82A0108116ED9EC5AF051
:108A780085EC66F00001E2510101AC6FAC51D8B44D
:108A880048EF45F04AEF45F06FEF45F0550E00010D
:108A98008A6FFB0E8B6FACC18CF08D6B4EEC6FF058
:108AA800010E4D6E0001FF51140D130EF324D96E03
:108AB800010EF420DA6EFF51140D130EF324E16E4B
:108AC800010EF420E26EE7500409DF6E4DC0EDF0B0
:108AD800EE6B9CEF45F0AA51AB11D8A476EF45F0A8
:108AE80078EF45F06AEF44F0210E00018A6FF70E27
:108AF8008B6FCECF8CF08D6BCDCF8EF08F6BAFC1DF
:108B080090F0B0C191F0B1C192F0B2C193F04EECC7
:108B18006FF08FA492EF45F094EF45F096EF45F093
:108B2800010E4D6E8390000E0001EE6F000EED6F8A
:108B38001200340E0101B56F0B0EB66FEBC012F0C8
:108B4800ECC013F0DFEC6BF012500101A96FCB0EF3
:108B58000001A46F000EA56F000EA66F000EA76F90
:108B6800000EA86F000EA96FCDEC17F00101B26FCF
:108B7800B251D8B4C2EF45F0C4EF45F0D6EF45F096
:108B8800F40E00018A6FFA0E8B6F4EEC6FF0000E38
:108B98000001CB6F000ECC6F000ECD6F000ECE6FB4
:108BA80019EF47F0CB0E00018C6F000E8D6FB5C129
:108BB8008EF0B6C18FF0010E916F000E906FB00E5F
:108BC800926F010E936FD0EC1EF00101B26FB2519B
:108BD800D8B4F1EF45F0F3EF45F0FCEF45F0B30EF4
:108BE80000018A6FFB0E8B6F4EEC6FF0CBEF45F0F8
:108BF800B5C1D9FFB6C1DAFF800EDE18D8B407EFC9
:108C080046F009EF46F012EF46F0300E00018A6F89
:108C1800FD0E8B6F4EEC6FF0CBEF45F020EE0AF0B7
:108C2800B551D926B651DA22DF500001ED6FED516A
:108C3800EF6FEE6B010120EE0BF0B551D926B6515E
:108C4800DA22DF500001F06FF051EE250101AE6F1E
:108C5800000E0001EF210101AF6F9C0E00018A6F29
:108C6800FB0E8B6FAEC18CF0AFC18DF04EEC6FF088
:108C7800CB0E0001A46F000EA56F0101AE510001DB
:108C8800EE6FED6BEDC0A6F0EEC0A7F0A86BA96B78
:108C9800CDEC17F00101B26FB251D8B456EF46F0DF
:108CA80058EF46F05AEF46F0CBEF45F0CB0E0001F7
:108CB8008C6F000E8D6FB5C18EF0B6C18FF0010EAE
:108CC800916F000E906FB00E926F010E936FD0EC03
:108CD8001EF00101B26FB251D8B475EF46F077EFCC
:108CE80046F079EF46F0CBEF45F0000EB46F000E7A
:108CF800B36FEBC00CF0ECC00DF0B3C1EDF0B4C134
:108D0800EEF0050ED8900001ED37EE37E82E86EF2D
:108D180046F0ED510101B5250E6E0001EE5101013D
:108D2800B6210F6EA9C110F0116AE3EC61F00C5086
:108D38000D10D8A4A2EF46F0A4EF46F006EF47F0D6
:108D4800B3C1EDF0B4C1EEF0050ED8900001ED37D7
:108D5800EE37E82EA9EF46F0B5C1EFF0B6C1F0F056
:108D6800ED51EF27EE51F0230E0EEF25D96E000ED0
:108D7800F021DA6EDF50F16FF151F36FF26BB3C18E
:108D8800F4F0B4C1F5F0050ED890F437F537E82EB5
:108D9800C8EF46F0B5C1F6F0B6C1F7F0F451F627C2
:108DA800F551F7230F0EF625D96E000EF721DA6E6E
:108DB800DF50F86FF96BF251F827F351F923F8C037
:108DC800AAF1F9C0ABF10101000EABBFFF0EAC6F09
:108DD800AD6FF40E00018A6FFD0E8B6FAAC18CF087
:108DE800ABC18DF0ACC18EF0ADC18FF04EEC6FF021
:108DF800AAC1CBF0ABC1CCF0ACC1CDF0ADC1CEF0C7
:108E080019EF47F00101B34BB42BB4BF15EF47F08E
:108E1800B45109E10F0EB35DD8A015EF47F017EF75
:108E280047F07DEF46F0CBEF45F0120001016DBF32
:108E380020EF47F022EF47F023EF47F06E936DBF26
:108E480030EF47F06D5106E16C05D8B02EEF47F0D2
:108E580030EF47F037EF47F0000E0001656F010E65
:108E6800646F3BEF47F06CC164F06DC165F06AC197
:108E780066F06BC167F001016EA945EF47F047EF57
:108E880047F04CEF47F00001FE0E6627FF0E672300
:108E98002AC068F02BC069F02CC06AF02DC06BF0B6
:108EA8002EC06CF02FC06DF030C06EF031C06FF086
:108EB800000E0001716F1F0E706F000E0201A36F8C
:108EC8001BEF48F000017007D8A071070F0E681556
:108ED800726F736B73BF7AEF47F0735109E10A0E33
:108EE800725DD8A07AEF47F07CEF47F084EF47F047
:108EF800570E7225726F000E7321736F8AEF47F059
:108F0800300E7225726F000E7321736FBF0E336EB1
:108F1800FF0E346E3250356E366A33503526345073
:108F2800362236500AE11A0E355CD8A09EEF47F07B
:108F3800A1EF47F0010EA2EF47F0000E606F616BE2
:108F480060516111D8B4ABEF47F0ADEF47F0DDEFFA
:108F580047F09F0E336EFF0E346E200E7211356E81
:108F6800000E7311366E3350352634503622365083
:108F78000AE11A0E355CD8A0C4EF47F0C7EF47F0F6
:108F8800010EC8EF47F0000E626F636B6251631108
:108F9800D8B4D1EF47F0D3EF47F0DDEF47F072C018
:108FA80012F073C013F0E0EC6AF012C072F013C054
:108FB80073F0840E00017025D96E020E7121DA6EED
:108FC80072C0DFFF6407D8A065076607D8A06707E7
:108FD80068C033F069C034F06AC035F06BC036F051
:108FE8006CC037F06DC038F06EC039F06FC03AF021
:108FF800050E08EF48F0D8903A3239323832373215
:109008003632353234323332E82EFFEF47F033C090
:1090180068F034C069F035C06AF036C06BF037C00C
:109028006CF038C06DF039C06EF03AC06FF00001D6
:1090380071BF28EF48F0715109E1020E705DD8A0A8
:1090480028EF48F02AEF48F05BEF48F068516911C3
:109058006A116B116C116D116E116F11D8A437EF75
:1090680048F039EF48F066EF47F065BF46EF48F043
:10907800655106E16405D8B044EF48F046EF48F082
:1090880066EF47F067BF51EF48F0675108E16605A2
:10909800D8A051EF48F053EF48F05BEF48F00101DA
:1090A8006EB359EF48F05BEF48F066EF47F0010107
:1090B8006EA961EF48F063EF48F07AEF48F00001DD
:1090C8007007D8A07107840E7025D96E020E712121
:1090D800DA6E32C0DFFF7007D8A07107840E7025E2
:1090E800D96E020E7121DA6E300EDF6E28C01DF0C7
:1090F80029C01EF0840E000170251F6E020E71211A
:10910800206E66C021F067C022F0E9EC63F01DC054
:1091180028F01EC029F012001C6E1C50D8B497EF1E
:1091280048F099EF48F09CEF48F0010EF5EF49F050
:1091380051A2A1EF48F0A3EF48F0A6EF48F0515034
:10914800F5EF49F0000EBAEC6CF00A0E276EB0EF9E
:1091580048F00CEC6FF027062750D8A4B6EF48F07B
:10916800B8EF48F0ADEF48F0000E246E000E156E13
:10917800000E166E000E176E000E186E000E0FEC25
:109188006BF0E806D8A4CBEF48F0CDEF48F0E6EF57
:1091980049F0AA0E156E010E166E000E176E000E1F
:1091A800186E080E0FEC6BF0E806D8A4DEEF48F056
:1091B800E0EF48F079EF49F0000E276E1D0E2724E6
:1091C800D96EDA6A000EDA220CEC6FF0DF6E272A0D
:1091D800030E2764F2EF48F0F4EF48F0E2EF48F0AE
:1091E8001F04D8A4FAEF48F0FCEF48F0E6EF49F086
:1091F800AA0E2018D8A403EF49F005EF49F0E6EFCE
:1092080049F0030E266EE80E256E2BEF49F0000E8E
:10921800156E000E166E000E176E400E186EA90E13
:109228000FEC6BF00009D8A41CEF49F01EEF49F0D1
:1092380020EF49F034EF49F0150E1B6EC60EE82EEC
:10924800FED71B2EFCD700D02506D8A02606255011
:109258002610D8A432EF49F034EF49F00BEF49F06B
:1092680025502610D8B43BEF49F03DEF49F0E6EF22
:1092780049F0000E156E000E166E000E176E000EE9
:10928800186E3A0E0FEC6BF00009D8A44EEF49F0B7
:1092980050EF49F0E6EF49F0000E276E1D0E272427
:1092A800D96EDA6A000EDA220CEC6FF0DF6E272A2C
:1092B800030E276462EF49F064EF49F052EF49F07A
:1092C8001DBC69EF49F06BEF49F071EF49F0000EF2
:1092D800226E040E216E75EF49F0000E226E0C0E00
:1092E800216E21C024F0E6EF49F0000E156E000E45
:1092F800166E000E176E000E186EA90E0FEC6BF0AE
:109308001B6E020E1B608BEF49F08DEF49F093EF57
:1093180049F0020E246EA90E236E97EF49F0010E54
:10932800246E010E236E030E266EE80E256EBDEF29
:1093380049F0000E156E000E166E000E176E000E28
:10934800186E23500FEC6BF00009D8A4AEEF49F06B
:10935800B0EF49F0B2EF49F0C6EF49F0150E1B6EB9
:10936800C60EE82EFED71B2EFCD700D02506D8A0A7
:10937800260625502610D8A4C4EF49F0C6EF49F0B8
:109388009DEF49F025502610D8B4CDEF49F0CFEF26
:1093980049F0E2EF49F0000E156E020E166E000E4F
:1093A800176E000E186E100E0FEC6BF00009D8B493
:1093B800E0EF49F0E2EF49F0E6EF49F0000E246EE5
:1093C800E6EF49F024C04EF077EC6FF02450D8B4A3
:1093D800F0EF49F0F2EF49F0A3EF48F05190A3EF16
:1093E80048F012008EA6FBEF49F0FDEF49F003EFBD
:1093F8004AF01E0E246EFE0E256E07EF4AF0AF0EE1
:10940800246EFF0E256E8EAA0CEF4AF00EEF4AF07E
:1094180014EF4AF01E0E266EFE0E276E18EF4AF065
:10942800AA0E266EFF0E276E8EA81DEF4AF01FEFBC
:109438004AF025EF4AF01E0E286EFE0E296E29EF1F
:109448004AF0B40E286EFF0E296E8EAE2EEF4AF04B
:1094580030EF4AF036EF4AF01E0E2A6EFE0E2B6EE3
:109468003AEF4AF0B90E2A6EFF0E2B6E8EAC3FEF24
:109478004AF041EF4AF047EF4AF01E0E2C6EFE0EFE
:109488002D6E4BEF4AF0A50E2C6EFF0E2D6E8EA49E
:1094980050EF4AF052EF4AF058EF4AF01E0E2E6E87
:1094A800FE0E2F6E5CEF4AF0C30E2E6EFF0E2F6E6F
:1094B8008EA261EF4AF063EF4AF069EF4AF01E0EA0
:1094C800306EFE0E316E6DEF4AF0C80E306EFF0E34
:1094D800316E8EA072EF4AF074EF4AF07AEF4AF0DC
:1094E8001E0E326EFE0E336E7EEF4AF0BE0E326EE8
:1094F800FF0E336E90AE83EF4AF085EF4AF08BEFA4
:109508004AF01E0E346EFE0E356E8FEF4AF0F60EE0
:10951800346EFF0E356E90AC94EF4AF096EF4AF039
:109528009CEF4AF01E0E366EFE0E376EA0EF4AF024
:10953800F30E366EFF0E376E90AAA5EF4AF0A7EF2E
:109548004AF0ADEF4AF01E0E386EFE0E396EB1EFDE
:109558004AF0F00E386EFF0E396E90A8B6EF4AF05A
:10956800B8EF4AF0BEEF4AF01E0E3A6EFE0E3B6EA2
:10957800C2EF4AF0ED0E3A6EFF0E3B6E90A6C7EFB3
:109588004AF0C9EF4AF0CFEF4AF01E0E3C6EFE0ECD
:109598003D6ED3EF4AF0EA0E3C6EFF0E3D6E90A48E
:1095A800D8EF4AF0DAEF4AF0E0EF4AF01E0E3E6ECE
:1095B800FE0E3F6EE4EF4AF0E70E3E6EFF0E3F6E82
:1095C80090A2E9EF4AF0EBEF4AF0F1EF4AF01E0EF5
:1095D800406EFE0E416EF5EF4AF0E40E406EFF0E4F
:1095E800416E90A0FAEF4AF0FCEF4AF002EF4BF020
:1095F8001E0E426EFE0E436E06EF4BF0E10E426EFB
:10960800FF0E436EE60E00018A6FF50E8B6F9050C9
:10961800FF0A236E23508C6F8D6B8ECF8EF08F6B6D
:1096280042C090F043C091F040C092F041C093F026
:109638003EC094F03FC095F03CC096F03DC097F016
:109648003AC098F03BC099F038C09AF039C09BF006
:1096580036C09CF037C09DF034C09EF035C09FF0F6
:1096680032C0A0F033C0A1F030C0A2F031C0A3F0E6
:109678002EC0A4F02FC0A5F02CC0A6F02DC0A7F0D6
:109688002AC0A8F02BC0A9F028C0AAF029C0ABF0C6
:1096980026C0ACF027C0ADF024C0AEF025C0AFF0B6
:1096A8004EEC6FF01200000120EE04F06051D92654
:1096B8006151DA22000EDF6E20EE2AF06051D926C1
:1096C8006151DA22FF0EDE6EFF0EDE6EFF0EDE6ED9
:1096D800FF0EDD6E60C03AF061C03BF062C03CF046
:1096E80063C03DF064C03EF065C03FF0AFEC64F08D
:1096F8000009D8B482EF4BF084EF4BF087EF4BF0C2
:10970800030E9EEF4CF0000122EE2DF06051D92699
:109718006151DA22DF50666F6651686F676B22EE1F
:109728002CF06051D9266151DA22DF50696F6951F6
:109738006713000E6813550E671909E1AA0E681918
:10974800D8B4A9EF4BF0ABEF4BF0AEEF4BF0020EF5
:109758009EEF4CF020EE65F06051D9266151DA2277
:10976800DF50666F6651686F676B20EE66F0605178
:10977800D9266151DA22DF50696F69C06AF06B6BD4
:109788006C6B6D6B6BC06DF06AC06CF06B6B6A6B69
:1097980020EE67F06051D9266151DA22DF506E6FF2
:1097A8006EC06FF0706B716B726B6FC072F0716B23
:1097B800706B6F6B6A516F11736F6B517011746FAF
:1097C8006C517111756F6D517211766F675173110C
:1097D800776F68517411786F000E7511796F000EEC
:1097E80076117A6F20EE64F06051D9266151DA2241
:1097F800DF507B6F7B5177117C6F78517D6F79518A
:109808007E6F7A517F6FFF0E7C15806FFF0E7D157E
:10981800816FFF0E7E15826F000E7F15836F460ED7
:1098280080190BE1410E811908E1540E8219831148
:10983800D8A421EF4CF023EF4CF026EF4CF0000EAB
:109848009EEF4CF020EE81F06051D9266151DA226A
:10985800DF50666F6651686F676B20EE82F060516B
:10986800D9266151DA22DF50696F69C06AF06B6BE3
:109878006C6B6D6B6BC06DF06AC06CF06B6B6A6B78
:1098880020EE83F06051D9266151DA22DF506E6FE5
:109898006EC06FF0706B716B726B6FC072F0716B32
:1098A800706B6F6B6A516F11736F6B517011746FBE
:1098B8006C517111756F6D517211766F675173111B
:1098C800776F68517411786F000E7511796F000EFB
:1098D80076117A6F20EE80F06051D9266151DA2234
:1098E800DF507B6F7B5177117C6F78517D6F795199
:1098F8007E6F7A517F6FFF0E7C15806FFF0E7D158E
:10990800816FFF0E7E15826F000E7F15836F460EE6
:1099180080190BE1410E811908E1540E8219831157
:10992800D8A499EF4CF09BEF4CF09DEF4CF023EF4F
:109938004CF0010E1200BD0E00018A6FFE0E8B6FF7
:1099480027C08CF028C08DF023C08EF024C08FF083
:1099580025C090F026C091F04EEC6FF0000E306EEE
:10996800000E2F6EAEEF4DF0850E00018A6FFC0ED3
:109978008B6F4EEC6FF0000E326E000E316EEEEF14
:109988004CF02FC029F030C02AF0293A2A3AF00EBC
:109998002A1629500F0B2A12F00E291623C02BF075
:1099A80024C02CF029502B262A502C2231502B244D
:1099B800D96E32502C20DA6EDF502E6E990E0001CF
:1099C8008A6FFF0E8B6F2EC08CF08D6B4EEC6FF094
:1099D800314A322A32BEFCEF4CF0325007E1100E09
:1099E800315CD8B0FAEF4CF0FCEF4CF01CEF4DF0C6
:1099F8002FC029F030C02AF0293A2A3AF00E2A1648
:109A080029500F0B2A12F00E2916315029263250F0
:109A18002A222950255C2650800A2B6E2A50800A5B
:109A28002B58D8B01AEF4DF01CEF4DF0C5EF4CF0A5
:109A3800DD0E00018A6FFF0E8B6F4EEC6FF0000E8B
:109A4800326E000E316E7EEF4DF02FC029F030C01F
:109A58002AF0293A2A3AF00E2A1629500F0B2A1210
:109A6800F00E291623C02BF024C02CF029502B26E9
:109A78002A502C2231502B24D96E32502C20DA6EE9
:109A8800200EDF644AEF4DF04CEF4DF075EF4DF0CE
:109A9800F90E00018A6FFF0E8B6F2FC029F030C0BE
:109AA8002AF0293A2A3AF00E2A1629500F0B2A12C0
:109AB800F00E291623C02BF024C02CF029502B2699
:109AC8002A502C2231502B24D96E32502C20DA6E99
:109AD800DF502D6E2D508C6F8D6B4EEC6FF07CEF40
:109AE8004DF0FC0E00018A6FFF0E8B6F4EEC6FF08D
:109AF800314A322A32BE8CEF4DF0325007E1100E57
:109B0800315CD8B08AEF4DF08CEF4DF0ACEF4DF0F2
:109B18002FC029F030C02AF0293A2A3AF00E2A1626
:109B280029500F0B2A12F00E2916315029263250CF
:109B38002A222950255C2650800A2B6E2A50800A3A
:109B48002B58D8B0AAEF4DF0ACEF4DF029EF4DF0FF
:109B58002F4A302A30BEBCEF4DF0305007E1500E8E
:109B68002F5CD8B0BAEF4DF0BCEF4DF0D8EF4DF008
:109B78002FC029F030C02AF0293A2A3AF00E2A16C6
:109B880029500F0B2A12F00E29162550295C2A504D
:109B9800800A2B6E2650800A2B58D8A0D6EF4DF09D
:109BA800D8EF4DF0B8EF4CF0850E00018A6FFC0E2F
:109BB8008B6F4EEC6FF01200000E0001CC6F010E9F
:109BC800CB6FFB0E8A6FF60E8B6F4AC08CF08D6BD5
:109BD8004BC08EF08F6B4CC090F0916B4BC0B4F0C3
:109BE800B56BB66BB76B040ED890B437B537B637CC
:109BF800B737E82EF8EF4DF04AC0B8F0B96BBA6B3A
:109C0800BB6B040ED890B837B937BA37BB37E82ED4
:109C180006EF4EF0D890B835BC6FB935BD6FBA3580
:109C2800BE6FBB35BF6FB451BC25C06FB551BD21E8
:109C3800C16FB651BE21C26FB751BF21C36F4C501F
:109C4800C025926F000EC121936F000EC221946F40
:109C5800000EC321956F4EEC6FF0000E0001C76F28
:109C6800000EC86F000EC96F000ECA6F01EF4FF0EB
:109C7800040E8C6F020E8D6F340E8E6F0B0E8F6F6D
:109C8800010E916F000E906FCF0E926F000E936FC2
:109C9800D0EC1EF00001C46F4C0E8A6FFC0E8B6F67
:109CA800C4C08CF08D6BCFC08EF0D0C08FF04EEC5E
:109CB8006FF05350FD0B536ECFC023F0D0C024F08B
:109CC80045EC3DF023C0CDF024C0CEF00001CD51CD
:109CD800C725C76FCE51C821C86F000EC921C96FEB
:109CE800000ECA21CA6F8EBC7CEF4EF07EEF4EF09C
:109CF80080EF4EF00BEF4FF0CF51CD1909E1D05165
:109D0800CE19D8B48AEF4EF08CEF4EF098EF4EF0A3
:109D1800D70E8A6FFE0E8B6FCDC08CF0CEC08DF043
:109D28004EEC6FF00BEF4FF068EC6EF072EC6FF0EA
:109D38000C500D10D8B4A3EF4EF0A5EF4EF0B7EFCE
:109D48004EF0840E00018A6FFD0E8B6F72EC6FF07F
:109D58000CC08CF00DC08DF04EEC6FF0010E0101BF
:109D68008B6F0BEF4FF0000E0001C66F050EC56F2D
:109D7800E3EF4EF0D00E0001B46FC90EE82EFED707
:109D8800B42FFCD700D072EC6FF00C500D10D8B483
:109D9800D0EF4EF0D2EF4EF0E3EF4EF0000E0001A0
:109DA800CC6F000ECB6F740E8A6FFD0E8B6FC5C023
:109DB8008CF0C6C08DF04EEC6FF0F1EF4EF0000164
:109DC800C507D8A0C607C52906E1C629D8A4EFEF5C
:109DD8004EF0F1EF4EF0BEEF4EF072EC6FF00C501B
:109DE8000D10D8B4FAEF4EF0FCEF4EF001EF4FF043
:109DF800000E0001CC6F000ECB6F0001CB51CC11CF
:109E0800D8A409EF4FF00BEF4FF03CEF4EF0D70E10
:109E180000018A6FFC0E8B6FC7C08CF0C8C08DF034
:109E2800C9C08EF0CAC08FF04EEC6FF0000E010171
:109E38008B6F83901200F80E00018A6FF70E8B6FFC
:109E4800CECF8CF08D6BCDCF8EF08F6BFFC090F0A6
:109E5800916B4EEC6FF053500209536E340E0C6E3A
:109E68000B0E0D6E000E0F6E000E0E6E010E116EB3
:109E7800000E106ED9EC5AF02BEE34F0FFC0DFFF65
:109E8800FF0EE8CF35FB0001FF51140D130EF3242C
:109E9800D96E010EF420DA6E0101DFA456EF4FF0FF
:109EA80058EF4FF05BEF4FF0010EE8CF38FB0001A1
:109EB800FF51140D130EF324D96E010EF420DA6E3F
:109EC8000101DFA06AEF4FF06CEF4FF06FEF4FF03A
:109ED800020EE8CF3AFB0001FF51140D130EF324D4
:109EE800D96E010EF420DA6E0101DFA27EEF4FF089
:109EF80080EF4FF083EF4FF0020EE8CF3AFB8FA4CC
:109F080088EF4FF08AEF4FF08DEF4FF0080EE8CF53
:109F18003AFB000E2C6E000E2B6EBE0E00018A6FEF
:109F2800F80E8B6FCECF8CF08D6BCDCF8EF08F6B04
:109F38002BC090F02CC091F0360E2B24D96E0B0E4E
:109F48002C20DA6EDF50296E2950926F936B4EECFD
:109F58006FF0500E2B24D96E010E2C20DA6EDF50D4
:109F6800FF0A2A6E360E2B24D96E0B0E2C20DA6EC1
:109F7800360E2B24E16E0B0E2C20E26EE7502A14CD
:109F8800DF6E640E00018A6FFF0E8B6F360E2B2476
:109F9800D96E0B0E2C20DA6EDF50296E29508C6F8B
:109FA8008D6B4EEC6FF02B4A2C2A2CBEE5EF4FF050
:109FB8002C5009E1070E2B5CD8A0E5EF4FF0E7EF36
:109FC8004FF091EF4FF00001FF51140D130EF324E1
:109FD800D96E010EF420DA6EDF504D6EFF51140D6C
:109FE800010EF324D96E010EF420DA6EDF50296ECB
:109FF80029C03FFBFF51140D020EF324D96E010E48
:10A00800F420DA6EDF50296E29C040FBFF51140D91
:10A01800030EF324D96E010EF420DA6EDF50296E98
:10A0280029C041FBFF51140D040EF324D96E010E13
:10A03800F420DA6EDF50296E29C042FBFF51140D5F
:10A04800050EF324D96E010EF420DA6EDF50296E66
:10A0580029C043FBFF51140D060EF324D96E010EDF
:10A06800F420DA6EDF50296E29C044FB000E246EFE
:10A07800140E236E45EC3DF05350FD0B536E839048
:10A08800120047C00DF048C00EF085EC63F00001E7
:10A098006C6F6C51D8A453EF50F055EF50F060EF4F
:10A0A80051F020EE04F04750D9264850DA22DFAAB2
:10A0B80060EF50F062EF50F060EF51F047C0D9FF09
:10A0C80048C0DAFFDECF3AF0DDCF3BF020EE1AF0E1
:10A0D8004750D9264850DA22DECF3CF0DECF3DF09B
:10A0E800DECF3EF0DECF3FF0AFEC64F000016C6FE6
:10A0F8006C51D8A482EF50F084EF50F060EF51F02B
:10A1080020EE1EF04750D9264850DA22DECF71F0F3
:10A11800DDCF72F020EE0BF07151D9267251DA22A0
:10A12800000EDB8A20EE0AF04750D9264850DA2282
:10A1380010EE1CF07151E1267251E222DFCFE7FFE9
:10A1480020EE1DF07151D9267251DA2210EE0AF074
:10A158004750E1264850E222E6CF68F0E5CF69F0A3
:10A1680069C068F0696B6851DF6E20EE1EF07151AE
:10A17800D9267251DA2210EE0AF04750E1264850EB
:10A18800E222E6CF68F0E6CF69F0E6CF6AF0E6CFE4
:10A198006BF0110ED5EF50F0D8906B336A336933FA
:10A1A8006833E82ED0EF50F06851DF6E20EE1FF0D4
:10A1B8007151D9267251DA2210EE0AF04750E12681
:10A1C8004850E222E6CF68F0E6CF69F0E6CF6AF0C1
:10A1D800E6CF6BF0190EF6EF50F0D8906B336A3378
:10A1E80069336833E82EF1EF50F06851DF6E71C0C3
:10A1F8000CF072C00DF020EE0EF04750D9264850F2
:10A20800DA22DECF0EF0DECF0FF0DECF10F0DECF99
:10A2180011F0DBEC6CF0000120EE16F07151D9263C
:10A228007251DA22000EDF6E20EE17F07151D92636
:10A238007251DA22000EDF6E20EE18F07151D92625
:10A248007251DA22210EDF6E20EE19F07151D926F3
:10A258007251DA22460EDF6E20EE12F07151D926C5
:10A268007251DA22000EDF6E20EE13F07151D926FA
:10A278007251DA22000EDF6E20EE04F04750D92624
:10A288004850DA22DF0EDF1647C0D9FF48C0DAFF90
:10A2980010EE04F0DE50E126DD50E222010EE76EFA
:10A2A80047C0D9FF48C0DAFFDECF44F0DDCF45F024
:10A2B80013EC3FF000016C6F6C5112000001FF516C
:10A2C800140D070EF324D96E010EF420DA6EDECFDA
:10A2D800DEF0DECFDFF0DECFE0F0DECFE1F0CE0E55
:10A2E8008A6FF60E8B6FCECF8CF08D6BCDCF8EF044
:10A2F8008F6BDEC090F0DFC091F0E0C092F0E1C05B
:10A3080093F0DEC094F0DFC095F0E0C096F0E1C0B5
:10A3180097F04EEC6FF00001FF51140D070EF32477
:10A32800D96E010EF420DA6EFF51140D0B0EF324D2
:10A33800E16E010EF420E26EDE50E65CDE50E65877
:10A34800DE50E658DE50E658D8B0ADEF51F0AFEF2A
:10A3580051F0CBEF51F0FB0E8A6FFC0E8B6F4EEC79
:10A368006FF0010E4D6E0001FF51140D130EF32412
:10A37800D96E010EF420DA6EFF51140D130EF3247A
:10A38800E16E010EF420E26EE7500409DF6EFF5122
:10A39800140D0F0EF324D96E010EF420DA6EDECF01
:10A3A800CDF0DECFCEF0DECFCFF0DECFD0F0FF5154
:10A3B800140D070EF324D96E010EF420DA6EDECFE9
:10A3C800D1F0DECFD2F0DECFD3F0DECFD4F0CD5156
:10A3D800D125D56FCE51D221D66FCF51D321D76F8A
:10A3E800D051D421D86FFF51140D0B0EF324D96E20
:10A3F800010EF420DA6ED551DE5CD651DE58D75105
:10A40800DE58D851DE58D8B00CEF52F00EEF52F0AB
:10A418002AEF52F0E90E8A6FFC0E8B6F4EEC6FF04C
:10A42800010E4D6E0001FF51140D130EF324D96E69
:10A43800010EF420DA6EFF51140D130EF324E16EB1
:10A44800010EF420E26EE7500409DF6E000E4D6E37
:10A45800FF51200D040EF324A46F020EF420A56F03
:10A46800DEC0A6F0DFC0A7F0E0C0A8F0E1C0A9F008
:10A47800CDEC17F00001DD6FDD51D8B446EF52F096
:10A4880048EF52F06FEF52F03D0E8A6FFB0E8B6F64
:10A49800DEC08CF0DFC08DF0E0C08EF0E1C08FF040
:10A4A800DDC090F0916B4EEC6FF0010E4D6E000127
:10A4B800FF51140D130EF324D96E010EF420DA6E39
:10A4C800FF51140D130EF324E16E010EF420E26E19
:10A4D800E7500409DF6E4DC0CBF0CC6B1200BFC053
:10A4E800F6FFC0C0F7FF000EF86E0E0EF76403D03B
:10A4F8000800F55005D0F6CFE9FFF7CFEAFFEF5097
:10A508002F0AD8B48AEF52F08CEF52F0A5EF52F030
:10A51800BFC0F6FFC0C0F7FF000EF86E0E0EF7645E
:10A5280003D00800F55005D0F6CFE9FFF7CFEAFFD2
:10A53800EF505C0AD8A4A3EF52F0A5EF52F0A8EFB1
:10A5480052F00001BF4BC02B000120EE06F0BD51B8
:10A55800D926BE51DA22DE6ADE6ADE6ADD6ABFC04B
:10A56800F6FFC0C0F7FF000EF86E0E0EF76403D0BA
:10A578000800F55005D0F6CFE9FFF7CFEAFFEF5016
:10A588000001C16F200EC161CCEF52F0CEEF52F046
:10A59800E6EF52F0BDC045F0BEC046F0000E486E72
:10A5A800000E476ED4EC40F00001C56F20EE12F0AB
:10A5B800BD51D926BE51DA22000EDE6E000EDD6EC8
:10A5C8006FEF53F0BDC014F0BEC015F0BF0E166E8D
:10A5D800000E176E4DEC35F00001C56FC551D8B4AB
:10A5E800F8EF52F0FAEF52F0FCEF52F06FEF53F041
:10A5F800BDC0B7F0BEC0B8F0D1EC5EF00001C56FC9
:10A6080020EE14F0BD51D926BE51DA2210EE0BF01F
:10A61800DE50E126DD50E222E750C46FC551D8B4C0
:10A6280018EF53F01AEF53F02EEF53F0040EC5193C
:10A63800D8A421EF53F023EF53F06FEF53F0C4B5D4
:10A6480028EF53F02AEF53F06FEF53F0050EC56F64
:10A658006FEF53F0C4A533EF53F035EF53F037EFF6
:10A6680053F06FEF53F020EE12F0BD51D926BE51D2
:10A67800DA22DECFC2F0DDCFC3F020EE0BF0C251FC
:10A68800D926C351DA22DFB84CEF53F04EEF53F01E
:10A6980050EF53F02AEF53F0BDC0D9FFBEC0DAFF28
:10A6A800DECF0CF0DDCF0DF0C2C00EF0C3C00FF04E
:10A6B800B9EC62F0000120EE06F0BD51D926BE517A
:10A6C800DA220CC0DEFF0DC0DEFF0EC0DEFF0FC0B9
:10A6D800DEFFE6EF52F0C55112004CC0CBF000018E
:10A6E800CC6BCD6BCE6BCDC0CEF0CCC0CDF0CBC09B
:10A6F800CCF0CB6B4BC0CFF0D06BD16BD26BD1C051
:10A70800D2F0D0C0D1F0CFC0D0F0CF6B040ED8902B
:10A71800CF37D037D137D237E82E8BEF53F04AC036
:10A72800D3F0D46BD56BD66B040ED890D337D4370F
:10A73800D537D637E82E99EF53F0D5C0D6F0D4C028
:10A74800D5F0D3C0D4F0D36BD890D335D76FD435E8
:10A75800D86FD535D96FD635DA6FCF51D725DB6F9E
:10A76800D051D821DC6FD151D921DD6FD251DA21F6
:10A77800DE6FCB51DB25E06FCC51DC21E16FCD5191
:10A78800DD21E26FCE51DE21E36F1E0E8A6FF90ED6
:10A798008B6F49C08CF08D6B4AC08EF08F6B4BC0AD
:10A7A80090F0916B4CC092F0936B4BC0CBF0CC6B9C
:10A7B800CD6BCE6B040ED890CB37CC37CD37CE3798
:10A7C800E82EDFEF53F04AC0CFF0D06BD16BD26BDD
:10A7D800040ED890CF37D037D137D237E82EEDEFE7
:10A7E80053F0D890CF35D36FD035D46FD135D56FDE
:10A7F800D235D66FCB51D325D76FCC51D421D86F52
:10A80800CD51D521D96FCE51D621DA6F4C50D725ED
:10A81800946F000ED821956F000ED921966F000E07
:10A82800DA21976F4EEC6FF0850E00018A6FFB0EF0
:10A838008B6FE0C08CF0E1C08DF0E2C08EF0E3C019
:10A848008FF0E0C090F0E1C091F0E2C092F0E3C078
:10A8580093F04EEC6FF0040E0001A46F020EA56F8A
:10A86800E0C0A6F0E1C0A7F0E2C0A8F0E3C0A9F0FC
:10A87800CDEC17F00001DF6FDF51D8B446EF54F08C
:10A8880048EF54F059EF54F03D0E8A6FFB0E8B6F72
:10A89800E0C08CF0E1C08DF0E2C08EF0E3C08FF034
:10A8A800DFC090F0916B4EEC6FF0000E01018B6FE2
:10A8B8008390120076C0D9FF77C0DAFFDECFF6FFAB
:10A8C800DDCFF7FF0800F550250AD8A46EEF54F045
:10A8D80070EF54F02CEF55F076C0D9FF77C0DAFF4F
:10A8E800DE2A000EDD22000E01016B6F000E6A6F7A
:10A8F8006AC16EF16BC16FF16C696D6976C0D9FF81
:10A9080077C0DAFFDECFF6FFDDCFF7FF0800F5509E
:10A91800780AD8B492EF54F094EF54F0A6EF54F0BC
:10A9280076C0D9FF77C0DAFFDECFF6FFDDCFF7FFBD
:10A938000800F550580AD8A4A4EF54F0A6EF54F034
:10A94800F4EF54F076C0D9FF77C0DAFFDECFF6FF18
:10A95800DDCFF7FF0800F5CF47F076C0D9FF77C005
:10A96800DAFFDE2A000EDD2278C0D9FF79C0DAFFCF
:10A97800DFCF3BF0020EDE26DFCF3CF0000EDD22FB
:10A988003BC0D9FF3CC0DAFFDECF3DF0DDCF3EF063
:10A998003DC03FF03EC040F0416A426A436A446AA3
:10A9A800456A466A74C028F075C029F03FC02AF08D
:10A9B80040C02BF041C02CF042C02DF043C02EF017
:10A9C80044C02FF045C030F046C031F047C032F0E7
:10A9D8001AEC47F028C074F029C075F047EF55F01D
:10A9E80076C0D9FF77C0DAFFDECFF6FFDDCFF7FFFD
:10A9F8000800F550250AD8A404EF55F006EF55F0E5
:10AA08001EEF55F076C0D9FF77C0DAFFDE2A000EB8
:10AA1800DD22000E0E6E250E0D6E74C00FF075C08F
:10AA280010F020EC63F0000E0001756F010E746FDA
:10AA380047EF55F076C0D9FF77C0DAFFDE2A000E5F
:10AA4800DD22000E0001756F000E746F47EF55F0A0
:10AA580076C0D9FF77C0DAFFDECFF6FFDDCFF7FF8C
:10AA68000800F5500D6E0E6A74C00FF075C010F036
:10AA780020EC63F076C0D9FF77C0DAFFDE2A000E3B
:10AA8800DD2217EF55F0120000019651951194112F
:10AA980009E1020E935DD8A054EF55F056EF55F03A
:10AAA8006BEF55F020EE12F09151D9269251DA222F
:10AAB800DE50935DDE509459DE509559DE5096591C
:10AAC800D8A069EF55F06BEF55F06FEF55F0020E17
:10AAD800976F1CEF56F0000E976F07EF56F091C076
:10AAE80060F092C061F093C062F094C063F095C0CA
:10AAF80064F096C065F072EC30F060C098F061C008
:10AB080099F062C09AF063C09BF0000198519911C6
:10AB18009A119B11D8A493EF55F095EF55F097EF44
:10AB280055F01CEF56F0980599119A119B11D8A46D
:10AB3800A0EF55F0A2EF55F0A4EF55F06BEF55F0EC
:10AB480098290AE1992908E19A2906E19B29D8A4BC
:10AB5800B0EF55F0B2EF55F0B6EF55F0010E976F24
:10AB68001CEF56F091C060F092C061F093C062F0A3
:10AB780094C063F095C064F096C065F0000E666FEF
:10AB8800000E676F000E686F000E696FFDEC2AF00B
:10AB98000001976F9751D8B4D4EF55F0D6EF55F020
:10ABA800D8EF55F01CEF56F020EE0EF09151D92653
:10ABB8009251DA22DE280CE1DE280AE1DE2808E1DB
:10ABC800DE28D8B4EAEF55F0ECEF55F0FFEF55F07A
:10ABD80020EE0EF09151D9269251DA22DE2A000E8B
:10ABE800DE22DE22DE2220EE05F09151D926925196
:10ABF800DA22000EDB8098C093F099C094F09AC0D6
:10AC080095F09BC096F020EE12F09151D926925102
:10AC1800DA22DE50935DDE509459DE509559DE50AD
:10AC28009659D8A01AEF56F01CEF56F073EF55F06E
:10AC380097511200900E00018A6FF70E8B6F4AC071
:10AC48008CF08D6B4BC08EF08F6B4CC090F0916B7D
:10AC58004BC0E4F0E56BE66BE76B040ED890E43785
:10AC6800E537E637E737E82E32EF56F04AC0E8F026
:10AC7800E96BEA6BEB6B040ED890E837E937EA37F3
:10AC8800EB37E82E40EF56F0D890E835EC6FE93511
:10AC9800ED6FEA35EE6FEB35EF6FE451EC25F06FB1
:10ACA800E551ED21F16FE651EE21F26FE751EF2109
:10ACB800F36F4C50F025926F000EF121936F000E48
:10ACC800F221946F000EF321956F4EEC6FF0000E99
:10ACD8000001F76F000EF66F000EF86FA5EF56F043
:10ACE80072EC6FF00C500D10D8B47DEF56F07FEF7A
:10ACF80056F092EF56F0F80E0C6E000E0D6E2CEC1E
:10AD080066F00001F46F000E5024D96EDA6A040E62
:10AD1800DA22F4C0DFFF502AF64BF72B0001F8AB1C
:10AD280098EF56F09AEF56F09CEF56F0B0EF56F0C9
:10AD38008EBCA1EF56F0A3EF56F0A5EF56F0B0EF9A
:10AD480056F0F7BFAEEF56F0F705D8A0AEEF56F0C5
:10AD5800B0EF56F074EF56F0F6C0F9F0F7C0FAF01D
:10AD68008FB4B9EF56F0BBEF56F0CFEF56F0040EA4
:10AD7800A46F020EA56F000EA66F040EA76F010E3A
:10AD8800A96F000EA86FF90EAA6F000EAB6F73ECD7
:10AD980013F00001F56FF551D8B4D5EF56F0D7EFA1
:10ADA80056F0E0EF56F0940E8A6FFD0E8B6FF5C0EB
:10ADB8008CF08D6B4EEC6FF0DB0E00018A6FFA0E93
:10ADC8008B6FF9C08CF0FAC08DF04EEC6FF094ECFC
:10ADD8005BF0000E01018B6F83901200246E2450EB
:10ADE800D8A4F9EF56F0FBEF56F004EF57F02150D6
:10ADF8002210D8A402EF57F004EF57F007EF57F0EE
:10AE0800040EC5EF57F051A00CEF57F00EEF57F0B6
:10AE180011EF57F0030EC5EF57F051A416EF57F096
:10AE280018EF57F01BEF57F0020EC5EF57F04EB66C
:10AE380020EF57F022EF57F02BEF57F0090ED8907C
:10AE48001D361E361F362036E82E23EF57F0210414
:10AE58002210D8A432EF57F034EF57F05DEF57F0D7
:10AE68001DC015F01EC016F01FC017F020C018F046
:10AE7800180E0FEC6BF00009D8A445EF57F047EF18
:10AE880057F0B8EF57F01BC00EF01CC00FF0FE0EC5
:10AE9800106E5FEC68F00009D8B455EF57F057EF23
:10AEA80057F0B8EF57F0000E226E000E216EB8EF83
:10AEB80057F04EC023F0060E2316D8B466EF57F0AD
:10AEC80068EF57F071EF57F021C015F022C016F067
:10AED800176A186A970E0FEC6BF01DC015F01EC0AC
:10AEE80016F01FC017F020C018F0190E0FEC6BF009
:10AEF8000009D8A482EF57F084EF57F0B8EF57F065
:10AF08001BC00EF01CC00FF0FC0E106E5FEC68F05A
:10AF18000009D8A492EF57F094EF57F096EF57F046
:10AF2800A4EF57F0020E1C262106D8A022062150B5
:10AF38002210D8A4A2EF57F0A4EF57F084EF57F0EF
:10AF4800000E0E6E000E0F6EFD0E106E5FEC68F0B8
:10AF58000009D8A4B2EF57F0B4EF57F0B8EF57F0A4
:10AF6800000E226E010E216E77EC6FF02150221038
:10AF7800D8A4C1EF57F0C4EF57F0010EC5EF57F052
:10AF8800000E1200000E0001FF6F000EFF6F030E8F
:10AF9800FF65D1EF57F0D3EF57F0D5EF57F079EFC2
:10AFA80058F0FF51140D130EF324D96E010EF4203E
:10AFB800DA6E000EDF6EFF51140D000EF324D96E09
:10AFC800010EF420DA6E000EDF6EFF51140D070E2D
:10AFD800F324D96E010EF420DA6EDE6ADE6ADE6AC8
:10AFE800DD6AE3C223F0246A256A266A25C026F0B2
:10AFF80024C025F023C024F0236AE2C227F0286A7F
:10B00800296A2A6A28C02AF027C029F0286A276AEC
:10B01800E1C22BF02C6A2D6A2E6A2BC02EF02D6A05
:10B028002C6A2B6A0201E0512B242F6E000E2C2073
:10B03800306E000E2D20316E000E2E20326E2750FD
:10B048002F24336E28503020346E29503120356E2D
:10B058002A503220366E23503324376E2450342041
:10B06800386E25503520396E265036203A6E00014C
:10B07800FF51140D0B0EF324D96E010EF420DA6E75
:10B0880037C0DEFF38C0DEFF39C0DEFF3AC0DEFF62
:10B098009E0E8A6FF80E8B6FFFC08CF08D6BFF5180
:10B0A800140D0B0EF324D96E010EF420DA6EDECFE8
:10B0B8008EF0DECF8FF0DECF90F0DECF91F0FF5133
:10B0C800140D0B0EF324D96E010EF420DA6EDECFC8
:10B0D80092F0DECF93F0DECF94F0DECF95F04EEC19
:10B0E8006FF00001FF2BCBEF57F0000E01018F6FBF
:10B0F800000E0001FE6F000E0101A46F000E8E6F9E
:10B10800000E756F000E746F020E4D6E8390120064
:10B11800000E216E000E206E000E1A6E000E196EC3
:10B1280098EF58F0134A142A010E1F6E13C0D9FF66
:10B1380014C0DAFF200EDE18D8B4A5EF58F0A7EF38
:10B1480058F0C3EF58F0F70E156EFF0E166E13C0C9
:10B15800D9FF14C0DAFFDF50176E186A155017268A
:10B1680016501822185009E1050E175CD8A0BFEF39
:10B1780058F0C1EF58F0C3EF58F0000E1F6E1FC013
:10B188001BF01C6A1B501C10D8A4CDEF58F0CFEF51
:10B1980058F096EF58F0D9EF58F0000E1A6E010EDD
:10B1A800196E134A142A0EEF59F013C0D9FF14C0B0
:10B1B800DAFFDF50156E166A1650000AD8B4E7EFAA
:10B1C80058F00EEF59F015502B0AD8B4D5EF58F0B7
:10B1D800060AD8B4D1EF58F00EEF59F020C00CF0A1
:10B1E80021C00DF0000E0F6E0A0E0E6E8EEC6EF082
:10B1F80013C0D9FF14C0DAFFDF50156E15500C5E6E
:10B20800000E0D5A300E0C24206E000E0D20216EFB
:10B21800D5EF58F0D00E156EFF0E166E13C0D9FF7D
:10B2280014C0DAFFDF50176E186A1550172616502B
:10B23800182218500AE10A0E175CD8A026EF59F018
:10B2480029EF59F0010E2AEF59F0000E1D6E1E6A03
:10B258001D501E10D8A433EF59F035EF59F0F2EF16
:10B2680058F019501A10D8A43CEF59F03EEF59F095
:10B278004CEF59F020C015F021C016F0151E161E0F
:10B28800154A162A15C013F016C014F050EF59F0DD
:10B2980020C013F021C014F01200146815680CC007
:10B2A800D9FF0DC0DAFFDE50DE10D8B45EEF59F0DA
:10B2B80060EF59F008EF5AF00CC0D9FF0DC0DAFF63
:10B2C800DECF18F0DDCF19F06CEF59F0184A192AC3
:10B2D80018C0F6FF19C0F7FF000EF86E0E0EF764DF
:10B2E80003D00800F55005D0F6CFE9FFF7CFEAFF05
:10B2F800EF500E6E200E0E6484EF59F086EF59F071
:10B308009FEF59F018C0F6FF19C0F7FF000EF86E4E
:10B318000E0EF76403D00800F55005D0F6CFE9FF0C
:10B32800F7CFEAFFEF503A0AD8A49DEF59F09FEF04
:10B3380059F06AEF59F018C0F6FF19C0F7FF000E70
:10B34800F86E0E0EF76403D00800F55005D0F6CF5E
:10B35800E9FFF7CFEAFFEF503A0AD8A4B6EF59F061
:10B36800B8EF59F00EEF5AF00CC0D9FF0DC0DAFF54
:10B37800DECF12F0DDCF13F012C0F6FF13C0F7FFD7
:10B38800000EF86E0E0EF76403D00800F55005D0D5
:10B39800F6CFE9FFF7CFEAFFEF500E6ED00E0E247E
:10B3A800166E176AFF0E1722124A132A175007E162
:10B3B8000A0E165CD8B0E3EF59F0E5EF59F008EF44
:10B3C8005AF01850121807E119501318D8A4EFEFC3
:10B3D80059F0F1EF59F008EF5AF016501710D8A4A9
:10B3E800F8EF59F0FAEF59F008EF5AF016C014F0D8
:10B3F80017C015F0184A192A0CC0D9FF0DC0DAFF7A
:10B4080018C0DEFF19C0DDFF14C00CF015C00DF028
:10B4180014EF5AF0000E156E000E146E08EF5AF075
:10B428001200000E336E20EE04F02550D926265067
:10B43800DA22DF50D8B423EF5AF025EF5AF0D7EFCD
:10B448005AF020EE2AF02550D9262650DA22DECFEF
:10B4580036F0DECF37F0DECF38F0DECF39F02E0E03
:10B4680025241B6E000E26201C6E36C01DF037C02A
:10B478001EF038C01FF039C020F0000E226E010EF9
:10B48800216E20EE01F02550D9262650DA22DF5011
:10B49800F2EC56F00009D8B454EF5AF056EF5AF0CF
:10B4A8005AEF5AF0010E336ED7EF5AF020EE04F03F
:10B4B8002550D9262650DA22000EDF6E20EE16F02F
:10B4C8002550D9262650DA2210EE1EF02550E12606
:10B4D8002650E222E6CF2BF0E6CF2CF0E6CF2DF077
:10B4E800E6CF2EF02B50365C2F6E2C503758306E2E
:10B4F8002D503858316E2E503958326EDE502F5C30
:10B50800DE503058DE503158DE503258D8B08FEF08
:10B518005AF091EF5AF0D7EF5AF020EE03F0255089
:10B52800D9262650DA22DF50276E2750346E356A26
:10B53800355007E1020E345CD8B0A5EF5AF0A7EFFA
:10B548005AF0A9EF5AF0D7EF5AF020EE16F025502E
:10B55800D9262650DA22DE503626DE503722DE5033
:10B568003822DD5039222E0E25241B6E000E26208F
:10B578001C6E36C01DF037C01EF038C01FF039C031
:10B5880020F0000E226E010E216E20EE01F02550F3
:10B59800D9262650DA22DF50F2EC56F03406D8A02D
:10B5A80035069CEF5AF0335012000CC016F00DC04F
:10B5B80017F010501110D8A4E4EF5AF0E6EF5AF043
:10B5C800E8EF5AF093EF5BF016C0D9FF17C0DAFF27
:10B5D8000EC0DFFF10501624126E11501720136E84
:10B5E800FF0E1224D96EFF0E1320DA6E0EC0DFFF95
:10B5F800115007E1030E105CD8B005EF5BF007EFC0
:10B608005BF009EF5BF093EF5BF020EE01F0165072
:10B61800D9261750DA220EC0DFFF20EE02F01650AE
:10B62800D9261750DA220EC0DFFF10501624126EEA
:10B6380011501720136EFE0E1224D96EFF0E132020
:10B64800DA6E0EC0DFFF10501624126E115017204C
:10B65800136EFD0E1224D96EFF0E1320DA6E0EC083
:10B66800DFFF115007E1070E105CD8B03EEF5BF02A
:10B6780040EF5BF042EF5BF093EF5BF020EE03F0FE
:10B688001650D9261750DA220EC0DFFF10501624A4
:10B69800126E11501720136EFC0E1224D96EFF0E75
:10B6A8001320DA6E0EC0DFFF115007E1090E105C9F
:10B6B800D8B061EF5BF063EF5BF065EF5BF093EFA1
:10B6C8005BF016C012F017C013F0121E131E124AB8
:10B6D800132A030E1214146E156A145016261550E8
:10B6E80017221450105E1550115AFC0E1016FF0E3A
:10B6F80011168AEF5BF016C0D9FF17C0DAFF0EC02B
:10B70800DFFF1006D8A01106164A172A105011108C
:10B71800D8A491EF5BF093EF5BF07FEF5BF0120042
:10B728004C2A0F0E4C649BEF5BF09DEF5BF0ABEF88
:10B738005BF0000E4C6E4B2A010E4B64A6EF5BF0DB
:10B74800A8EF5BF0ABEF5BF0000E4B6E4A2A4CC0E3
:10B75800CBF00001CC6BCD6BCE6BCDC0CEF0CCC0A6
:10B76800CDF0CBC0CCF0CB6B4BC0CFF0D06BD16B56
:10B77800D26BD1C0D2F0D0C0D1F0CFC0D0F0CF6B57
:10B78800040ED890CF37D037D137D237E82EC5EF4F
:10B798005BF04AC0D3F0D46BD56BD66B040ED8904F
:10B7A800D337D437D537D637E82ED3EF5BF0D5C0AB
:10B7B800D6F0D4C0D5F0D3C0D4F0D36BD890D3355D
:10B7C800D76FD435D86FD535D96FD635DA6FCF5115
:10B7D800D725DB6FD051D821DC6FD151D921DD6F4E
:10B7E800D251DA21DE6FCB51DB25DF6FCC51DC2162
:10B7F800E06FCD51DD21E16FCE51DE21E26F3F0ECA
:10B808008A6FFA0E8B6F49C08CF08D6B4AC08EF030
:10B818008F6B4BC090F0916B4CC092F0936B4EECD9
:10B828006FF0040E0001A46F020EA56FDFC0A6F032
:10B83800E0C0A7F0E1C0A8F0E2C0A9F0CDEC17F095
:10B848000001E36FE351D8B42CEF5CF02EEF5CF00D
:10B858003FEF5CF03D0E8A6FFB0E8B6FDFC08CF004
:10B86800E0C08DF0E1C08EF0E2C08FF0E3C090F050
:10B87800916B4EEC6FF0000E01018B6F12006C0E95
:10B8880000018A6FF70E8B6F4AC08CF08D6B4BC02E
:10B898008EF08F6B4CC090F0916B4BC0B4F0B56BD1
:10B8A800B66BB76B040ED890B437B537B637B73721
:10B8B800E82E57EF5CF04AC0B8F0B96BBA6BBB6BB7
:10B8C800040ED890B837B937BA37BB37E82E65EFCA
:10B8D8005CF0D890B835BC6FB935BD6FBA35BE6F5E
:10B8E800BB35BF6FB451BC25C06FB551BD21C16F09
:10B8F800B651BE21C26FB751BF21C36F4C50C0258E
:10B90800926F000EC121936F000EC221946F000E3A
:10B91800C321956F4EEC6FF0000E0001C76F000E4B
:10B92800C86F000EC96F000ECA6F040E8C6F020E2E
:10B938008D6F340E8E6F0B0E8F6F010E916F000E90
:10B94800906FCB0E926F000E936FD0EC1EF000013B
:10B95800C66F1A0E8A6FF80E8B6FC6C08CF08D6B8F
:10B96800CBC08EF0CCC08FF04EEC6FF05350FD0B77
:10B97800536E010E01019E6FCBC023F0CCC024F0A2
:10B9880045EC3DF023C0C4F024C0C5F0000E010111
:10B998009E6F0001C451C725C76FC551C821C86F24
:10B9A800000EC921C96F000ECA21CA6FD70E8A6F4F
:10B9B800FC0E8B6FC7C08CF0C8C08DF0C9C08EF06C
:10B9C800CAC08FF04EEC6FF0000E01018B6F8390B0
:10B9D80012008380000E0C6E040E0D6E000E0F6EAA
:10B9E800F60E0E6E010E116E000E106ED9EC5AF0A6
:10B9F8006C0E00018A6FFE0E8B6F4EEC6FF0000E1E
:10BA08000001E96F000EE86F2E0E1DEC6FF08FB489
:10BA180010EF5DF012EF5DF027EF5DF0040E00010E
:10BA2800A46F020EA56F000EA66F040EA76F010E7D
:10BA3800A96F000EA86FE50EAA6F000EAB6F73EC2E
:10BA480013F00001E76F0001E751D8B42EEF5DF065
:10BA580030EF5DF03BEF5DF05D0E8A6FFF0E8B6F90
:10BA6800E7C08CF08D6B4EEC6FF095EF5DF072ECEB
:10BA78006FF00C500D10D8B444EF5DF046EF5DF058
:10BA880080EF5DF0EA0E0C6E000E0D6E2CEC66F089
:10BA98000001E46FEA51100B236E000E246EE4518E
:10BAA8006CEC1BF023C0EBF024C0ECF0040E00019A
:10BAB800EB19EC11D8A463EF5DF065EF5DF067EF6B
:10BAC8005DF075EC6CF0020E0001EB19EC11D8A4D6
:10BAD80070EF5DF072EF5DF074EF5DF0A9EC69F066
:10BAE8000001EB05EC11D8A47CEF5DF07EEF5DF072
:10BAF80080EF5DF071EC53F00001E84BE92BE95160
:10BB080009E1C80EE85DD8A08CEF5DF08EEF5DF01E
:10BB180008EF5DF01D0E8A6FFF0E8B6F4EEC6FF015
:10BB280083901200B7C045F0B8C046F0000E486ECA
:10BB3800000E476ED4EC40F00001C06FC051D8A48D
:10BB4800A8EF5DF0AAEF5DF027EF5EF0000EBF6F83
:10BB5800000EBE6FB7C0D9FFB8C0DAFFDECF3AF02B
:10BB6800DDCF3BF020EE0EF0B751D926B851DA22DE
:10BB7800DECF3CF0DECF3DF0DECF3EF0DECF3FF053
:10BB8800AFEC64F00001C06FC051D8B4CEEF5DF0E7
:10BB9800D0EF5DF0D2EF5DF027EF5EF020EE12F00F
:10BBA800B751D926B851DA22DECFBBF0DDCFBCF0D1
:10BBB800BBC0D9FFBCC0DAFFE50EDE18D8B4E7EF8A
:10BBC8005DF0E9EF5DF0FFEF5DF020EE12F0B751A8
:10BBD800D926B851DA22DECFBBF0DDCFBCF0BBC02E
:10BBE800D9FFBCC0DAFFDF50D8A4FDEF5DF0FFEF4E
:10BBF8005DF00FEF5EF0BE4BBF2BB951BE1907E1E8
:10BC0800BA51BF19D8A40BEF5EF00DEF5EF013EF39
:10BC18005EF027EF5EF0000EBF6F000EBE6FB7C07C
:10BC2800A4F0B8C0A5F0000EA76F010EA66FE8EC4F
:10BC380032F00001C06FC051D8B425EF5EF027EF95
:10BC48005EF0AEEF5DF0040EC019D8A42EEF5EF0E2
:10BC580030EF5EF032EF5EF0070EC06FC051120099
:10BC6800236E2350D8A43BEF5EF03DEF5EF046EF25
:10BC78005EF021502210D8A444EF5EF046EF5EF04B
:10BC880049EF5EF0040ED0EF5EF051A04EEF5EF08B
:10BC980050EF5EF053EF5EF0030ED0EF5EF04EB65D
:10BCA80058EF5EF05AEF5EF063EF5EF0090ED89041
:10BCB8001D361E361F362036E82E5BEF5EF022500A
:10BCC80007E1020E215CD8B06CEF5EF06EEF5EF01B
:10BCD80074EF5EF0000E256E110E246E78EF5EF0A4
:10BCE800000E256E120E246E24C026F01DC015F01D
:10BCF8001EC016F01FC017F020C018F026500FEC19
:10BD08006BF00009D8A48BEF5EF08DEF5EF0C3EF07
:10BD18005EF01BC00CF01CC00DF0020E0F6E000E82
:10BD28000E6E82EC67F00009D8A49DEF5EF09FEFDD
:10BD38005EF0A1EF5EF0AFEF5EF0020E1C2621066A
:10BD4800D8A0220621502210D8A4ADEF5EF0AFEFA4
:10BD58005EF08DEF5EF0120E2618D8A4B6EF5EF0F6
:10BD6800B8EF5EF0C3EF5EF0000E156E000E166EB3
:10BD7800000E176E000E186E0C0E0FEC6BF077ECC1
:10BD88006FF021502210D8A4CCEF5EF0CFEF5EF018
:10BD9800010ED0EF5EF0000E1200B7C045F0B8C03B
:10BDA80046F0000E486E000E476ED4EC40F00001DD
:10BDB800BC6FBC51D8B4E3EF5EF0E5EF5EF0E9EF9D
:10BDC8005EF00001BC516CEF5FF0B7C0D9FFB8C09E
:10BDD800DAFFDECF3AF0DDCF3BF020EE0EF0B751C0
:10BDE800D926B851DA22DECF3CF0DECF3DF0DECFE7
:10BDF8003EF0DECF3FF0AFEC64F00001BC6FBC5109
:10BE0800D8B409EF5FF00BEF5FF00DEF5FF0E5EFEF
:10BE18005EF020EE12F0B751D926B851DA22DECF03
:10BE2800BAF0DDCFBBF0BAC0D9FFBBC0DAFFDF5034
:10BE3800B96FB951D8A423EF5FF025EF5FF029EF70
:10BE48005FF0040EBC6FE5EF5EF020EE0BF0BA5128
:10BE5800D926BB51DA22DFB634EF5FF036EF5FF058
:10BE680055EF5FF0BAC00CF0BBC00DF020EE14F037
:10BE7800B751D926B851DA22DECF0EF0DDCF0FF058
:10BE8800000E116E0B0E106E6CEC69F00C500D105C
:10BE9800D8A451EF5FF053EF5FF055EF5FF0E5EF97
:10BEA8005EF0B7C0A4F0B8C0A5F0000E0001A76FFF
:10BEB800000EA66FE8EC32F00001BC6FBC51D8B49C
:10BEC80068EF5FF06AEF5FF0E9EF5EF0E5EF5EF0D4
:10BED80012002F6C696664617461302E62696E208D
:10BEE800002F6C696664617461312E62696E20008E
:10BEF8002F6C696664617461322E62696E20002F4E
:10BF08006C696664617461332E62696E20002F6CFF
:10BF1800696664617461342E62696E20002F6C69F1
:10BF28006664617461352E62696E20002F6C6966E3
:10BF380064617461362E62696E20002F6C696664D4
:10BF4800617461372E62696E20002F6C69666461C6
:10BF58007461382E62696E20002F6C6966646174A2
:10BF680061392E62696E20002F6C696664617461A4
:10BF7800612E62696E20002F6C696664617461626B
:10BF88002E62696E20002F6C696664617461632E8D
:10BF980062696E20002F6C696664617461642E6248
:10BFA800696E20002F6C696664617461652E626930
:10BFB8006E20002F6C696664617461662E62696E1A
:10BFC8002000000000000000000000000000000049
:10BFD8000000000000000000000000000000000059
:10BFE8000000000000000000000000000000000049
:10BFF8000000000000000000000000000000818E2A
:10C00800819CDA0EF66EBE0EF76E000EF86E0DEE1F
:10C0180034F011EE2CF00900F5CFEEFFE550E150B9
:10C02800FAE1E250F8E15C0EF66EDE0EF76E000EF5
:10C03800F86E03EE80F010EE20F00900F5CFEEFF69
:10C04800E550E150FAE1A40EF66ED80EF76E000E38
:10C05800F86E02EEA4F010EE46F00900F5CFEEFF00
:10C06800E550E150FAE10E0EF66EDF0EF76E000EA7
:10C07800F86E0900F5CFE0F10900F5CFE1F10C0EFB
:10C08800F66EDF0EF76E000EF86E0900F5CF51F070
:10C098000900F5CF52F005EE00F018EE34F0EE6A24
:10C0A800E550E150FCE1E250FAE104EE00F011EE57
:10C0B80000F0EE6AE550E150FCE1E250FAE103EEEF
:10C0C80000F0800EEE6AE806FDE102EE00F0A40E34
:10C0D800EE6AE806FDE101EE00F0A90EEE6AE80658
:10C0E800FDE10001FF6BFE6B00EE49F0080EEE6A01
:10C0F800E806FDE154905492000EF86E0001F5EF49
:10C1080009F0C1C0B7F0C2C0B8F0000E0001BA6FA4
:10C11800010EB96F96EC5DF00001C36FC351D8A44E
:10C1280098EF60F09AEF60F0F7EF60F0C1C0D9FFC8
:10C13800C2C0DAFFDECF3AF0DDCF3BF020EE0EF0E2
:10C14800C151D926C251DA22DECF3CF0DECF3DF014
:10C15800DECF3EF0DECF3FF0AFEC64F00001C36FFE
:10C16800C351D8A4BAEF60F0BCEF60F0F7EF60F00D
:10C1780020EE12F0C151D926C251DA22DECF0CF0DE
:10C18800DDCF0DF0000E0F6E000E0E6E000E116E5C
:10C19800200E106E92EC6DF0000120EE12F0C151ED
:10C1A800D926C251DA22DECF0CF0DDCF0DF020EE19
:10C1B80014F0C151D926C251DA22DECF0EF0DDCFFC
:10C1C8000FF0000E116E0B0E106E07EC6CF0C1C074
:10C1D800D9FFC2C0DAFF10EE04F0DE50E126DD50D0
:10C1E800E222010EE76E0001C3511200DFC0E5F044
:10C1F800E0C0E6F0E50E0C6E000E0D6E51EC59F045
:10C208000CC0E7F00DC0E8F00001E8BF10EF61F0E6
:10C218000EEF61F013EF61F00B0E6EEF61F0D89046
:10C22800E735D96EE835DA6E7E0ED926010EDA22A8
:10C23800DECFE3F0DDCFE4F0E351E411D8B427EF2B
:10C2480061F029EF61F02FEF61F0E3C0D9FFE4C09E
:10C25800DAFF000EDF6EDD51DE11D8B436EF61F083
:10C2680038EF61F03EEF61F0DDC0D9FFDEC0DAFFE4
:10C27800000EDF6ED890E735D96EE835DA6E7E0E9F
:10C28800D926010EDA22DDC0DEFFDEC0DDFFDD517A
:10C29800DE11D8B452EF61F054EF61F05CEF61F059
:10C2A800E105D8B45AEF61F05CEF61F05FEF61F03F
:10C2B800000E6EEF61F0DD0E846F000E856FDF0EED
:10C2C800866F000E876F000E886F37EC01F0000153
:10C2D800E26FE25112000001FF51140D070EF32422
:10C2E800D96E010EF420DA6E000EDE24CB6F010E3B
:10C2F800DE20CC6F000EDE20CD6F000EDE20CE6F6C
:10C30800FF51140D070EF324D96E010EF420DA6ED6
:10C31800CBC0DEFFCCC0DEFFCDC0DEFFCEC0DEFF6F
:10C32800FF51140D070EF324D96E010EF420DA6EB6
:10C33800DECFD0F0DDCFD1F06B0E8A6FF60E8B6FAB
:10C34800CECF8CF08D6BCDCF8EF08F6BD0C090F0B0
:10C35800D1C091F0D0C092F0D1C093F04EEC6FF004
:10C368000001FF51200D040EF324A46F020EF420E7
:10C37800A56FD0C0A6F0D1C0A7F0A86BA96BCDEC73
:10C3880017F00001CF6FCF51D8B4CDEF61F0CFEFE8
:10C3980061F0E0EF61F03D0E8A6FFB0E8B6FD0C04D
:10C3A8008CF0D1C08DF0CFC08EF08F6B4EEC6FF05B
:10C3B800010E4D6EE2EF61F0000E4D6E12000CC0E2
:10C3C80014F00DC015F00EC016F00FC017F01006CF
:10C3D800D8A01106102806E11128D8A4F6EF61F0BC
:10C3E800F8EF61F005EF62F0000E0D6E000E0C6EB6
:10C3F8004DEF62F0144A152A164A172A1006D8A0DB
:10C40800110614C0F6FF15C0F7FF0800F550000923
:10C41800D8B411EF62F013EF62F03AEF62F016C091
:10C42800D9FF17C0DAFFDF50D8B41DEF62F01FEF55
:10C4380062F03AEF62F010501110D8B426EF62F0B3
:10C4480028EF62F03AEF62F016C0D9FF17C0DAFFA2
:10C4580014C0F6FF15C0F7FFDE500900F518D8B470
:10C4680038EF62F03AEF62F0FEEF61F014C0F6FFC9
:10C4780015C0F7FF0800F5CF12F016C0D9FF17C096
:10C48800DAFFDF50136E1350125C0C6E0D6AD8A0E1
:10C498000D06120074EC6DF0CC0EA1EC6EF0660E79
:10C4A800A1EC6EF002EC6EF0296E2950D8A45FEF73
:10C4B80062F061EF62F06BEF62F0000E236E000E27
:10C4C800246E000E256E000E266EB8EF62F0000E88
:10C4D800286E000E276E290E2724D96E000E2820FC
:10C4E800DA6E02EC6EF0DF6E274A282A28BE86EF45
:10C4F80062F0285009E1040E275CD8A086EF62F0AC
:10C5080088EF62F06FEF62F0380E00018A6FFC0E60
:10C518008B6F29C08CF08D6B2AC08EF08F6B2BC06F
:10C5280090F0916B2CC092F0936B29C094F02AC0C4
:10C5380095F02BC096F02CC097F04EEC6FF02C5075
:10C548002B102A1009E10B0E295CD8A0AEEF62F07F
:10C55800B0EF62F061EF62F029C023F02AC024F046
:10C568002BC025F02CC026F012001A0E0E24106ED7
:10C57800000E0F20116E010E1024D96E000E11202E
:10C58800DA6EDF50126E1250146E136A1A0E0E24F1
:10C59800D96E000E0F20DA6EDF50156E155013128B
:10C5A800000E141213C01AF014C01BF01C6A1D6A86
:10C5B8000CC0D9FF0DC0DAFF030EDE18D8A4E7EFD0
:10C5C80062F0E9EF62F017EF63F0140E0E24106EBC
:10C5D800000E0F20116E010E1024D96E000E1120CE
:10C5E800DA6EDF50126E1250146E136A140E0E2497
:10C5F800D96E000E0F20DA6EDF50156E155013102D
:10C60800166E1450176E186A196A17C019F016C0FA
:10C6180018F0176A166A16501A1217501B1218507B
:10C628001C1219501D121AC00CF01BC00DF01CC0B2
:10C638000EF01DC00FF012000F501010D8B427EFE5
:10C6480063F029EF63F032EF63F00F501010D8A4B5
:10C6580030EF63F032EF63F037EF63F00D50FBEC2F
:10C668006EF084EF63F020EE04F00F50D9261050DE
:10C67800DA22DE50DE10D8B444EF63F046EF63F000
:10C6880061EF63F020EE04F00F50D9261050DA2243
:10C6980010EE02F00F50E1261050E222DE50E65C68
:10C6A800E650800A156EDE50800A1558D8B05FEF44
:10C6B80063F061EF63F084EF63F020EE02F00F5057
:10C6C800D9261050DA22DECF11F0DDCF12F00FC0DC
:10C6D800D9FF10C0DAFFDECF13F0DDCF14F0115010
:10C6E8001324D96E12501420DA6E0DC0DFFF20EE2D
:10C6F80002F00F50D9261050DA22DE2A000EDD2271
:10C7080012000DC013F00EC014F013501410D8B45A
:10C7180090EF63F092EF63F0E4EF63F013C0D9FF9A
:10C7280014C0DAFFDE50DE10D8B49DEF63F09FEF3F
:10C7380063F0E4EF63F013C0D9FF14C0DAFFDECF73
:10C748000FF0DDCF10F00FC0D9FF10C0DAFFDF50B7
:10C75800D8B4B1EF63F0B3EF63F0E4EF63F020EE29
:10C7680002F01350D9261450DA2213C0E1FF14C086
:10C77800E2FF00EE06F0E650E926E550EA22DE5038
:10C78800EE1807E1DE50EE18D8A4CDEF63F0CFEF36
:10C7980063F0E4EF63F013C0D9FF14C0DAFF10EEC2
:10C7A80001F0DE50E126DD50E222E7505DEC6FF04B
:10C7B8000F6E0FA0E2EF63F0E4EF63F0E7EF63F0D2
:10C7C800090EE8EF63F0000E120001016EA1EFEF11
:10C7D80063F0F1EF63F0FBEF63F01FC016F020C0C9
:10C7E80017F01DC018F01EC019F098EC6CF022BEAE
:10C7F80000EF64F002EF64F008EF64F021C026F067
:10C8080022C027F00CEF64F0000E276E000E266E93
:10C81800000E256E000E246E1EEF64F0000E0E6EE4
:10C82800200E0D6E1DC00FF01EC010F020EC63F03E
:10C83800244A252A2650245C2550800A236E275036
:10C84800800A2358D8A02BEF64F02DEF64F012EF84
:10C8580064F001016EB133EF64F035EF64F03FEF3F
:10C8680064F01FC016F020C017F01DC018F01EC0DD
:10C8780019F098EC6CF01FC012F020C013F0DFEC38
:10C888006BF0265012241D6E275013201E6E1200C6
:10C89800020E1A5E000E1B5A1C5A1D5A20EE12F088
:10C8A8001850D9261950DA22FE0EDE241E6EFF0E0D
:10C8B800DE201F6EFF0EDE20206EFF0EDE20216EB2
:10C8C8001E501A5C1F501B5820501C5821501D58D0
:10C8D800D8A071EF64F073EF64F07DEF64F0000EA0
:10C8E800186E000E196E000E1A6E000E1B6EAEEF5B
:10C8F80064F020EE26F01850D9261950DA22DECF3F
:10C908001EF0DECF1FF0DECF20F0DECF21F020EECC
:10C9180002F01850D9261950DA22DF50226E225020
:10C928000C6E0D6A0E6A0F6A1AC010F01BC011F067
:10C938001CC012F01DC013F01AEC6AF01E500C2433
:10C94800186E1F500D20196E20500E201A6E21509F
:10C958000F201B6E1200000E446E20EE2AF03A5093
:10C96800D9263B50DA223C50DE180FE13D50DE1844
:10C978000CE13E50DE1809E13F50DE18D8B4C7EF8D
:10C9880064F0C9EF64F00FEF65F03AC025F03BC0E2
:10C9980026F015EC5AF0446E4450D8A4D6EF64F053
:10C9A800D8EF64F00FEF65F02E0E3A241B6E000EE0
:10C9B8003B201C6E3CC01DF03DC01EF03EC01FF069
:10C9C8003FC020F0000E226E010E216E20EE01F015
:10C9D8003A50D9263B50DA22DF5034EC5EF0000999
:10C9E800D8B4F9EF64F0FBEF64F001EF65F03C6850
:10C9F8003D683E683F68010E446E20EE2AF03A50CA
:10CA0800D9263B50DA223CC0DEFF3DC0DEFF3EC0E7
:10CA1800DEFF3FC0DEFF44501200000E866E000E9F
:10CA2800846E8B688968000E01019E6F000E506E3F
:10CA3800000E876F000E866F83928394000EA46F9A
:10CA4800000EA36F200EA66F400EA56F000E856F17
:10CA5800000E846F3AEF65F0000E8425D96E040E3F
:10CA68008521DA6E000EDF6E844B852B85BF43EF80
:10CA780065F08505D8A043EF65F045EF65F030EF28
:10CA880065F0000E856F000E846F55EF65F0340E6B
:10CA98008425D96E0B0E8521DA6E000EDF6E844B6D
:10CAA800852B85BF5EEF65F08505D8A05EEF65F044
:10CAB80060EF65F04BEF65F00F011769D6501F0B5B
:10CAC8004009D66ED6980F0ED612D5980F0ED512ED
:10CAD8000E01C29BD58E1200146E0C0E1418D8B419
:10CAE80078EF65F07AEF65F089EF65F077EC6FF035
:10CAF80053EC6EF00009D8A484EF65F086EF65F07A
:10CB080089EF65F0FF0ECEEF65F0145040097BEC1D
:10CB18006EF011507BEC6EF010507BEC6EF00F5005
:10CB28007BEC6EF00E507BEC6EF0010E136E145021
:10CB3800D8A4A1EF65F0A3EF65F0A5EF65F0950E19
:10CB4800136E080E1418D8A4ACEF65F0AEEF65F0BC
:10CB5800B0EF65F0870E136E13507BEC6EF00C0E81
:10CB68001418D8A4BAEF65F0BCEF65F0BEEF65F015
:10CB78000CEC6FF00A0E136E0CEC6FF0126E12AE26
:10CB8800C8EF65F0CAEF65F0CDEF65F0132EC0EF82
:10CB980065F012501200D5EF65F00C4A0D2A0E4AC6
:10CBA8000F2A0EC0D9FF0FC0DAFFDF50106E0CC07D
:10CBB800F6FF0DC0F7FF000EF86E0E0EF76403D0F7
:10CBC8000800F55005D0F6CFE9FFF7CFEAFFEF50A0
:10CBD8001018D8A4F2EF65F0F4EF65F00DEF66F0E9
:10CBE8000CC0F6FF0DC0F7FF000EF86E0E0EF764CE
:10CBF80003D00800F55005D0F6CFE9FFF7CFEAFFDC
:10CC0800EF500009D8A40BEF66F00DEF66F0D1EFF6
:10CC180065F00CC0F6FF0DC0F7FF000EF86E0E0EA3
:10CC2800F76403D00800F55005D0F6CFE9FFF7CF39
:10CC3800EAFFEF50106E0EC0D9FF0FC0DAFFDF50C9
:10CC4800116E1150105C0C6E0D6AD8A00D06120002
:10CC580025EE04F0DE50DE10D8B435EF66F037EF7D
:10CC680066F02CEF66F000C514F001C515F0060E4D
:10CC78001424D96E050E1520DA6EDF50126E060EDA
:10CC88001424D96E070E1520DA6EDF50136E144A7D
:10CC9800152AFF0E0E6E010E0F6E14C010F015C08F
:10CCA80011F00E5010160F50111610C000F511C0DB
:10CCB80001F5F29E25EE04F0DE06000EDD5AF28E36
:10CCC8000CC0D9FF0DC0DAFF13C0DFFF25EE04F05A
:10CCD800010EDBBE7BEF66F0000EDE5C020EDE5856
:10CCE800D8B079EF66F07BEF66F083EF66F083A249
:10CCF80080EF66F082EF66F083EF66F0898212506B
:10CD0800120062EC51F0CBC0E8F0CCC0E9F00001B1
:10CD1800E851E911D8B493EF66F095EF66F09BEF10
:10CD280066F0E8C0E2F0E9C0E3F0DBEF66F08FB44C
:10CD3800A0EF66F0A2EF66F0BAEF66F0FF51200DA3
:10CD4800040EF324A46F020EF420A56F000EA66F44
:10CD5800040EA76F010EA96F000EA86FE60EAA6F4A
:10CD6800000EAB6F73EC13F00001EC6FEC51D8B40C
:10CD7800C0EF66F0C2EF66F0D1EF66F0940E8A6FEE
:10CD8800FD0E8B6FECC08CF08D6B4EEC6FF0ECC031
:10CD9800E2F00001E36BDBEF66F06FEC61F0010E8F
:10CDA8000101906F000E0001E36F000EE26F1200A8
:10CDB800F7EF66F0030E0E6E2EEF67F0050E0E6E9F
:10CDC800000E0101756F000E746F2EEF67F0010EF3
:10CDD8000E6E2EEF67F0020E0E6E2EEF67F0000E4D
:10CDE8000E6E2EEF67F074C10CF075C10DF00D508A
:10CDF800000AD8B40EEF67F0020AD8B419EF67F04A
:10CE08000F0AD8B420EF67F02A0AD8B427EF67F0E2
:10CE1800F3EF66F00C500A0AD8B4DEEF66F01E0A8B
:10CE2800D8B4E2EF66F0F3EF66F00C50BC0AD8B461
:10CE3800EFEF66F0F3EF66F00C50AC0AD8B4EBEF06
:10CE480066F0F3EF66F00C500F0AD8B42EEF67F0D7
:10CE5800F3EF66F00E501200000E146E000E156E01
:10CE6800000E166E000E176E1050111012101310CF
:10CE7800D8B441EF67F043EF67F079EF67F0010E40
:10CE8800186E4DEF67F0D8901036113612361336FB
:10CE9800182A13AE52EF67F054EF67F047EF67F0C8
:10CEA800D890143615361636173610500C5C1150BB
:10CEB8000D5812500E5813500F58D8A066EF67F04F
:10CEC80068EF67F071EF67F010500C5E11500D5A63
:10CED80012500E5A13500F5A1480D890133212322F
:10CEE80011321032182E54EF67F014C00CF015C030
:10CEF8000DF016C00EF017C00FF01200070E116EDD
:10CF0800D00E106E9FEF67F00CEC6FF0126E1228C7
:10CF1800D8B491EF67F093EF67F095EF67F0A8EF5B
:10CF280067F0E40E00D000D0E82EFCD700D000D087
:10CF38001006D8A0110610501110D8A4A6EF67F05B
:10CF4800A8EF67F088EF67F0FE0E1218D8B4AFEFBD
:10CF580067F0B1EF67F0B4EF67F0000ECEEF67F05F
:10CF68000CEC6FF00CC0D9FF0DC0DAFFDF6E0C4A75
:10CF78000D2A0E06D8A00F060E500F10D8A4C7EF22
:10CF880067F0C9EF67F0B4EF67F00CEC6FF00CECEA
:10CF98006FF0010E1200EE0E00018A6FF90E8B6F12
:10CFA800CECF8CF08D6BCDCF8EF08F6B4EEC6FF0BB
:10CFB8005350FD0B536E340E0C6E0B0E0D6EE50EBA
:10CFC8000E6E020E0F6E000E116E050E106EB7EC8F
:10CFD8006BF0390E0C6E0B0E0D6EC50E0E6E020E3A
:10CFE8000F6E000E116E130E106EB7EC6BF05350EF
:10CFF8000209536E4C0E0C6E0B0E0D6ED80E0E6E93
:10D00800020E0F6E000E116E0D0E106EB7EC6BF067
:10D01800000E246E250E236E45EC3DF05350FD0B9B
:10D02800536E83901200250E00018A6FFB0E8B6FE2
:10D03800CECF8CF08D6BCDCF8EF08F6B4EEC6FF02A
:10D04800000E246E000E236E0001FF51140D070E12
:10D05800F324D96E010EF420DA6EDE6ADE6ADE6A27
:10D06800DD6AFF51140D130EF324D96E010EF4205E
:10D07800DA6E000EDF6EFF51140D0F0EF324D96E19
:10D08800010EF420DA6EDE6ADE6ADE6ADD6A234AA1
:10D09800242A24BE59EF68F0245009E1040E235CC9
:10D0A800D8A059EF68F05BEF68F028EF68F083903C
:10D0B800000E4D6E12004FEC6AF00009D8A467EF1D
:10D0C80068F069EF68F06CEF68F0000EA5EF68F0A3
:10D0D80010507BEC6EF0FD0E1018D8B476EF68F0A7
:10D0E80078EF68F0A4EF68F0020E126E000E116E71
:10D0F8000EC0D9FF0FC0DAFFDF507BEC6EF00E4A8E
:10D108000F2A1106D8A0120611501210D8A48FEFBA
:10D1180068F091EF68F07CEF68F00CEC6FF00CECC5
:10D128006FF00CEC6FF0136E13501F0B050AD8B498
:10D13800A0EF68F0A2EF68F0A4EF68F069EF68F07C
:10D14800010E12001050111012101310D8B4AFEFC6
:10D1580068F0B1EF68F0E1EF68F0010E146EBBEF14
:10D1680068F0D8901036113612361336142A13AEDA
:10D17800C0EF68F0C2EF68F0B5EF68F010500C5CD3
:10D1880011500D5812500E5813500F58D8A0CFEF09
:10D1980068F0D1EF68F0D9EF68F010500C5E1150CC
:10D1A8000D5A12500E5A13500F5AD8901332123289
:10D1B80011321032142EC2EF68F00CC00CF00DC002
:10D1C8000DF00EC00EF00FC00FF0120012C018F0D4
:10D1D80013C019F00BEF69F01606D8A0170614C093
:10D1E800D9FF15C0DAFF144A152A18C0E1FF19C083
:10D1F800E2FF184A192ADFCFE7FFE750D8A407EF64
:10D2080069F009EF69F00BEF69F01EEF69F016504D
:10D218001710D8A412EF69F014EF69F0F0EF68F076
:10D228001EEF69F018C0D9FF19C0DAFF000EDF6ED3
:10D23800184A192A1606D8A01706162806E117282C
:10D24800D8A429EF69F02BEF69F016EF69F0120006
:10D25800246EA10E256EF50E266E000E236E46EF87
:10D2680069F025C0F6FF26C0F7FF254A262A0800E0
:10D27800F5500009D8A443EF69F045EF69F035EFA0
:10D2880069F0232A24502318D8B44DEF69F04FEFE2
:10D2980069F05DEF69F025C0F6FF26C0F7FF0800CA
:10D2A800F5500009D8A45BEF69F05DEF69F035EF40
:10D2B80069F0880E00018A6FFE0E8B6F24C08CF017
:10D2C8008D6B25C08EF026C08FF04EEC6FF01200EB
:10D2D8000CC014F00DC015F00EC016F00FC017F0FA
:10D2E800000E196E000E186E1006D8A01106102830
:10D2F80008E11128D8B483EF69F085EF69F0A4EF4D
:10D3080069F014C0D9FF15C0DAFF144A152ADF5096
:10D31800126E16C0D9FF17C0DAFF164A172ADF5057
:10D32800136E1350125C186E196AD8A0190618509B
:10D338001910D8B4A2EF69F0A4EF69F078EF69F09A
:10D3480018C00CF019C00DF012001F0E00018A6FF2
:10D35800FD0E8B6F4EEC6FF053500209536E2BEE9F
:10D3680034F089C1DFFF000EE8CF35FB0D0EE8CFA2
:10D3780036FB000EE8CF37FB8FA4C5EF69F0C7EF87
:10D3880069F0CAEF69F0600EE8CF37FB8FA4CFEFE2
:10D3980069F0D1EF69F0D7EF69F036CB29F0200EAC
:10D3A800291229C036FB000E246E040E236E45ECAC
:10D3B8003DF05350FD0B536E000E0101896F8390B1
:10D3C80012007CC080F07DC081F0000E0101696F01
:10D3D800000E686F07EF6AF07AC074F07BC075F0D2
:10D3E800800E0001766F000E776F7EC078F07FC0E8
:10D3F80079F05EEC54F000017451010168270001D6
:10D4080075510101692380C0F6FF81C0F7FF08004C
:10D41800F5500009D8A413EF6AF015EF6AF0F0EFA1
:10D4280069F068C17AF069C17BF01200000E146ED1
:10D43800000E156E000E166E000E176E0CA027EF6C
:10D448006AF029EF6AF031EF6AF010501426115093
:10D4580015221250162213501722D8901036113662
:10D4680012361336D8900F320E320D320C320C5061
:10D478000D100E100F10D8A444EF6AF046EF6AF0B2
:10D4880022EF6AF014C00CF015C00DF016C00EF0B3
:10D4980017C00FF01200130E0D6E880E0C6E6BEF96
:10D4A8006AF00CEC6FF0FF0AD8A45DEF6AF05FEF4A
:10D4B8006AF061EF6AF074EF6AF0E40E00D000D011
:10D4C800E82EFCD700D000D00C06D8A00D060C50D2
:10D4D8000D10D8A472EF6AF074EF6AF055EF6AF095
:10D4E8000C500D10D8A47BEF6AF07EEF6AF0010EA5
:10D4F8007FEF6AF0000E120097EF6AF00DC0F6FF9A
:10D508000EC0F7FF000EF86E0E0EF76403D0080089
:10D51800F55005D0F6CFE9FFF7CFEAFFEF501DEC45
:10D528006FF00D4A0E2A0DC0F6FF0EC0F7FF000E71
:10D53800F86E0E0EF76403D00800F55005D0F6CF4C
:10D54800E9FFF7CFEAFFEF500009D8A4AEEF6AF081
:10D55800B0EF6AF082EF6AF01200B5EF6AF00C4A99
:10D568000D2A0CC0F6FF0DC0F7FF0800F5500009A2
:10D57800D8B4C1EF6AF0C3EF6AF0D7EF6AF00CC015
:10D58800F6FF0DC0F7FF0800F550106E116A0E5037
:10D59800101807E10F501118D8A4D5EF6AF0D7EF8B
:10D5A8006AF0B3EF6AF00CC0F6FF0DC0F7FF080091
:10D5B800F5500C6E0D6A12009F0E146EFF0E156E5C
:10D5C80012C016F013C017F0145016261550172263
:10D5D80017500AE11A0E165CD8A0F5EF6AF0F8EFBA
:10D5E8006AF0010EF9EF6AF0000E186E196A185009
:10D5F8001910D8B402EF6BF004EF6BF00AEF6BF080
:10D608005F0E1214126E136A0EEF6BF012C012F056
:10D6180013C013F01200196E19AE15EF6BF017EF67
:10D628006BF02FEF6BF0199E000E0E6E000E0F6E52
:10D63800000E106E000E116E370E70EC65F01A6E4B
:10D64800010E1A642AEF6BF02CEF6BF02FEF6BF0E2
:10D658001A503AEF6BF015C00EF016C00FF017C055
:10D6680010F018C011F0195070EC65F0120073C07A
:10D6780047F074C048F045EC50F00001756F7551E3
:10D68800D8A449EF6BF04BEF6BF063EF6BF073C00E
:10D698000DF074C00EF085EC63F00001756F7551E4
:10D6A800D8A459EF6BF05BEF6BF063EF6BF073C0CE
:10D6B800D9FF74C0DAFF000EDE6E000EDD6E755104
:10D6C8001200860E00018A6F000E8B6F82C08CF0EC
:10D6D80083C08DF0000E8F6F000E8E6F000E916F5D
:10D6E800000E906F8C0E7A6F000E7B6F84C07CF0FA
:10D6F80085C07DF08A0E7E6F000E7F6FE5EC69F0C5
:10D7080000018E518225D96E8F518321DA6E000E69
:10D71800DF6E1200010E126E200E0C180D10D8B418
:10D7280098EF6BF09AEF6BF0B3EF6BF0F70E0E6EAD
:10D73800FF0E0F6E0CC010F00DC011F00E50102629
:10D748000F501122115009E1050E105CD8A0AFEF5F
:10D758006BF0B1EF6BF0B3EF6BF0000E126E12C00E
:10D768000CF00D6A12000EC015F00FC016F00CC0B8
:10D7780013F00DC014F0D1EF6BF015C0D9FF16C02F
:10D78800DAFFDF50126E154A162A13C0D9FF14C0EB
:10D79800DAFF12C0DFFF134A142A1006D8A01106B8
:10D7A800102806E11128D8A4DCEF6BF0DEEF6BF04F
:10D7B800C1EF6BF0120012C014F013C015F0E7EFC0
:10D7C8006BF0124A132A12C0F6FF13C0F7FF000EBF
:10D7D800F86E0E0EF76403D00800F55005D0F6CFAA
:10D7E800E9FFF7CFEAFFEF500009D8A4FEEF6BF08E
:10D7F80000EF6CF0E5EF6BF01450125C126E1550F0
:10D808001358136E12000CC012F00DC013F00EC0A6
:10D8180014F00FC015F01FEF6CF014C0D9FF15C03D
:10D82800DAFF12C0E1FF13C0E2FFDFCFE7FF144ABF
:10D83800152A124A132A1006D8A01106102806E144
:10D848001128D8A42AEF6CF02CEF6CF011EF6CF0D3
:10D8580012000C6E0C50D8B434EF6CF036EF6CF04C
:10D8680045EF6CF07CEC6FF0200EE82EFED77FECD5
:10D878006FF0CC0E00D0E82EFDD700D000D051EFCD
:10D888006CF07CEC6FF0C00E00D0E82EFDD77FEC7A
:10D898006FF0350EE82EFED700F0120080004C41E4
:10D8A80042454C3100000002800000000000000EDC
:10D8B800000068706469736B2E6366670001091263
:10D8C80020010001001700002D119420D00F000145
:10D8D80000000000000000000000099F0280010213
:10D8E800E805310E00018A6FFF0E8B6F4EEC6FF06A
:10D8F800340E0C6E0B0E0D6E000E0F6E000E0E6EBB
:10D90800010E116E000E106ED9EC5AF02BEE34F0A9
:10D918008BC1DFFF000E246E010E236E45EC3DF037
:10D92800000E01018B6F1200000E1C6E000E1B6EA4
:10D93800A9EF6CF01AC00DF00E6A18C00FF019C0EC
:10D9480010F020EC63F01B4A1C2A1B501624D96ED9
:10D958001C501720DA6EDF501A6E1A50D8A4B7EF91
:10D968006CF0B9EF6CF09EEF6CF012000C6E0C507E
:10D97800D8B4C1EF6CF0C3EF6CF0CEEF6CF0000ED2
:10D98800966E4F0E936E2A0E966E400E956E968A80
:10D99800DAEF6CF0000E966E100E966E2A0E966EEA
:10D9A800F00E936E400E956ECBEF6CF0120020EEE9
:10D9B8001AF00C50D9260D50DA220EC0DFFF20EEE7
:10D9C8001BF00C50D9260D50DA220F50DF6E20EED6
:10D9D80014F00C50D9260D50DA2210C0DFFF20EECB
:10D9E80015F00C50D9260D50DA221150DF6E1200B6
:10D9F800E30E00018A6FFE0E8B6F4EEC6FF0340E53
:10DA08000C6E0B0E0D6E000E0F6E000E0E6E010EDC
:10DA1800116E000E106ED9EC5AF02BEE34F08BC15B
:10DA2800DFFF8390000E01018B6F1200340E0C6E25
:10DA38000B0E0D6E000E0F6E000E0E6E010E116EA7
:10DA4800000E106ED9EC5AF0010EE8CF34FB53509B
:10DA58000209536E000E246E010E236E45EC3DF054
:10DA68005350FD0B536E12009150070B0C6E888AB1
:10DA78008DAA41EF6DF043EF6DF046EF6DF00C505D
:10DA8800080F0C6E020E01019719D8A44EEF6DF025
:10DA980050EF6DF054EF6DF00C50FF0A0F0B0C6E49
:10DAA8000C5012009F0E0E6EFF0E0F6E200E0C1003
:10DAB800106E000E0D10116E0E5010260F50112210
:10DAC80011500AE11A0E105CD8A06DEF6DF070EFDE
:10DAD8006DF0010E71EF6DF0000E0C6E0D6A120004
:10DAE8007CEC6FF00A0E0D6EF80EE82EFED70D2EA8
:10DAF800FCD700D07FEC6FF0E00E00D0E82EFDD709
:10DB08003EEC6FF00E6E090E0D6E840EE82EFED7F9
:10DB18000D2EFCD77FEC6FF00E5012000CC012F0E7
:10DB28000DC013F0A0EF6DF012C0D9FF13C0DAFFDB
:10DB38000EC0DFFF124A132A1006D8A011061028BB
:10DB480006E11128D8A4ABEF6DF0ADEF6DF098EFBA
:10DB58006DF012009F0E0E6EFF0E0F6E0CC010F0CF
:10DB68000DC011F00E5010260F50112211500AE16D
:10DB78001A0E105CD8A0C3EF6DF0C6EF6DF0010E61
:10DB8800C7EF6DF0000E0C6E0D6A1200BF0E0E6E20
:10DB9800FF0E0F6E0CC010F00DC011F00E501026C5
:10DBA8000F50112211500AE11A0E105CD8A0DFEFB5
:10DBB8006DF0E2EF6DF0010EE3EF6DF0000E0C6E0C
:10DBC8000D6A1200D00E0E6EFF0E0F6E0CC010F014
:10DBD8000DC011F00E5010260F50112211500AE1FD
:10DBE8000A0E105CD8A0FBEF6DF0FEEF6DF0010E91
:10DBF800FFEF6DF0000E0C6E0D6A1200000E0E6E37
:10DC0800000E0F6ED8900E32B4EC6EF00009D8B446
:10DC180010EF6EF012EF6EF013EF6EF00E8E0F2A0B
:10DC2800070E0F641AEF6EF01CEF6EF006EF6EF041
:10DC38000E50120060900F0E0F01596F070E396FCA
:10DC4800070E356F4F0E936E000E8A6E8A888A8291
:10DC58008A82000E8F6E130E0E01B76F0F0EFA6FC9
:10DC6800100EFC6F140EB86F12009F869E84090E6A
:10DC78000E01FD6F9F98890E9B6E000E9C6E9E98FC
:10DC88009D8E9D889D9AC599F28AF28E9E909D9C44
:10DC98009E9A9E8A01019191000E926F120084EC67
:10DCA8006FF00CEC6FF04FEC6AF00009D8B45FEF3E
:10DCB8006EF061EF6EF064EF6EF0010E67EF6EF0DC
:10DCC80077EC6FF0000E1200000EE8CF00F5000EA2
:10DCD800E8CF01F5000EE8CF02F5000EE8CF03F516
:10DCE800000EE8CF04F5000EE8CF05F512000C6E23
:10DCF8000CC092FF95B083EF6EF085EF6EF07EEF6B
:10DD08006EF095A08AEF6EF08CEF6EF085EF6EF0F6
:10DD1800925012000C500E02F3CF10F0F4CF11F015
:10DD28000C500F02F35011260D500E02F35011261D
:10DD380010C00CF011C00DF012000D6E000E0E6E2A
:10DD48000D50010B2DEC6CF0D8900D320E2A070EF9
:10DD58000E64B1EF6EF0B3EF6EF0A4EF6EF0120048
:10DD68007CEC6FF0200EE82EFED77FEC6FF0300EC3
:10DD7800E82EFED73EEC6FF00D6EB00E00D0E82E08
:10DD8800FDD70D501200070E00018A6FFF0E8B6F32
:10DD98004EEC6FF0000E4C6E000E4B6E000E4A6E8D
:10DDA8008390000E01018B6F12000C6EDEEF6EF097
:10DDB800838C839C0C060C28D8A4E5EF6EF0E7EF63
:10DDC8006EF0DCEF6EF000F000F01200000E0101C2
:10DDD8008D6F000E8C6F000E736F000E726F020E47
:10DDE8008B6F8390000E8A6F000E896F12000C6E85
:10DDF80001EF6FF089EC6FF004000E01CDA907EF79
:10DE08006FF009EF6FF0FEEF6EF00CC09AFF120092
:10DE1800926895B012EF6FF014EF6FF00DEF6FF09E
:10DE280095A019EF6FF01BEF6FF014EF6FF09250A1
:10DE380012000C6E23EF6FF089EC6FF004000E01F6
:10DE4800CDA929EF6FF02BEF6FF020EF6FF00CC02A
:10DE58009AFF12004D5946494C453132333400017E
:10DE68000000000100002000131012000000010053
:10DE78000000000088888DA844EF6FF046EF6FF02F
:10DE88004AEF6FF0010E0C6E4CEF6FF0000E0C6E47
:10DE98000C5012008C0E216E000E226E8AC019F0F2
:10DEA8008BC01AF0210E1B6E000E1C6E1BEC25F0A9
:10DEB80012000C6E0C50D8B464EF6FF066EF6FF080
:10DEC80069EF6FF0010E6AEF6FF051501200838016
:10DED800010E4D6E000E4D6E8390120004C50CF0BD
:10DEE80005C50DF0120082EC6FF00CEC6FF012001B
:10DEF8008398889812008398888812008F8012006F
:0CDF08008F90120001E7340B1200120091
:10F5A000004F4B004449534B5F455252004E4F545D
:10F5B0005F5245414459004E4F5F46494C45004E0D
:10F5C0004F545F4F50454E4544004E4F545F454E9B
:10F5D00041424C4544004E4F5F46494C455F5359AC
:10F5E0005354454D00000D0A20253258202532582D
:10F5F0002025327320253273202532732025327363
:10F600002025327320253273202532732025327352
:10F61000202534732025347320253473202534733A
:10F62000202534732025347320253473202534732A
:10F6300020000D0A253032582530325820535338D7
:10F64000303A53657420537461747573206D61731F
:10F650006B2025582025582025582025582025582E
:10F6600020255820255820255820000D0A25303205
:10F67000582530325820535338303A20496E63723F
:10F68000656D656E743A205365656B696E672074AD
:10F690006F20256C642028256C582920000D0A480D
:10F6A000504469736B204D6B2049492028313846FE
:10F6B00034364B34302920257320257320257320C0
:10F6C0005374617274696E672E2E2E0D0A000D0A36
:10F6D00025303258253032582053533830783A5339
:10F6E00065656B3A205365656B696E6720746F20A2
:10F6F000256C752028256C582920000D0A414D3AAB
:10F70000556E6275666620726420632F682F733AA7
:10F710002025642F25642F256420733A256C6420EE
:10F72000000D0A25303258253032582053533830D6
:10F730003A4275666620777220256C64206279747F
:10F74000657320727820000D0A5472696564207414
:10F750006F2074616C6B207768696C7374206E6FB6
:10F760007420616464726573736564000D0A414DB1
:10F770003A4275666620726420632F682F733A20C0
:10F7800025642F25642F256420733A256C6420009E
:10F790000D0A414D3A4275666620777220632F68E4
:10F7A0002F733A2025642F25642F256420733A2572
:10F7B0006C64000D0A253032582530325820313A19
:10F7C000526561642072746E2025582C20256420B7
:10F7D0007265616420000D0A253032582530325898
:10F7E0002053533830783A577269746520256C6419
:10F7F0002028256C582920000D0A25303258253044
:10F8000032582053533830783A5374617475732CDE
:10F8100020756E697420256420000D0A52656164AC
:10F820002072657475726E732025582C2025642013
:10F8300062797465732072656164000D0A25303247
:10F8400058253032582053533830783A5265616425
:10F8500020256C752028256C582920000D0A25309C
:10F8600032582530325820535338303A536574207B
:10F870006164647265737320256C5820000D0A253D
:10F880003032582530325820535338303A436820AC
:10F89000696E6420436C65617220256420000D0A46
:10F8A0004D617820566563746F72206469736B20B4
:10F8B000256420256C642028256C582920000D0A19
:10F8C00025303258253032582053533830783A5347
:10F8D00074617475735B25645D20255820000D0AE2
:10F8E000253032582530325820535338303A53653A
:10F8F00074206C656E67746820256C5820000D0AB2
:10F90000253032582530325820535338303A416D23
:10F9100069676F20436C65617220256420000D0AC1
:10F92000414D3A205365656B3A20256420256420BB
:10F9300025642025642C20733A256C64000D0A256B
:10F940003032582530325820535338303A5365748A
:10F9500020766F6C756D6520256420000D0A2530BA
:10F9600032582530325820535338303A5270742070
:10F97000515354415420256420000D0A44736B7385
:10F98000656C2069732025642C206E756D6265722C
:10F9900020697320256420000D0A25303258253057
:10F9A000325820566563746F7220256C64202825B8
:10F9B0006C582920000D0A25303258253032582045
:10F9C000535338303A53657420756E69742025643A
:10F9D00020000D0A25303258253032582053533834
:10F9E000303A556E6B6E6F776E20255820000D0AE9
:10F9F00025303258253032582053533830783A4425
:10FA00006573637269626520000D0A2530325825DE
:10FA100030325820535338303A496E697420646943
:10FA2000736B20000D0A2530325825303258205390
:10FA30005338303A52712073746174757320000D1D
:10FA40000A414D3A20496E63723A202564202564AC
:10FA50002025642025642C20000D0A323A5265616D
:10FA6000642072746E2025582C20256420726561F4
:10FA70006420000D0A253032582530325820535367
:10FA800038303A446573637269626520000D0A2557
:10FA900030325825303258202564206279746573DD
:10FAA0002073656E742000466F756E6420616E2051
:10FAB0005254432066696C652061742025580D0AF4
:10FAC000004C6F6F6B696E6720666F7220616E20ED
:10FAD0005254432066696C650D0A000D0A414D3A87
:10FAE000427566662077722025642062797465739A
:10FAF0002072780046696E6446696C6520666169AB
:10FB00006C6564207365617263680D0A000D0A47B5
:10FB10005049422072633A2564202564206279743A
:10FB200065730D0A000D0A253032582530325820F1
:10FB300053533830783A436C65617220000D0A5394
:10FB400065656B20746F20256C64206661696C6547
:10FB500064202564000D0A57726974655F736563DC
:10FB6000746F7273206661696C202564000D0A440D
:10FB700069736B2073656C656374206E756D626567
:10FB800072202564000D0A5365656B696E672074E9
:10FB90006F20256C642028256C5829005365656BFF
:10FBA000696E6720746F20736563746F72202558C7
:10FBB0000D0A0046696E6446696C65206661696C71
:10FBC000656420726561640D0A000D0A25303258A3
:10FBD0002530325820535338303A577269746520B3
:10FBE000000D0A4F70656E696E67206578697374E1
:10FBF000696E6720257320000D0A253032582530A4
:10FC0000325820535338303A5265616420000D0A4F
:10FC1000253032582530325820535338303A445327
:10FC20004A20000D0A2530325825303258205353CF
:10FC300038303A4E4F50200025582025582025585E
:10FC400020255820256C752020200A000D0A72639B
:10FC50002025582C2025642062797465730D0A00D4
:10FC60000D0A566563746F7220256C642028256C1C
:10FC7000582920004469736B206368616E67653A98
:10FC800020256420200D0A000D0A4469736B20535F
:10FC900074617475733A2025582C20000D0A576141
:10FCA0006974696E6720666F7220636172642000F8
:10FCB0003C6964656E743E202558202558202564D3
:10FCC000202564000D0A46696C6520257320697340
:10FCD000206F70656E20000D0A20256C642062790B
:10FCE0007465732073656E74000D0A52656164203B
:10FCF0006265796F6E6420656E64000D0A536565F8
:10FD00006B206265796F6E6420656E64000D0A4F2A
:10FD100070656E696E67206E657720257320000D13
:10FD20000A414D3A53656E642073746174757300B3
:10FD30004E6F742061204C4946206469736B0D0A34
:10FD4000000D0A545844415441206C656E202564CE
:10FD500020000D0A46696C6520255820697320250E
:10FD60007320000D0A4469736B20255820697320A5
:10FD7000257320000D0A486F737420627974653210
:10FD8000202564000D0A486F7374206279746573CE
:10FD9000202564000D0A5772697465206661696CDC
:10FDA000202564000D0A52656164696E6720525413
:10FDB000430D0A000D0A416D69676F2039313231F8
:10FDC000440D0A000D0A53532F3830203931323296
:10FDD000440D0A000D0A44736B73656C206973202F
:10FDE000256420000D0A5265616420256420627933
:10FDF00074657300566563746F72206973202558AB
:10FE00000D0A00222A2B2C3A3B3C3D3E3F5B5D7C99
:10FE10007F000D0A4F70656E696E67202573202084
:10FE2000000D0A446562756720697320256420000F
:10FE30000D0A50726F746F20697320256420000DC5
:10FE40000A5265616420636F6E66696720000D0A5F
:10FE500046696C656E616D652025732000204154F4
:10FE60004E20617373657274656420000D0A466FDD
:10FE7000726D617474696E6720000D0A56616C754D
:10FE8000653A2025580D0A0072633D2575204652BB
:10FE90005F25730D0A002A2A20566572696679204B
:10FEA0002A2A000D0A4E6F206361726420256400C7
:10FEB0002F6C6966646174612E62696E000D0A259B
:10FEC000732025582025580D0A007B5050256420AA
:10FED00025642025647D000D0A73627974657320A2
:10FEE0002564000D0A414D3A57616B657570000D30
:10FEF0000A4D6F756E74696E6720004A616E20321C
:10FF0000352032303230000D0A414D3A436C656184
:10FF1000720068706469736B2E63666700466D7467
:10FF2000206578697420005B535251206F66665DCE
:10FF3000000D0A414D3A44534A0031313A35323AC4
:10FF40003137005B2532582025645D005B535251E8
:10FF5000206F6E5D005B25582025645D0072633D57
:10FF6000256420002D3E20255820005458446174FB
:10FF7000610044534B53454C004E414D45255800BC
:10FF80004449534B2558005B4D4C415D004445426C
:10FF900055470050524F544F002025303258007BB7
:10FFA0004552527D004946432000454F49200052AA
:10FFB000454E200041544E200053525120004441F0
:10FFC0005620004E444143004E52464400302E39E4
:10FFD00000525443002025580025325800207C2030
:10FFE00000443000443100443200443300443400C3
:0FFFF0004435004436004437002563002E0000DE
:020000040020DA
:10000000FF0FFF0FFF0FFF0FFF0FFF0FFF0FFF0F80
:020000040030CA
:0C0000008CFFFFFF9FFFFFFFFFFFFFFFD3
:00000001FF
